:040C0000B8EF5AF0FF
:080C0800046ED8CF05F0E0CF27
:100C100006F00001E9CF0CF0EACF07F0E1CF08F0D1
:100C2000E2CF09F0D9CF0AF0DACF0BF0F3CF12F010
:100C3000F4CF13F0FACF14F0F5CF15F0F6CF16F08D
:100C4000F7CF17F000C00EF001C00FF002C010F097
:100C500003C011F09DA030EF06F09EB063EF06F0E8
:100C6000A0A236EF06F0A1B26BEF06F0F2A83CEFBF
:100C700006F0F2B286EF06F00EC000F00FC001F0F1
:100C800010C002F011C003F00CC0E9FF07C0EAFF7A
:100C9000078E08C0E1FF09C0E2FF0AC0D9FF0BC000
:100CA000DAFF12C0F3FF13C0F4FF14C0FAFF15C03F
:100CB000F5FF16C0F6FF17C0F7FF045006C0E0FFAF
:100CC00005C0D8FF1000B10ECF6EE00ECE6E1980B9
:100CD0009E903CEF06F0010E01016327000E642395
:100CE00064530AE163511F080DE2FF0A05E16253F4
:100CF00003E16151000806E21992646B080E636F0C
:100D0000626B616BA19200013CEF06F001015C2B6C
:100D10005C5109081AE2B2500701676F675101017F
:100D200061255D6F0701B350010162215E6F000E06
:100D300063215F6F000E6421606F5C6BB36AB26AFF
:100D4000646B636B626B616B1982F29200013CEF22
:100D500006F0070141514303F3CF01F0F4CF00F057
:100D60004403F350002642514303F3500020026E27
:100D7000000112000601C86BC76BC96BC66BC56B5F
:100D8000C651030818E303E1C551230814E3F2CF69
:100D9000CFF6F29EC6C675FFC5C674FF7F9C7F9EC8
:100DA0007F807350CFBFF28EC727000EC823C52B9C
:100DB000D8B4C62BE5D7C71FC81F010EC727000E22
:100DC000C823F2CFCFF6F29E030E756E250E746E19
:100DD0007F9C7F9E7F807350CFBFF28ED06FF2CF0B
:100DE000D1F6F29E030E756E240E746E7F9C7F9E6C
:100DF0007F807350D1BFF28ED26FD0C603F0D25134
:100E0000C75D03E10350C85D03E0010EC96F9B6F2E
:100E1000F2CFCFF6F29E756A746A7F9C7F9E7F80C8
:100E20007350CFBFF28EFD0803E2020EC96F9B6FB5
:100E3000F2CFCFF6F29E756A010E746E7F9C7F9E94
:100E40007F807350CFBFF28E030804E2020EC96F99
:100E5000030E9B6FC66BC56BC65320E1C5510308DB
:100E60001DE3030EC525CF6F000EC621D06FF2CF54
:100E7000D1F6F29ED0C675FFCFC674FF7F9C7F9ED1
:100E80007F807350D1BFF28E1F0804E2020EC96F3B
:100E9000040E9B6FC52BD8B4C62BDED7F2CFCFF68E
:100EA000F29E756A3F0E746E7F9C7F9E7F807350AA
:100EB000CFBFF28E0A0804E2020EC96F050E9B6FC7
:100EC000C953D8A40CD1CB6BCA6BCBC642F7CAC6E8
:100ED00041F70701446B8F0E436F00013ADF02C0F8
:100EE00003F00150500F0601CF6F000E0320D06FAA
:100EF000F2CFD1F6F29ED0C675FFCFC674FF7F9CAD
:100F00007F9E7F807350D1BFF28ECE6FCE53D8B408
:100F1000DBD0CE5108080EE2030ECA25C96FCA35D0
:100F2000026ECB35036E02360336FC0E02160250FB
:100F3000060F9B6FCBC642F7CAC641F70701446B49
:100F40008F0E436F000105DF02C003F00150500F08
:100F50000601CF6F000E0320D06F070ECF27000EC3
:100F6000D023F2CFD1F6F29ED0C675FFCFC674FF64
:100F70007F9C7F9E7F807350D1BFF28ECC6FCBC69B
:100F800042F7CAC641F70701446B8F0E436F000159
:100F9000E0DE02C003F00150500F0601CF6F000EDB
:100FA0000320D06F080ECF27000ED023F2CFD1F64A
:100FB000F29ED0C675FFCFC674FF7F9C7F9E7F8058
:100FC0007350D1BFF28ECD6FCC513F0807E3CD51A6
:100FD000200804E3CD51CC2540080EE2030ECA25BB
:100FE000C96FCA35026ECB35036E02360336FC0E6E
:100FF00002160250070F9B6FCBC642F7CAC641F7D5
:101000000701446B8F0E436F0001A3DE02C003F0A3
:101010000150500F0601CF6F000E0320D06F830EDA
:10102000CF27000ED023F2CFD1F6F29ED0C675FFA7
:10103000CFC674FF7F9C7F9E7F807350D1BFF28E9E
:101040000C080EE2030ECA25C96FCA35026ECB35F5
:10105000036E02360336FC0E02160250080F9B6F19
:10106000CBC642F7CAC641F70701446B8F0E436FE8
:1010700000016FDE02C003F00150500F0601CF6F78
:10108000000E0320D06F830ECF27000ED023F2CFA7
:10109000D1F6F29ED0C675FFCFC674FF7F9C7F9EAF
:1010A0007F807350D1BFF28E01080EE3030ECA2574
:1010B000C96FCA35026ECB35036E02360336FC0E9D
:1010C00002160250090F9B6FCA2BD8B4CB2BC95301
:1010D00006E1CB5304E1CA510308D8B0F6D6C95390
:1010E00041E1F2CFCFF6F29E020E756E8C0E746E59
:1010F0007F9C7F9E7F807350CFBFF28ECE6FCE538A
:1011000031E0CE51030804E2070EC96F160E9B6F43
:10111000F2CFCFF6F29E020E756E970E746E7F9C24
:101120007F9E7F807350CFBFF28ECC6FF2CFCFF611
:10113000F29E020E756E980E746E7F9C7F9E7F806D
:101140007350CFBFF28ECD6FCC513F0807E3CD5126
:10115000200804E3CD51CC25400804E2070EC96FF6
:10116000170E9B6FC953D8A4A3D0CB6BCA6BCA35DB
:10117000026ECB35036E0236033602360336023674
:10118000033602360336E00E02160250B40FCF6F5C
:10119000020E0320D06FF2CFD1F6F29ED0C675FFBB
:1011A000CFC674FF7F9C7F9E7F807350D1BFF28E2D
:1011B000CE6FCE3D01D071D0CE5104080AE2080EA8
:1011C000CA25C96FD890CA35026ECB350250180FA8
:1011D0009B6FCA35026ECB35036E0236033602367C
:1011E00003360236033602360336E00E021602508C
:1011F000B40FCF6F020E0320D06F060ECF27000E64
:10120000D023F2CFD1F6F29ED0C675FFCFC674FFC1
:101210007F9C7F9E7F807350D1BFF28ECC6FCA358A
:10122000026ECB35036E02360336023603360236C3
:10123000033602360336E00E02160250B40FCF6FAB
:10124000020E0320D06F050ECF27000ED023F2CF61
:10125000D1F6F29ED0C675FFCFC674FF7F9C7F9EED
:101260007F807350D1BFF28ECD6FCC513F0807E322
:10127000CD51200804E3CD51CC2540080EE2D89092
:10128000CA35026ECB350250080FC96FD890CA35E7
:10129000026ECB350250190F9B6FCA2BD8B4CB2BE3
:1012A000C95306E1CB5304E1CA510108D8B05FD756
:1012B000C9533BE1F2CFCFF6F29E020E756EF40EEB
:1012C000746E7F9C7F9E7F807350CFBFF28ECE6FF7
:1012D000CE532BE0F2CFCFF6F29E030E756E090EC1
:1012E000746E7F9C7F9E7F807350CFBFF28ECC6FD9
:1012F000F2CFCFF6F29E020E756EA20E746E7F9C38
:101300007F9E7F807350CFBFF28ECD6FCC513F0850
:1013100007E3CD51200804E3CD51CC25400805E278
:101320000A0ECA25C96F1D0E9B6FC95313E1F2CF78
:10133000CFF6F29E030E756E1C0E746E7F9C7F9E20
:101340007F807350CFBFF28E0A0804E20B0EC96F84
:101350001E0E9B6FC9C601F000011200010E0601AE
:10136000CF5DFC0FD8B035D1040F0001EBEF0AF0D0
:101370000601D051010A00010FE0030A14E0010A3E
:1013800018E0070A1CE0010A20E0030A1EE0010A37
:1013900029E00F0A27E031D0959A8C9A939A8A9A7D
:1013A00095908C902FD0958A939A8A9A95908C904C
:1013B00029D0958A939A8A9A95908C8023D0958A81
:1013C000939A8A8A95908C901DD0959A8C9A939A2C
:1013D0008A9A95908C800301126B116B106B0F6BC6
:1013E000000110D0958A939A8A9A95908C80030177
:1013F000126B116B106B0F6B0001958A939A8A9A8E
:1014000095908C800601E5D00601D051010A0001BB
:101410000FE0030A14E0010A18E0070A1CE0010AC1
:1014200020E0030A1EE0010A29E00F0A27E031D07C
:1014300094908B9094928B9295928C922FD09480D2
:1014400094928B9295928C9229D0948094928B92C4
:1014500095928C8223D0948094928B8295928C92D8
:101460001DD094908B9094928B9295928C820301D4
:10147000166B156B146B136B000110D09480949253
:101480008B9295928C820301166B156B146B136B08
:101490000001948094928B9295928C82060199D04F
:1014A0000601D051010A00010FE0030A14E0010A0D
:1014B00018E0070A1CE0010A20E0030A1EE0010A06
:1014C00029E00F0A27E031D0949A8B9A949C8B9C48
:1014D00095948C942FD0948A949C8B9C95948C9406
:1014E00029D0948A949C8B9C95948C8423D0948A44
:1014F000949C8B8C95948C941DD0949A8B9A949CEC
:101500008B9C95948C8403011A6B196B186B176B69
:10151000000110D0948A949C8B9C95948C84030138
:101520001A6B196B186B176B0001948A949C8B9C37
:1015300095948C8406014DD00601D051010A00011A
:101540000FE0030A14E0010A18E0070A1CE0010A90
:1015500020E0030A1EE0010A29E00F0A27E031D04B
:1015600094968B9694988B9895968C962FD094867B
:1015700094988B9895968C9629D0948694988B986D
:1015800095968C8623D0948694988B8895968C9685
:101590001DD094968B9694988B9895968C86030183
:1015A0001E6B1D6B1C6B1B6B000110D094869498F6
:1015B0008B9895968C8603011E6B1D6B1C6B1B6BA9
:1015C0000001948694988B9895968C86060101D09C
:1015D000060100011200E824F76AF736F10FF66EF3
:1015E000150EF7220A00F550FA6E0800F550F96E54
:1015F00070130814A0143815016A026A006A036A9D
:101600000601F45102E1F35118E0100EF56FD89085
:10161000F137F23700360336F451035C02E1F3513F
:10162000005C07E3F351005ED8A00306F451035EAB
:10163000D88001360236F52FEAD7000112008E0E4F
:10164000006E54C701F053C702F0036A015209E16A
:1016500002C001F0026A080E005E015202E1006A57
:1016600008D0D89001BE04D0023601360006F9D762
:10167000019E12000601C66BC56BC65336E1C5510B
:10168000030833E3C6C642F7C5C641F70701446BFA
:101690008F0E436F0001A9EC06F002C003F0015069
:1016A000500F0601C86F000E0320C96FF2CFCAF6B3
:1016B000F29EC9C675FFC8C674FF7F9C7F9E7F805F
:1016C0007350CABFF28EC76F010EC525C86F000EDA
:1016D000C621C96FC8C6CFF6C7C6D0F600013EDE28
:1016E0000601C52BD8B4C62BC8D7F2CFC8F6F29ED8
:1016F000756A450E746E7F9C7F9E7F807350C8BF55
:10170000F28E0101746F745324E0FF0ED88074557B
:10171000006E0F0ED8A0E806036E00C0C8F60601E2
:10172000C96F0F0EF26FF16903C0F4F600C0F3F653
:10173000000162DF02C054F701C053F700017FDFF0
:1017400003C073F102C072F101C071F100C070F109
:1017500001010001B1EF5BF00601CA39700B006EA8
:10176000D89000361F0E6F1400106F6E6ECF00F011
:10177000003A0030070BCA5DF9E1000112000601D2
:10178000CA51000A000107E0010A0BE0030A0FE05A
:10179000010A13E019D0C00E0E0143150F09436F63
:1017A00018D0C00E0E0143150709436F12D0C00EAA
:1017B0000E0143150309436F0CD0C00E0E014315F3
:1017C0000109436F06D00001C00E0E014315070941
:1017D000436F3F0E4315436FF80E44150209446FE3
:1017E000C70E44152809446F449D448FF80E4515D3
:1017F0000509456F459D0001B4EF0CF00601FE534D
:1018000060E0F9C603F0F8C6E9FF03C0EAFFFAC6D4
:10181000EFFFF851D8B4F907F807F9C603F0F8C696
:10182000E9FF03C0EAFFFBC6EFFFF851D8B4F907A0
:10183000F807F9C603F0F8C6E9FF03C0EAFFFC5158
:10184000030BEF6EF9C603F0F8C6E9FF03C0EAFF29
:10185000FCC600F0003600360036F80E00160050C8
:10186000E00BEF10EF6EF9C603F0F8C6E9FF03C016
:10187000EAFFEF500809EF6EF851D8B4F907F807FE
:10188000F9C603F0F8C6E9FF03C0EAFFFCC600F0A2
:10189000003A0032070E00160050070BEF6EF9C633
:1018A00003F0F8C6E9FF03C0EAFFFDC600F000360A
:1018B00000360036F80E00160050F80BEF10EF6EF1
:1018C00049D0F9C603F0F8C6E9FF03C0EAFFEF6AA2
:1018D000F851D8B4F907F807F9C603F0F8C6E9FFDC
:1018E00003C0EAFFEF6AF851D8B4F907F807F9C660
:1018F00003F0F8C6E9FF03C0EAFFFAC600F0003AB9
:101900000036E00E00160050E00BEF6EF851D8B430
:10191000F907F807F9C603F0F8C6E9FF03C0EAFFC4
:10192000FAC600F00032003200321F0E00160050DE
:101930001F0BEF6EF9C603F0F8C6E9FF03C0EAFF1C
:10194000FBC600F0003A0036E00E00160050E00B37
:10195000EF10EF6E00011200040E0601CA6F0001C5
:10196000FBDEC9C6CAF60BD70601A36B606A9F0EE1
:101970006014606E608460CF30FF709A7098709EC3
:10198000709C0E0EF96FFB0EF86FFD6BFC6BFB6B22
:10199000FA6B010EFE6F000131DF0E0E0601F96FCA
:1019A000F869FD6BFC6BFB6BFA6B010EFE6F0001BF
:1019B00025DF0E0E0601F96FE30EF86FFD6BFC6B71
:1019C000FB6BFA6B010EFE6F000118DF0E0E0601B5
:1019D000F96FE70EF86FFD6BFC6BFB6BFA6B010E9A
:1019E000FE6F00010BDF0E0E0601F96FEB0EF86FB4
:1019F000FD6BFC6BFB6BFA6B010EFE6F0001FEDEF4
:101A00000E0E0601F96FEF0EF86FFD6BFC6BFB6BB2
:101A1000FA6B010EFE6F0001F1DE0E0E0601F96F8A
:101A2000F30EF86FFD6BFC6BFB6BFA6B010EFE6F38
:101A30000001E4DE0E0E0601F96FF70EF86FFD6B84
:101A4000FC6BFB6BFA6B010EFE6F0001D7DE0E0E16
:101A50000601F96F4B0EF86FFD6BFC6BFB6BFA6BBD
:101A6000010EFE6F0001CADE0E0E0601F96F4F0E69
:101A7000F86FFD6BFC6BFB6BFA6B010EFE6F0001E8
:101A8000BDDE0E0E0601F96F530EF86FFD6BFC6B99
:101A9000FB6BFA6B010EFE6F0001B0DE0E0E06014D
:101AA000F96F570EF86FFD6BFC6BFB6BFA6B010E59
:101AB000FE6F0001A3DE0E0E0601F96F5B0EF86FDC
:101AC000FD6BFC6BFB6BFA6B010EFE6F000196DE8B
:101AD0000E0E0601F96F5F0EF86FFD6BFC6BFB6B72
:101AE000FA6B010EFE6F000189DE0E0E0601F96F22
:101AF000630EF86FFD6BFC6BFB6BFA6B010EFE6FF8
:101B000000017CDE0E0E0601F96F670EF86FFD6BAB
:101B1000FC6BFB6BFA6B010EFE6F00016FDE0E0EAD
:101B20000601F96F6B0EF86FFD6BFC6BFB6BFA6BCC
:101B3000010EFE6F000162DE0E0E0601F96F6F0EE0
:101B4000F86FFD6BFC6BFB6BFA6B010EFE6F000117
:101B500055DE9350FB0B08090601936ECA6B00011A
:101B6000FBDD12000601C52D09D0010EC96F000171
:101B7000F3DE1B6A959C8C9C37D00601F2CFC7F62A
:101B8000F29E756A010E746E7F9C7F9E7F807350FB
:101B9000C7BFF28EC86FC8C6C9F60001DDDEF2CF3E
:101BA000C7F6F29E756A746A7F9C7F9E7F80735031
:101BB0000601C7BFF28E1B6E1B50FD0801E21B6AB7
:101BC000F2CFC7F6F29E756A460E746E7F9C7F9EBA
:101BD0007F807350C7BFF28E000A03E1959C8C8C06
:101BE00002D0959C8C9C00010601C66BC6510A0868
:101BF0000EE3D890C635036A340FE96E000E032059
:101C0000EA6EEC6AED52C6C6EFFFC62BEFD70001B5
:101C100012000601C56BC551070817E3C551040D35
:101C2000F350036A340FE96E010E0320EA6EEF6A87
:101C3000EC6AEC6AEC6A036AC551540FE96E010E56
:101C40000320EA6EEF68C52BE6D70001B8EF5BF022
:101C50000601C56BC5510308D8A086D0C551040D37
:101C6000F350C76BC66F570EC625E96E060EC72127
:101C7000EA6EC5518F0DF350500F190FCA6FF2CF96
:101C8000CBF6F29E756ACAC674FF7F9C7F9E7F80EA
:101C90007350CBBFF28EEC6AED52EF6EC551040D5E
:101CA000F350C76BC66F570EC625E96E060EC721E7
:101CB000EA6EECCF42F7ED52EFCF41F70701446BEC
:101CC000630E436F0001A9EC06F001C0EFFF02C0F4
:101CD000ECFF0601C551040DF350C76BC66F020E31
:101CE000C625016E000EC721036E0150570FE96E25
:101CF000060E0320EA6EC5518F0DF350500F200FD2
:101D0000C86FF2CFC9F6F29E756AC8C674FF7F9C91
:101D10007F9E7F807350C9BFF28EEC6AED52EF6EEA
:101D2000C551040DF350C76BC66F020EC625016E78
:101D3000000EC721036E0150570FE96E060E0320F7
:101D4000EA6EECCF42F7ED52EFCF41F70701446B5B
:101D5000630E436F0001A9EC06F001C0EFFF02C063
:101D6000ECFF0601C52B76D70001BAEF5BF0F2CF8E
:101D7000C7F6F29E020E756EB40E746E7F9C7F9E47
:101D80007F8073500601C7BFF28EC56FF2CFC7F6D2
:101D9000F29E020E756EB50E746E7F9C7F9E7F80E4
:101DA0007350C7BFF28EC66FC551030803E0C5511B
:101DB000040840E1F2CFC7F6F29E020E756EB80E2F
:101DC000746E7F9C7F9E7F807350C7BFF28EC86FFA
:101DD000F2CFC9F6F29E020E756EB70E746E7F9C3E
:101DE0007F9E7F807350C9BFF28ECA6FF2CFCBF651
:101DF000F29E020E756EB60E746E7F9C7F9E7F8083
:101E00007350CBBFF28ECC6F6F6BC8C66EF6CAC66E
:101E10006DF6CCC66CF6F2CFC7F6F29E020E756E6A
:101E2000CF0E746E7F9C7F9E7F807350C7BFF28EF3
:101E3000746F04D06F696E696D696C69F2CFC7F613
:101E4000F29E020E756ED40E746E7F9C7F9E7F8014
:101E50007350C7BFF28EC56FF2CFC7F6F29E020E67
:101E6000756ED50E746E7F9C7F9E7F807350C7BF4A
:101E7000F28EC66FC551030803E0C551040840E166
:101E8000F2CFC7F6F29E020E756ED80E746E7F9C6E
:101E90007F9E7F807350C7BFF28EC86FF2CFC9F6A6
:101EA000F29E020E756ED70E746E7F9C7F9E7F80B1
:101EB0007350C9BFF28ECA6FF2CFCBF6F29E020EFC
:101EC000756ED60E746E7F9C7F9E7F807350CBBFE5
:101ED000F28ECC6F736BC8C672F6CAC671F6CCC6EA
:101EE00070F6F2CFC7F6F29E020E756EEF0E746EAC
:101EF0007F9C7F9E7F807350C7BFF28E756F04D02A
:101F000073697269716970690001BCEF5BF0060169
:101F1000CB6BCA6BCA51040833E3036ACA51940FEE
:101F2000E96E060E0320EA6EEF50CB27F00ECA25AD
:101F3000CC6F030ECD6FD8B0CD2B036ACA51940F6E
:101F4000E96E060E0320EA6EEFCFCEF6F250006E79
:101F5000F29ECDC675FFCCC674FFCEC673FF7F9CC4
:101F60007F9E7F840F01550E7E6EAA0E7E6E7F824D
:101F70007FB2FED77F940050F2120601CA2BCAD757
:101F8000CB1F010ECB27F250006EF29E030E756E32
:101F9000F50E746ECBC673FF7F9C7F9E7F840F010E
:101FA000550E7E6EAA0E7E6E7F827FB2FED77F9424
:101FB0000050F212000112000601C66BC56BC5513C
:101FC00004081EE3036AC551940FE96E060E032050
:101FD000EA6EF00EC525C96F030ECA6FD8B0CA2BC2
:101FE000F2CFCBF6F29ECAC675FFC9C674FF7F9CBE
:101FF0007F9E7F807350CBBFF28EEF6EC52BDFD7F5
:10200000C56BC55104080BE3036AC551940FE96E13
:10201000060E0320EA6EEF50C627C52BF2D7C61F67
:10202000010EC627F2CFC7F6F29E030E756EF50EAF
:10203000746E7F9C7F9E7F807350C7BFF28EC65D9B
:1020400011E0C56BC55104080AE3036AC551940F3A
:10205000E96E060E0320EA6EEF6AC52BF3D7000186
:1020600056DF0601199E0001BEEF5BF046C74DF733
:1020700007014A514D1B4DAF05D0D894D89046BFAB
:10208000D8802FD046C74DF749C74EF745514E5F10
:1020900006E04DAF26D0D850010AD86E22D04AC7EC
:1020A0004EF746514E5F06E04DAF1BD0D850010AA7
:1020B000D86E17D04BC74EF747514E5F06E04DAF75
:1020C00010D0D850010AD86E0CD04CC74EF74851EA
:1020D0004E5F06E04DAF05D0D850010AD86E01D052
:1020E000D89000011200800ED8A202D007015C1B1C
:1020F0000701616B626B58C760F75C51601B5751F9
:10210000D8B4DFD05F6F006E5B51D8B4E3D05F5FAF
:10211000D8B483D03EE35CC765F7658F5DC764F7CD
:102120005EC763F7626BD8906533643363336233A1
:102130005F2FF8D760AF03D06181E0D061915F91EC
:102140006189070EEA6E5A0EE96EEBD0619960BFA5
:102150000AD05FA113D06533643363336233002A3E
:10216000D8B4C7D00BD065BF0CD0D89062376337D6
:10217000643765370006D8B4BCD0F5D7618D6DD013
:10218000619D58C760F758AF02D0658FABD0659F8F
:10219000A9D05BC75FF75BC700F057515F5F58C7B7
:1021A00065F7658F59C764F75AC763F7626BD890B4
:1021B00065336433633362335F2FF8D760AF03D086
:1021C00061839CD061935F91618B070EEA6E5E0E16
:1021D000E96EA7D0619B60BF0AD05FA113D06533C1
:1021E000643363336233002AD8B483D00BD065BF25
:1021F0000CD0D89062376337643765370006D8B49F
:1022000078D0F5D7618F29D0619F5CC760F75CAF4C
:1022100002D0658F67D0659F65D05CC765F7658F15
:102220005DC764F75EC763F760AF04D0659F6185E3
:1022300065D06195626B5F91070EEA6E5A0EE96E8A
:1022400070D060BF1CD058C760F75FA106D065335F
:10225000643363336233002A4CE062AF0BD0632BEC
:1022600009E1642B07E1652B05E1653364336333D2
:10227000002A3FE061BD84D761BFC6D71CD0800E65
:10228000651B65AF04D03AD05CC760F70AD058C769
:1022900060F7655306E1645304E1635302E1006AA9
:1022A00021D065BF08D0D89062376337643765376F
:1022B000002EF7D71ED060AF02D0658F13D0659F78
:1022C00011D05BC700F05CC765F75DC764F75EC7F8
:1022D00063F708D057C700F058C765F759C764F7C8
:1022E0005AC763F765C701F064C702F063C703F01C
:1022F00034D0006A016A026A036A2FD0626B631FDE
:10230000641F651F621F622B05E1632B03E1642BD1
:1023100001E1652B61B112D761B354D761B589D79B
:10232000B3D7EF50632705E3642B03E1652BD8B4E3
:102330005F81ED52EF50642703E3652BD8B45F81D2
:10234000ED52EF50EFBE01D0800A6527D8B05F8113
:1023500061B9FCD661BB3ED774D7000112000701FA
:102360005351D8B471D0006E5751D8B46DD00026F7
:1023700004E3810E002668E204D07F0E005E64E371
:1023800063E054C75BF758515B1B548F588F56510D
:102390005A03F4CF5DF755515903F4CF03F0F3CF4F
:1023A0005CF75A03F3505D27F4505C23000E0322C0
:1023B00056515903F3505D27F4505C23000E026A16
:1023C0000322022254515A03F3505C27F450032293
:1023D000000E022254515903F3500326F4500222F6
:1023E000000E016A012256515803F3505C27F45045
:1023F0000322000E0222012255515803F3500326F6
:10240000F4500222000E012254515803F3500226C8
:10241000F4500122002A01BE05D05C370336023693
:1024200001360006000E5CAF0AD0032A0222012208
:10243000015005E1025003E1035001E1002A5BBFB6
:10244000018E5BAF019E04D0006A016A026A036AD2
:10245000000112008E0E006E0601EE51005EEFC606
:1024600002F0F0C601F0028E005209E0D89002524C
:1024700002E1015204E002320132002EF7D7EFAF41
:1024800005D0011E021E012AD8B4022A0001120042
:10249000036A0601CD51DE0FE96E020E0320EA6EDB
:1024A000EF3C37D0D16BD1511E081DE3CD513E0D0D
:1024B000F3500701146B136FD8900601D135036AEE
:1024C00007011325016E145103220150E60FE96E36
:1024D000010E0320EA6ECFC6ECFFED52CEC6EFFF31
:1024E0000601D12BE0D7036ACD51DE0FE96E020E53
:1024F0000320EA6EEF6AD890CD35036AE20FE96EE9
:10250000020E0320EA6ECFC6ECFFED52CEC6EFFFFF
:1025100017D1D05303E1010ED06F05D0D0511F0861
:1025200002E21F0ED06FCD513E0DF3500701146B28
:10253000136F036A0601CD51DE0FE96E020E032010
:10254000EA6ED890EF34036A07011325016E145127
:1025500003220150E60FE96E010E0320EA6ECFC69A
:10256000ECFFED52CEC6EFFF036A0601CD51DE0F40
:10257000E96E020E0320EA6EEF2AD051EF5C08E309
:10258000036ACD51DE0FE96E020E0320EA6EEF6A98
:10259000D16BD051D15D34E2D890D135036AD50FDB
:1025A000016E060E032201C013F703C014F70601E3
:1025B000CD513E0DF3500701166B156FD8900601F3
:1025C000D135036A07011525016E1651032201500A
:1025D000E60FE96E010E0320EA6EECCF03F0ED5238
:1025E000EFCF15F703C016F714C7EAFF13C7E9FFCB
:1025F00003C0ECFFED5215C7EFFF0601D12BC9D781
:10260000D291D16B010ED05DD15D01E070E2D89026
:10261000D135036AD50FE96E060E0320EA6EECCFC2
:1026200014F7ED52EFCF13F7010ED125006ED890BD
:1026300000360050036AD50FE96E060E0320EA6EDD
:10264000ECCF03F0ED52EFCF01F003500701145D22
:102650004BE303E11351015C47E2D8900601D13509
:10266000036AD50FE96E060E0320EA6EECCFD4F6AE
:10267000ED52EFCFD3F6D890D135036AD50F016E66
:10268000060E032203C014F7010E0601D125006EC9
:10269000D89000360050036AD50FE96E060E03206D
:1026A000EA6EECCF03F0ED52EFCF15F7070114C738
:1026B000EAFF01C0E9FF03C0ECFFED5215C7EFFFD1
:1026C000010E0601D125006ED89000360050036A35
:1026D000D50FE96E060E0320EA6ED4C6ECFFED526C
:1026E000D3C6EFFFD28107010601D12B8BD7D2B120
:1026F00087D7D890CD35036AE20F016E020E032210
:10270000070103C014F7D8900601D031006ED890AD
:1027100000360050036AD50FE96E060E0320EA6EFC
:10272000ECCF03F0ED52EFCF15F7070114C7EAFF26
:1027300001C0E9FF03C0ECFFED5215C7EFFF060132
:10274000000112000601F351070B006EF331016E18
:10275000013201321F0E01160150F425E96E000E00
:10276000F521EA6EEFCF01F0002A01D00132002EF0
:10277000FDD7010E0116000112000601FE51070BE4
:10278000006EFE31016E013201321F0E0116015042
:1027900007010025E96E000E0121EA6E016A012A97
:1027A000002A01D00136002EFDD70601FF5303E0B9
:1027B0000150EF1203D0011E0150EF16000112006C
:1027C00007015351D8B4A5D05F6F5751D8B4A1D0E9
:1027D0005F5F05E37F0E5F27D8B09BD006D0810EE8
:1027E0005F5FD8A096D0D8B494D05FC700F0016ADC
:1027F000026A036A5E6B54C75DF75D8F55C75CF76D
:1028000056C75BF7190E5F6F5A515B5F0DE2010E01
:102810005C5F0AE25D5F08E25E5F06E25E2B5D2BB5
:102820005C2B5A515B2728D059515C5F12E2010E94
:102830005D5F0FE25E5F0DE25E2B5D2B59515C2701
:102840005A515B2719E35C2B17E15D2B15E15E2BD9
:1028500013D0585180095D5F0EE2010E5E5F0BE2FE
:102860005E2B585180095D2759515C27E9E35D2BA8
:10287000E7E15E2BE5D703805F2F01D00BD0D89026
:102880005B375C375D375E37D890033602360136EA
:102890006037BAD760A106D0D89001320232033235
:1028A000603302D0000635E060BF1ED0D8905B37A1
:1028B0005C375D375E375A515B5F07E2010E5C5F44
:1028C00004E25D5F02E25E5F1AE359515C5F05E27C
:1028D000010E5D5F02E25E5F12E3585180095D5FA9
:1028E00003E2010E5E5F0BE3032A09E1022A07E11E
:1028F000012A05E1002A0DE001320232033254C7F9
:102900005FF758515F1B5FAF02D0018E06D0019E6A
:1029100004D0006A016A026A036A00011200CDC68F
:10292000F3F6030E0601F56F020EF46F00010ADFE5
:102930000150010B31E10601CD51040DF350036A42
:10294000EA0FE96E020E0320EA6ECFC654F7CEC638
:1029500053F700011FEC0BF000C0EFFF01C0ECFFCC
:1029600002C0ECFF03C0ECFFD8900601CD35036A2E
:10297000FA0FE96E020E0320EA6EEC6AED52EF6A7E
:10298000CDC6FEF6010EFF6F030E0701016F020EAA
:10299000006F0001F2DEC2D0D8900601CD35036A87
:1029A000FA0FE96E020E0320EA6E010EEF24016EAB
:1029B000000EEC20ED5201C0EFFFEC6ECD51040D86
:1029C000F350036AEA0F016E020E032201C0D1F632
:1029D00003C0D2F603C0EAFF01C0E9FFEFCFD3F690
:1029E000ECCFD4F6ECCFD5F6ECCFD6F6CFC654F775
:1029F000CEC653F700011FEC0BF003C05AF702C01C
:102A000059F701C058F700C057F70601CD51040D22
:102A1000F350036AEA0FE96E020E0320EA6EEFCF6D
:102A20005BF7ECCF01F0ECCF02F0ECCF03F0EACF94
:102A3000DCF6E9CFDBF6D88203C05EF702C05DF7B3
:102A400001C05CF7000173EC10F0DCC6EAFFDBC6E6
:102A5000E9FF03C0DAF602C0D9F601C0D8F600C01B
:102A6000D7F6D8900601CD35036AFA0FE96E020E4B
:102A70000320EA6EECCFDEF6ED52EFCFDDF6DE534B
:102A800016E1D051DD5D13E2D890CD35036AFA0F1F
:102A9000E96E020E0320EA6EECCF03F0ED52EFCFA9
:102AA00053F703C054F700011FEC0BF007D00701E8
:102AB000546BD0C653F700011FEC0BF0DAC656F783
:102AC000D9C655F7D8C654F7D7C653F703C05AF737
:102AD00002C059F701C058F700C057F771DED8920D
:102AE000D6C65AF7D5C659F7D4C658F7D3C657F73E
:102AF00003C05EF702C05DF701C05CF700C05BF782
:102B000073EC10F0D2C6EAFFD1C6E9FF00C0EFFFB8
:102B100001C0ECFF02C0ECFF03C0ECFF1200070194
:102B20004A6B200E496F20502318231A2318206E59
:102B300021502218221A2218216E213620362132E5
:102B400000014AC703F0070149C7E9FF03C0EAFFD4
:102B5000EFCF00F0ECCF01F0ECCF02F0ECCF03F0C0
:102B600000011200030E07014325496F000E4421A6
:102B70004A6FF2CF4BF7F29E4AC775FF49C774FF01
:102B80007F9C7F9E7F8073504BBFF28E496F020EF9
:102B900043254C6F000E44214D6FF2CF4AF7F29E51
:102BA0004DC775FF4CC774FF7F9C7F9E7F8073501D
:102BB0004ABFF28E4C6F010E43254D6F000E44212B
:102BC0004E6FF2CF4FF7F29E4EC775FF4DC774FFA1
:102BD0007F9C7F9E7F8073504FBFF28E4D6FF2CFF0
:102BE0004EF7F29E44C775FF43C774FF7F9C7F9EDC
:102BF0007F8073504EBFF28E506F49C748F74CC765
:102C000047F74DC746F750C745F748C723F047C7B2
:102C100022F046C721F045C720F0000180DF1200F6
:102C20000701455308E1465306E1006A016A026A5A
:102C3000036A34D133D1D8904335026E4435036EE4
:102C40000250050FE96E030E0320EA6EECCF03F08D
:102C5000ED52EFCF53F703C054F700011FEC0BF018
:102C600003C04EF702C04DF701C04CF700C04BF750
:102C70004EC756F74DC755F74CC754F74BC753F7D8
:102C800007015A6B596B7A0E586F880E576F000107
:102C900097DD03C04EF702C04DF701C04CF700C0EE
:102CA0004BF746C754F745C753F71FEC0BF003C06B
:102CB00052F702C051F701C050F700C04FF752C79A
:102CC00056F751C755F750C754F74FC753F7070189
:102CD0005A6BF00E596F7F0E586F8A0E576F0001B6
:102CE0006FDD03C052F702C051F701C050F700C0BA
:102CF0004FF752C756F751C755F750C754F74FC74C
:102D000053F707015A6B596B200E586F810E576F9E
:102D10000001AFEC11F003C052F702C051F701C03F
:102D200050F700C04FF74EC756F74DC755F74CC781
:102D300054F74BC753F752C75AF751C759F750C703
:102D400058F74FC757F73CDD03C056F702C055F799
:102D500001C054F700C053F7D88203C05AF702C02D
:102D600059F701C058F700C057F707015E6B5D6B5C
:102D70005C6B7F0E5B6F000173EC10F003C04AF7D1
:102D800002C049F701C048F700C047F70701566B7A
:102D9000556B546B7F0E536F4AC75AF749C759F7A3
:102DA00048C758F747C757F700010ADD03C04AF77D
:102DB00002C049F701C048F700C047F74AC756F7B5
:102DC00049C755F748C754F747C753F707015A6B28
:102DD000596B7A0E586F880E576F0001AFEC11F0E7
:102DE00003C04AF702C049F701C048F700C047F7DF
:102DF0000701566B556B546B7F0E536F4AC75AF7DA
:102E000049C759F748C758F747C757F70001D8DCF3
:102E100003C04AF702C049F701C048F700C047F7AE
:102E2000D8824AC75AF749C759F748C758F747C71A
:102E300057F7A50E07015E6FDA0E5D6F7D0E5C6FB2
:102E40006E0E5B6F000173EC10F003C04AF702C016
:102E500049F701C048F700C047F70701566B556BAB
:102E6000546B7F0E536F4AC75AF749C759F748C783
:102E700058F747C757F70001A3DC03C04AF702C061
:102E800049F701C048F700C047F747C700F048C7F7
:102E900001F049C702F04AC703F007010001120020
:102EA00044C754F743C753F71FEC0BF003C048F770
:102EB00002C047F701C046F700C045F748C756F7BC
:102EC00047C755F746C754F745C753F707015A6B2D
:102ED000F00E596F7F0E586F8A0E576F000170DC2D
:102EE00003C048F702C047F701C046F700C045F7E6
:102EF00048C756F747C755F746C754F745C753F76E
:102F000007015A6B596B200E586F810E576F0001E5
:102F1000AFEC11F003C048F702C047F701C046F715
:102F200000C045F745C700F046C701F047C702F0AB
:102F300048C703F0120044C754F743C753F71FECC8
:102F40000BF003C048F702C047F701C046F700C0C6
:102F500045F748C756F747C755F746C754F745C71B
:102F600053F707015A6BF00E596F7F0E586F8A0E98
:102F7000576F000125DC03C048F702C047F701C0C6
:102F800046F700C045F748C756F747C755F746C745
:102F900054F745C753F707015A6B596B200E586F0A
:102FA000810E576F0001AFEC11F003C048F702C06B
:102FB00047F701C046F700C045F748C756F747C76F
:102FC00055F746C754F745C753F7CA0E07015A6F5E
:102FD000260E596F1B0E586F7C0E576F0001E0ECE8
:102FE00013F003C048F702C047F701C046F700C01E
:102FF00045F745C700F046C701F047C702F048C78C
:1030000003F0120044C754F743C753F71FEC0BF00B
:1030100003C048F702C047F701C046F700C045F7B4
:1030200048C756F747C755F746C754F745C753F73C
:1030300007015A6BF00E596F7F0E586F8A0E576F4B
:103040000001E0EC13F003C048F702C047F701C0ED
:1030500046F700C045F748C756F747C755F746C774
:1030600054F745C753F707015A6B596B200E586F39
:10307000810E576F0001AFEC11F003C048F702C09A
:1030800047F701C046F700C045F748C756F747C79E
:1030900055F746C754F745C753F707015A6B596BA5
:1030A000480E586F860E576F0001E0EC13F003C016
:1030B0004CF702C04BF701C04AF700C049F74CC7B4
:1030C00056F74BC755F74AC754F749C753F7070197
:1030D0005A6B596B7A0E586F880E576F0001AFEC20
:1030E00011F003C04CF702C04BF701C04AF700C013
:1030F00049F749C700F04AC701F04BC702F04CC777
:1031000003F01200CDC642F7CCC641F70701446B6D
:103110008F0E436F0001A9EC06F002C003F00150CE
:10312000500F0701416F000E0320426F830E4127AD
:10313000000E4223F2CF43F7F29E42C775FF41C70C
:1031400074FF7F9C7F9E7F80735043BFF28E060189
:10315000D06FCF6BD051CF5DD8B081D0CDC642F704
:10316000CCC641F70701446B8F0E436F0001A9ECF9
:1031700006F00150500F0701416F000E0220426F10
:10318000230E4127000E42230601CF51040DF350B8
:10319000070141253E6F000E42213F6F0601CF51CE
:1031A000040DF350036AD10F016E060E032201C015
:1031B00041F703C042F73FC744F73EC743F700015A
:1031C000D1DC42C7EAFF41C7E9FF00C0EFFF01C001
:1031D000ECFF02C0ECFF03C0ECFFCDC642F7CCC64B
:1031E00041F70701446B8F0E436F0001A9EC06F015
:1031F0000150500F0701416F000E0220426F530E25
:103200004127000E42230601CF51040DF350070160
:1032100041253E6F000E42213F6F0601CF51040D44
:10322000F350036A010F016E070E032201C041F73C
:1032300003C042F73FC744F73EC743F7000192DCA3
:1032400042C7EAFF41C7E9FF00C0EFFF01C0ECFF42
:1032500002C0ECFF03C0ECFF0601CF2B7BD7D4C626
:1032600048F7D3C647F7D2C646F7D1C645F7D8C602
:103270004CF7D7C64BF7D6C64AF7D5C649F7000173
:1032800036EC10F004E30701318103D0000107019F
:103290003191CDC642F7CCC641F7446B8F0E436FD8
:1032A0000001A9EC06F002C003F00150500F070125
:1032B000416F000E0320426F220E4127000E422371
:1032C000F2CF43F7F29E42C775FF41C774FF7F9C60
:1032D0007F9E7F80735043BFF28E406F010E0601C8
:1032E000CE5DFC0FD8B07DD0040F0001E5EF1DF0DE
:1032F000D8900601CC35026ECD35036E0250E20F38
:10330000E96E020E0320EA6EECCF46F7ED52EFCFE6
:1033100045F7CDC644F7CCC643F7000181DC03C0B6
:103320003DF702C03CF701C03BF700C03AF7060189
:1033300058D0D8900601CC35026ECD35036E0250C0
:10334000E20FE96E020E0320EA6EECCF44F7ED5275
:10335000EFCF43F70001A4DD03C03DF702C03CF707
:1033600001C03BF700C03AF706013BD0D8900601F8
:10337000CC35026ECD35036E0250E20FE96E020EBF
:103380000320EA6EECCF44F7ED52EFCF43F7000194
:10339000D2DD03C03DF702C03CF701C03BF700C0DF
:1033A0003AF706011ED0D8900601CC35026ECD3515
:1033B000036E0250E20FE96E020E0320EA6EECCFBC
:1033C00044F7ED52EFCF43F700011CDE03C03DF799
:1033D00002C03CF701C03BF700C03AF7060101D03C
:1033E0000601CE2D3CD00701486B400E476F1C0EE6
:1033F000466F8C0E456F3DC74CF73CC74BF73BC73C
:103400004AF73AC749F7000136EC10F0D8B002D0BD
:10341000060125D007014051030806E0405102088B
:10342000D8B402D006011BD00601CC35026ECD35D2
:10343000036E02360336FC0E021602500F0FE96EC1
:10344000030E0320EA6EEF6AEC6AEC6AEC6A1F0E68
:10345000CC25E96E030ECD21EA6E030EEF6ED890F7
:10346000CC35026ECD35036E0250E20FE96E020ECE
:103470000320EA6EECCF42F7ED52EFCF41F70701A0
:1034800042510E0828E2FF0A03E14151A00823E25D
:103490004051030803E0405102081DE10601CC350C
:1034A000026ECD35036E02360336FC0E0216025054
:1034B0000F0FE96E030E0320EA6EEF6AEC6AEC6A06
:1034C000EC6A1F0ECC25E96E030ECD21EA6E030EC9
:1034D000EF6E79D30701D8900601CC35026ECD3559
:1034E000036E0250E20FE96E020E0320EA6EECCF8B
:1034F00042F7ED52EFCF41F70701415324E1425328
:1035000022E14051030802E0402D1DD00601CC35D8
:10351000026ECD35036E02360336FC0E02160250E3
:103520000F0FE96E030E0320EA6EEF6AEC6AEC6A95
:10353000EC6A1F0ECC25E96E030ECD21EA6E040E57
:10354000EF6E41D307011F0E0601CC25E96E030E75
:10355000CD21EA6EEF68070131A198D1010E060175
:10356000D05D040DF350036AD10FE96E060E0320FF
:10357000EA6EEFCF45F7ECCF46F7ECCF47F7ECCF4D
:1035800048F73DC74CF73CC74BF73BC74AF73AC72C
:1035900049F7000136EC10F015E3010E0601D05D8D
:1035A000040DF350036AD10FE96E060E0320EA6E94
:1035B000EFCF3AF7ECCF3BF7ECCF3CF7ECCF3DF752
:1035C0001DD000013DC748F73CC747F73BC746F74A
:1035D0003AC745F7D4C64CF7D3C64BF7D2C64AF71D
:1035E000D1C649F736EC10F008E3D4C63DF7D3C690
:1035F0003CF7D2C63BF7D1C63AF70601CF6BD051A4
:10360000CF5DD8B041D1CF51040DF350036AD10F33
:10361000E96E060E0320EA6EEFCF49F7ECCF4AF7CA
:10362000ECCF4BF7ECCF4CF73DC748F73CC747F71B
:103630003BC746F73AC745F7000136EC10F002E207
:10364000D8A41FD10601CF51040DF350036AD10F46
:10365000E96E060E0320EA6EEFCF57F7ECCF58F76E
:10366000ECCF59F7ECCF5AF7010ECF5D040DF350B4
:10367000036AD10FE96E060E0320EA6EEFCF5BF707
:10368000ECCF01F0ECCF02F0ECCF03F0EACF46F73D
:10369000E9CF45F7D88203C05EF702C05DF701C0ED
:1036A0005CF7000173EC10F046C7EAFF45C7E9FF7D
:1036B00003C035F702C034F701C033F700C032F75A
:1036C0000601CF51040DF350036A010FE96E070E96
:1036D0000320EA6EEFCF57F7ECCF58F7ECCF59F74E
:1036E000ECCF5AF7010ECF5D040DF350036A010FC2
:1036F000E96E070E0320EA6EEFCF5BF7ECCF01F027
:10370000ECCF02F0ECCF03F0EACF46F7E9CF45F774
:10371000D88203C05EF702C05DF701C05CF700010C
:1037200073EC10F046C7EAFF45C7E9FF03C039F75D
:1037300002C038F701C037F700C036F735C756F773
:1037400034C755F733C754F732C753F739C75AF759
:1037500038C759F737C758F736C757F7E0EC13F0B3
:1037600003C035F702C034F701C033F700C032F7A9
:103770000601CF51040DF350036AD10FE96E060E16
:103780000320EA6EEFCF57F7ECCF58F7ECCF59F79D
:10379000ECCF5AF7EACF46F7E9CF45F7D8823DC7D5
:1037A0005EF73CC75DF73BC75CF73AC75BF70001C4
:1037B00073EC10F046C7EAFF45C7E9FF03C039F7CD
:1037C00002C038F701C037F700C036F739C756F7DF
:1037D00038C755F737C754F736C753F735C75AF7C1
:1037E00034C759F733C758F732C757F7E0EC13F02F
:1037F00003C039F702C038F701C037F700C036F709
:103800000601CC35026ECD35036E02360336FC0E52
:10381000021602500F0F016E030E032201C041F782
:1038200003C042F70601CF51040DF350036A010FA4
:10383000E96E070E0320EA6EEFCF57F7ECCF58F78B
:10384000ECCF59F7ECCF5AF7D88239C75EF738C7B3
:103850005DF737C75CF736C75BF7000173EC10F014
:1038600042C7EAFF41C7E9FF00C0EFFF01C0ECFF1C
:1038700002C0ECFF03C0ECFF010E0601D025CF6FA4
:1038800000010601CF2BBBD69ED10701D4C648F755
:10389000D3C647F7D2C646F7D1C645F73DC74CF762
:1038A0003CC74BF73BC74AF73AC749F7000136EC2C
:1038B00010F009E3D4C63DF7D3C63CF7D2C63BF7B8
:1038C000D1C63AF733D0010E0601D05D040DF35096
:1038D000036AD10FE96E060E0320EA6EEFCF49F7B7
:1038E000ECCF4AF7ECCF4BF7ECCF4CF73DC748F79E
:1038F0003CC747F73BC746F73AC745F7000136ECE8
:1039000010F014E3010E0601D05D040DF350036ABC
:10391000D10FE96E060E0320EA6EEFCF3AF7ECCF37
:103920003BF7ECCF3CF7ECCF3DF700010601CF6B46
:10393000D051CF5DD8B047D1CF51040DF350036AB9
:10394000D10FE96E060E0320EA6EEFCF45F7ECCFFC
:1039500046F7ECCF47F7ECCF48F73DC74CF73CC7ED
:103960004BF73BC74AF73AC749F7000136EC10F06E
:1039700002E2D8A425D1010E0601CF5D040DF3505B
:10398000036AD10FE96E060E0320EA6EEFCF57F7F8
:10399000ECCF58F7ECCF59F7ECCF5AF7CF51040DD5
:1039A000F350036AD10FE96E060E0320EA6EEFCFE3
:1039B0005BF7ECCF01F0ECCF02F0ECCF03F0EACFF5
:1039C00046F7E9CF45F7D88203C05EF702C05DF73E
:1039D00001C05CF7000173EC10F046C7EAFF45C771
:1039E000E9FF03C035F702C034F701C033F700C068
:1039F00032F70601CF51040DF350036A010FE96E4F
:103A0000070E0320EA6EEFCF57F7ECCF58F7ECCF55
:103A100059F7ECCF5AF7010ECF5D040DF350036A4E
:103A2000010FE96E070E0320EA6EEFCF5BF7ECCFD4
:103A300001F0ECCF02F0ECCF03F0EACF46F7E9CF8C
:103A400045F7D88203C05EF702C05DF701C05CF79E
:103A5000000173EC10F046C7EAFF45C7E9FF03C059
:103A600039F702C038F701C037F700C036F735C75D
:103A700056F734C755F733C754F732C753F739C72A
:103A80005AF738C759F737C758F736C757F7E0EC32
:103A900013F003C035F702C034F701C033F700C09C
:103AA00032F70601CF51040DF350036AD10FE96ECE
:103AB000060E0320EA6EEFCF5BF7ECCF01F0ECCF00
:103AC00002F0ECCF03F0EACF42F7E9CF41F7D8821A
:103AD0003DC75AF73CC759F73BC758F73AC757F79E
:103AE00003C05EF702C05DF701C05CF7000173EC34
:103AF00010F042C7EAFF41C7E9FF03C039F702C02F
:103B000038F701C037F700C036F739C756F738C75E
:103B100055F737C754F736C753F735C75AF734C781
:103B200059F733C758F732C757F7E0EC13F003C023
:103B300039F702C038F701C037F700C036F7060181
:103B4000CC35026ECD35036E02360336FC0E0216FE
:103B500002500F0F016E030E032201C041F703C094
:103B600042F70601CF51040DF350036A010FE96ECD
:103B7000070E0320EA6EEFCF57F7ECCF58F7ECCFE4
:103B800059F7ECCF5AF7D88239C75EF738C75DF7D7
:103B900037C75CF736C75BF7000173EC10F042C71C
:103BA000EAFF41C7E9FF00C0EFFF01C0ECFF02C020
:103BB000ECFF03C0ECFF010E0601D025CF6F000122
:103BC0000601CF2BB5D600011200E824F76AF736BC
:103BD000E50FF66E3B0EF7220A00F550FA6E08006C
:103BE000F550F96EF03232336C33A6331F0E0601F6
:103BF000CC25E96E030ECD21EA6EEF3CC7EF21F034
:103C0000CDC642F7CCC641F70701446B8F0E436F18
:103C10000001A9EC06F002C003F00150500F0601AC
:103C2000D56F000E0320D66F180ED527000ED623B1
:103C3000F2CFD7F6F29ED6C675FFD5C674FF7F9C2D
:103C40007F9E7F807350D7BFF28ECE6FCDC642F776
:103C5000CCC641F70701446B8F0E436F0001A9ECFE
:103C600006F002C003F00150500F0601D56F000EA0
:103C70000220D66F140ED527000ED623D6C644F7E1
:103C8000D5C643F70001B2EC15F003C0D2F602C06E
:103C9000D1F601C0D0F600C0CFF6CDC642F7CCC6F3
:103CA00041F70701446B8F0E436F0001A9EC06F04A
:103CB00002C003F00150500F0601D56F000E032023
:103CC000D66F1A0ED527000ED623F2CFD7F6F29E66
:103CD000D6C675FFD5C674FF7F9C7F9E7F807350CC
:103CE000D7BFF28ED36FCE51070BFB0F5EE2050FED
:103CF00000017FEF22F00601D49157D00601CC35A8
:103D0000026ECD35036E02360336FC0E02160250EB
:103D10000F0FE96E030E0320EA6EEFCF45F7ECCFED
:103D200046F7ECCF47F7ECCF48F7D2C64CF7D1C6F1
:103D30004BF7D0C64AF7CFC649F7000136EC10F072
:103D400001E204E10601D48103D000010601D4910F
:103D50002CD00601CC35026ECD35036E023603360B
:103D6000FC0E021602500F0FE96E030E0320EA6EDE
:103D7000EFCF49F7ECCF4AF7ECCF4BF7ECCF4CF74E
:103D8000D2C648F7D1C647F7D0C646F7CFC645F7E3
:103D9000000136EC10F001E204E10601D48103D009
:103DA00000010601D49101D00601D4A1A0D0CEA972
:103DB0007ED001016C5324E16D5322E10601CC3524
:103DC000D56FCD35D66FD537D637FC0ED517570EF4
:103DD000D525E96E060ED621EA6EECCFD8F6ED5267
:103DE000EFCFD7F6D7530AE1D85308E11F0ECC2501
:103DF000E96E030ECD21EA6ED3C6EFFF57D0010165
:103E00000601CC35D56FCD35D66FD537D637FC0EFC
:103E1000D517570ED525E96E060ED621EA6ECDC60A
:103E200042F7CCC641F70701446B8F0E436F000188
:103E3000A9EC06F002C003F00150500F0601D96F43
:103E4000000E0320DA6F190ED927000EDA23F2CF05
:103E5000DBF6F29EDAC675FFD9C674FF7F9C7F9EA3
:103E60007F807350DBBFF28EEC6AED52EF6ECC3583
:103E7000D56FCD35D66FD537D637FC0ED517570E43
:103E8000D525E96E060ED621EA6EECCF42F7ED524B
:103E9000EFCF41F70701446B630E436F0001A9ECBC
:103EA00006F001C0EFFF02C0ECFF06011FD0CC35C9
:103EB000D56FCD35D66FD537D637FC0ED517570E03
:103EC000D525E96E060ED621EA6EECCFD8F6ED5276
:103ED000EFCFD7F6D7530AE1D85308E11F0ECC2510
:103EE000E96E030ECD21EA6ED3C6EFFF55D0CC3577
:103EF000D56FCD35D66FD537D637FC0ED517570EC3
:103F0000D525E96E060ED621EA6ECDC642F7CCC69F
:103F100041F70701446B8F0E436F0001A9EC06F0D7
:103F200002C003F00150500F0601D96F000E0320AC
:103F3000DA6F190ED927000EDA23F2CFDBF6F29EE4
:103F4000DAC675FFD9C674FF7F9C7F9E7F80735051
:103F5000DBBFF28EEC6AED52EF6ECC35D56FCD350E
:103F6000D66FD537D637FC0ED517570ED525E96E47
:103F7000060ED621EA6EECCF42F7ED52EFCF41F7B5
:103F80000701446B630E436F0001A9EC06F001C00A
:103F9000EFFF02C0ECFF0601CDC642F7CCC641F7E9
:103FA0000701446B8F0E436F0001A9EC06F002C0BD
:103FB00003F00150500F0601D56F000E0320D66F9D
:103FC0001F0ED527000ED623F2CFD7F6F29ED6C607
:103FD00075FFD5C674FF7F9C7F9E7F807350D7BFCF
:103FE000F28ECE6FCDC642F7CCC641F70701446BC7
:103FF0008F0E436F0001A9EC06F002C003F00150E0
:10400000500F0601D56F000E0220D66F1B0ED5276C
:10401000000ED623D6C644F7D5C643F70001B2EC4E
:1040200015F003C0D2F602C0D1F601C0D0F600C030
:10403000CFF6CDC642F7CCC641F70701446B8F0ED1
:10404000436F0001A9EC06F002C003F00150500FCD
:104050000601D56F000E0320D66F210ED527000E66
:10406000D623F2CFD7F6F29ED6C675FFD5C674FF1B
:104070007F9C7F9E7F807350D7BFF28ED36F1F0EC1
:10408000CC25E96E030ECD21EA6EEF50D35DD8B09A
:104090007DD1CE51070BFB0F5EE2050F000191EFC2
:1040A00022F00601D49157D00601CC35026ECD35F1
:1040B000036E02360336FC0E021602500F0FE96E35
:1040C000030E0320EA6EEFCF45F7ECCF46F7ECCFB7
:1040D00047F7ECCF48F7D2C64CF7D1C64BF7D0C65E
:1040E0004AF7CFC649F7000136EC10F001E204E1CF
:1040F0000601D48103D000010601D4912CD0060121
:10410000CC35026ECD35036E02360336FC0E021638
:1041100002500F0FE96E030E0320EA6EEFCF49F74E
:10412000ECCF4AF7ECCF4BF7ECCF4CF7D2C648F7C1
:10413000D1C647F7D0C646F7CFC645F7000136ECE3
:1041400010F001E204E10601D48103D00001060170
:10415000D49101D00601D4A1B8D0CEA990D001014C
:104160006C532AE16D5328E10601CC35D56FCD356E
:10417000D66FD537D637FC0ED517020ED525016E72
:10418000000ED621036E0150570FE96E060E032074
:10419000EA6EECCFD6F6ED52EFCFD5F6D5530AE165
:1041A000D65308E11F0ECC25E96E030ECD21EA6E31
:1041B000D3C6EFFF63D001010601CC35D56FCD35F5
:1041C000D66FD537D637FC0ED517020ED525016E22
:1041D000000ED621036E0150570FE96E060E032024
:1041E000EA6ECDC642F7CCC641F70701446B8F0E8D
:1041F000436F0001A9EC06F002C003F00150500F1C
:104200000601D76F000E0320D86F200ED727000EAF
:10421000D823F2CFD9F6F29ED8C675FFD7C674FF61
:104220007F9C7F9E7F807350D9BFF28EEC6AED52E7
:10423000EF6ECC35D56FCD35D66FD537D637FC0E72
:10424000D517020ED525016E000ED621036E015042
:10425000570FE96E060E0320EA6EECCF42F7ED52DF
:10426000EFCF41F70701446B630E436F0001A9ECE8
:1042700006F001C0EFFF02C0ECFF060125D0CC35EF
:10428000D56FCD35D66FD537D637FC0ED517020E84
:10429000D525016E000ED621036E0150570FE96E31
:1042A000060E0320EA6EECCFD6F6ED52EFCFD5F630
:1042B000D5530AE1D65308E11F0ECC25E96E030E53
:1042C000CD21EA6ED3C6EFFF61D0CC35D56FCD35A9
:1042D000D66FD537D637FC0ED517020ED525016E11
:1042E000000ED621036E0150570FE96E060E032013
:1042F000EA6ECDC642F7CCC641F70701446B8F0E7C
:10430000436F0001A9EC06F002C003F00150500F0A
:104310000601D76F000E0320D86F200ED727000E9E
:10432000D823F2CFD9F6F29ED8C675FFD7C674FF50
:104330007F9C7F9E7F807350D9BFF28EEC6AED52D6
:10434000EF6ECC35D56FCD35D66FD537D637FC0E61
:10435000D517020ED525016E000ED621036E015031
:10436000570FE96E060E0320EA6EECCF42F7ED52CE
:10437000EFCF41F70701446B630E436F0001A9ECD7
:1043800006F001C0EFFF02C0ECFF0601B6D0CC354D
:10439000D56FCD35D66FD537D637FC0ED517570E1E
:1043A000D525E96E060ED621EA6ECDC642F7CCC6FB
:1043B00041F70701446B8F0E436F0001A9EC06F033
:1043C00002C003F00150500F0601D96F000E032008
:1043D000DA6F190ED927000EDA23F2CFDBF6F29E40
:1043E000DAC675FFD9C674FF7F9C7F9E7F807350AD
:1043F000DBBFF28EEC6AED52EF6ECC35D56FCD356A
:10440000D66FD537D637FC0ED517570ED525E96EA2
:10441000060ED621EA6EECCF42F7ED52EFCF41F710
:104420000701446B630E436F0001A9EC06F001C065
:10443000EFFF02C0ECFF0601CC35D56FCD35D66F4E
:10444000D537D637FC0ED517020ED525016E000ED6
:10445000D621036E0150570FE96E060E0320EA6E57
:10446000CDC642F7CCC641F70701446B8F0E436FB0
:104470000001A9EC06F002C003F00150500F060144
:10448000D76F000E0320D86F200ED727000ED82339
:10449000F2CFD9F6F29ED8C675FFD7C674FF7F9CBF
:1044A0007F9E7F807350D9BFF28EEC6AED52EF6E23
:1044B000CC35D56FCD35D66FD537D637FC0ED51761
:1044C000020ED525016E000ED621036E0150570F46
:1044D000E96E060E0320EA6EECCF42F7ED52EFCF05
:1044E00041F70701446B630E436F0001A9EC06F02E
:1044F00001C0EFFF02C0ECFF060100011200E8243A
:10450000F76AF736190FF66E450EF7220A00F550D6
:10451000FA6E0800F550F96EF63CFC3CFC3C523D4E
:10452000523DE824F76AF7363D0FF66E450EF72246
:104530000A00F550FA6E0800F550F96EA240A84046
:10454000A840FE40FE400601CD91D890CC35036ACC
:10455000DE0FE96E010E0320EA6EECCFCFF6ED52CE
:10456000EFCFCEF6CF510C0816E2FF0A03E1CE5191
:104570003F0811E2010ECC25CE6FCF6F020ED06F37
:104580000001AEEC09F0640E03010D6F960E0E6F84
:104590000601CD810FD003010D530DE1010E06017F
:1045A000CC25CE6FCF6F040ED06F0001AEEC09F0BA
:1045B0000601CD910301000E0601CDB1010E016E81
:1045C000000140EF28F0CDC642F7CCC641F7070105
:1045D000446B8F0E436F0001A9EC06F002C003F09C
:1045E0000150500F0601D76F000E0220D86F530EF6
:1045F000D727000ED823040ED727000ED823D8C6FD
:1046000044F7D7C643F70001B2EC15F003C0D2F669
:1046100002C0D1F601C0D0F600C0CFF6CDC642F739
:10462000CCC641F70701446B8F0E436F0001A9EC24
:1046300006F002C003F00150500F0601D76F000EC4
:104640000220D86F530ED727000ED823D8C644F7C0
:10465000D7C643F70001B2EC15F003C0D6F602C08E
:10466000D5F601C0D4F600C0D3F6050E0601CE5D26
:10467000FC0FD8B0B3EF27F0040F0001B5EF27F01F
:104680000601CC35026ECD35036E02360336FC0EC4
:10469000021602500F0FE96E030E0320EA6EEFCFF1
:1046A00045F7ECCF46F7ECCF47F7ECCF48F7D6C647
:1046B0004CF7D5C64BF7D4C64AF7D3C649F7000125
:1046C00036EC10F04DE1D8900601CC35026ECD35B8
:1046D000036E0250E20FE96E020E0320EA6EECCF89
:1046E000D8F6ED52EFCFD7F6F2CFD9F6F29E756A33
:1046F0000C0E746E7F9C7F9E7F807350D9BFF28EAC
:10470000DA6FF2CFDBF6F29E756A0B0E746E7F9C49
:104710007F9E7F807350DBBFF28EDC6FDAC603F0C2
:10472000DC51016ED851035C1AE303E1D751015CFF
:1047300016E3CC35026ECD35036E02360336FC0E21
:10474000021602500F0FE96E030E0320EA6ECFC669
:10475000EFFFD0C6ECFFD1C6ECFFD2C6ECFFABD06A
:104760000601CC35026ECD35036E02360336FC0EE3
:10477000021602500F0FE96E030E0320EA6EEFCF10
:1047800045F7ECCF46F7ECCF47F7ECCF48F7D2C66A
:104790004CF7D1C64BF7D0C64AF7CFC649F7000150
:1047A00036EC10F071E1D8900601CC35026ECD35B3
:1047B000036E0250E20FE96E020E0320EA6EECCFA8
:1047C000D8F6ED52EFCFD7F6F2CFD9F6F29E756A52
:1047D0000C0E746E7F9C7F9E7F807350D9BFF28ECB
:1047E000DA6FF2CFDBF6F29E756A0B0E746E7F9C69
:1047F0007F9E7F807350DBBFF28EDC6FDAC6DEF601
:10480000DCC6DDF6F2CFDFF6F29E756A100E746E2E
:104810007F9C7F9E7F807350DFBFF28EE06FF2CF70
:10482000E1F6F29E756A0F0E746E7F9C7F9E7F800C
:104830007350E1BFF28EE26FE0C603F0E251DD2576
:10484000016EDE5103220150016E0350D85D1AE360
:1048500003E10150D75D16E3CC35026ECD35036E12
:1048600002360336FC0E021602500F0FE96E030EDD
:104870000320EA6ED3C6EFFFD4C6ECFFD5C6ECFF2B
:10488000D6C6ECFF18D000010601CC35026ECD353E
:10489000036E02360336FC0E021602500F0FE96E4D
:1048A000030E0320EA6ED3C6EFFFD4C6ECFFD5C6D5
:1048B000ECFFD6C6ECFF57D30601CC35026ECD35E2
:1048C000036E02360336FC0E021602500F0FE96E1D
:1048D000030E0320EA6EEFCF45F7ECCF46F7ECCF9F
:1048E00047F7ECCF48F7D6C64CF7D5C64BF7D4C63A
:1048F0004AF7D3C649F7000136EC10F070E1D890C2
:104900000601CC35026ECD35036E0250E20FE96E22
:10491000020E0320EA6EECCFD8F6ED52EFCFD7F6B9
:10492000F2CFD9F6F29E756A0C0E746E7F9C7F9E54
:104930007F807350D9BFF28EDA6FF2CFDBF6F29E32
:10494000756A0B0E746E7F9C7F9E7F807350DBBFF9
:10495000F28EDC6FDAC6DEF6DCC6DDF6F2CFDFF60D
:10496000F29E756A100E746E7F9C7F9E7F807350DE
:10497000DFBFF28EE06FF2CFE1F6F29E756A0F0EA6
:10498000746E7F9C7F9E7F807350E1BFF28EE26FDA
:10499000E0C603F0E251DD25016EDE510322015035
:1049A000016E0350D85D1AE303E10150D75D16E3B1
:1049B000CC35026ECD35036E02360336FC0E021680
:1049C00002500F0FE96E030E0320EA6ECFC6EFFF11
:1049D000D0C6ECFFD1C6ECFFD2C6ECFF88D00601F2
:1049E000CC35026ECD35036E02360336FC0E021650
:1049F00002500F0FE96E030E0320EA6EEFCF45F76A
:104A0000ECCF46F7ECCF47F7ECCF48F7D2C64CF7E0
:104A1000D1C64BF7D0C64AF7CFC649F7000136ECEE
:104A200010F04EE1D8900601CC35026ECD35036E04
:104A30000250E20FE96E020E0320EA6EECCFD8F6C8
:104A4000ED52EFCFD7F6F2CFD9F6F29E756A0C0E83
:104A5000746E7F9C7F9E7F807350D9BFF28EDA6F19
:104A6000F2CFDBF6F29E756A0B0E746E7F9C7F9E12
:104A70007F807350DBBFF28EDC6FDAC603F0DC514F
:104A8000016ED851035C1AE303E1D751015C16E3D0
:104A9000CC35026ECD35036E02360336FC0E02169F
:104AA00002500F0FE96E030E0320EA6ED3C6EFFF2C
:104AB000D4C6ECFFD5C6ECFFD6C6ECFF18D000017B
:104AC0000601CC35026ECD35036E02360336FC0E80
:104AD000021602500F0FE96E030E0320EA6ED3C6D2
:104AE000EFFFD4C6ECFFD5C6ECFFD6C6ECFF3BD239
:104AF0000601CC35026ECD35036E02360336FC0E50
:104B0000021602500F0FE96E030E0320EA6EEFCF7C
:104B100045F7ECCF46F7ECCF47F7ECCF48F7D6C6D2
:104B20004CF7D5C64BF7D4C64AF7D3C649F70001B0
:104B300036EC10F04DE1D8900601CC35026ECD3543
:104B4000036E0250E20FE96E020E0320EA6EECCF14
:104B5000D8F6ED52EFCFD7F6F2CFD9F6F29E756ABE
:104B60000E0E746E7F9C7F9E7F807350D9BFF28E35
:104B7000DA6FF2CFDBF6F29E756A0D0E746E7F9CD3
:104B80007F9E7F807350DBBFF28EDC6FDAC603F04E
:104B9000DC51016E0350D85D1AE303E10150D75D8B
:104BA00016E3CC35026ECD35036E02360336FC0EAD
:104BB000021602500F0FE96E030E0320EA6ECFC6F5
:104BC000EFFFD0C6ECFFD1C6ECFFD2C6ECFFACD0F5
:104BD0000601CC35026ECD35036E02360336FC0E6F
:104BE000021602500F0FE96E030E0320EA6EEFCF9C
:104BF00045F7ECCF46F7ECCF47F7ECCF48F7D2C6F6
:104C00004CF7D1C64BF7D0C64AF7CFC649F70001DB
:104C100036EC10F072E1D8900601CC35026ECD353D
:104C2000036E0250E20FE96E020E0320EA6EECCF33
:104C3000D8F6ED52EFCFD7F6F2CFD9F6F29E756ADD
:104C40000E0E746E7F9C7F9E7F807350D9BFF28E54
:104C5000DA6FF2CFDBF6F29E756A0D0E746E7F9CF2
:104C60007F9E7F807350DBBFF28EDC6FDAC6DEF68C
:104C7000DCC6DDF6F2CFDFF6F29E756A100E746EBA
:104C80007F9C7F9E7F807350DFBFF28EE06FF2CFFC
:104C9000E1F6F29E756A0F0E746E7F9C7F9E7F8098
:104CA0007350E1BFF28EE26FE0C603F0E251DD5DCA
:104CB000006E0350DE59036E0050016ED851035C44
:104CC0001AE303E1D751015C16E3CC35026ECD3512
:104CD000036E02360336FC0E021602500F0FE96E09
:104CE000030E0320EA6ED3C6EFFFD4C6ECFFD5C691
:104CF000ECFFD6C6ECFF18D000010601CC35026EE1
:104D0000CD35036E02360336FC0E021602500F0F2D
:104D1000E96E030E0320EA6ED3C6EFFFD4C6ECFFA4
:104D2000D5C6ECFFD6C6ECFF1ED10601CC35026E0F
:104D3000CD35036E02360336FC0E021602500F0FFD
:104D4000E96E030E0320EA6EEFCF45F7ECCF46F78E
:104D5000ECCF47F7ECCF48F7D6C64CF7D5C64BF7A4
:104D6000D4C64AF7D3C649F7000136EC10F071E11A
:104D7000D8900601CC35026ECD35036E0250E20F9D
:104D8000E96E020E0320EA6EECCFD8F6ED52EFCFBB
:104D9000D7F6F2CFD9F6F29E756A0E0E746E7F9C2E
:104DA0007F9E7F807350D9BFF28EDA6FF2CFDBF631
:104DB000F29E756A0D0E746E7F9C7F9E7F8073508D
:104DC000DBBFF28EDC6FDAC6DEF6DCC6DDF6F2CFD4
:104DD000DFF6F29E756A100E746E7F9C7F9E7F8058
:104DE0007350DFBFF28EE06FF2CFE1F6F29E756A8C
:104DF0000F0E746E7F9C7F9E7F807350E1BFF28E9A
:104E0000E26FE0C603F0E251DD5D006E0350DE5953
:104E1000036E0050016ED851035C1AE303E1D751D1
:104E2000015C16E3CC35026ECD35036E02360336D7
:104E3000FC0E021602500F0FE96E030E0320EA6EFD
:104E4000CFC6EFFFD0C6ECFFD1C6ECFFD2C6ECFF59
:104E500088D00601CC35026ECD35036E023603369E
:104E6000FC0E021602500F0FE96E030E0320EA6ECD
:104E7000EFCF45F7ECCF46F7ECCF47F7ECCF48F74D
:104E8000D2C64CF7D1C64BF7D0C64AF7CFC649F7C2
:104E9000000136EC10F04EE1D8900601CC35026EE0
:104EA000CD35036E0250E20FE96E020E0320EA6E6A
:104EB000ECCFD8F6ED52EFCFD7F6F2CFD9F6F29E7F
:104EC000756A0E0E746E7F9C7F9E7F807350D9BF73
:104ED000F28EDA6FF2CFDBF6F29E756A0D0E746E0B
:104EE0007F9C7F9E7F807350DBBFF28EDC6FDAC6C3
:104EF00003F0DC51016E0350D85D1AE303E1015069
:104F0000D75D16E3CC35026ECD35036E023603361F
:104F1000FC0E021602500F0FE96E030E0320EA6E1C
:104F2000D3C6EFFFD4C6ECFFD5C6ECFFD6C6ECFF68
:104F300018D000010601CC35026ECD35036E023665
:104F40000336FC0E021602500F0FE96E030E03200B
:104F5000EA6ED3C6EFFFD4C6ECFFD5C6ECFFD6C6CB
:104F6000ECFF01D0060100011200E824F76AF736D1
:104F7000850FF66E4F0EF7220A00F550FA6E080004
:104F8000F550F96E8046B848F04A2A4DCAC642F735
:104F9000C9C641F70701446B8F0E436F0001A9ECAE
:104FA00006F002C003F00150500F0601CC6F000E56
:104FB0000320CD6FF2CFCEF6F29ECDC675FFCCC6E4
:104FC00074FF7F9C7F9E7F807350CEBFF28ECB6F2D
:104FD000CB51000A000115E0010A2EE0030A3CE073
:104FE000010A3AE0070A48E0010AD8B478D0030A77
:104FF000D8B490D0010AD8B4A8D00F0AD8B4C0D081
:10500000DBD00601C935026ECA35036E023603369F
:10501000FC0E021602500F0FE96E030E0320EA6E1B
:10502000EF6AEC6AEC6AEC6A1F0EC925E96E030EA2
:10503000CA21EA6EEF68DAD0CAC6CDF6C9C6CCF688
:10504000CBC6CEF682EC18F0CAC6CDF6C9C6CCF6F1
:10505000F6EC1DF00601CAD0CAC6CDF6C9C6CCF61C
:10506000CBC6CEF682EC18F0CAC6CDF6C9C6CCF6D1
:10507000F6EC1DF00601BAD0C9C6CCF6A3EF22F0BB
:10508000012C1DD00601C935026ECA35036E0236E9
:105090000336FC0E021602500F0FE96E030E0320BA
:1050A000EA6EEF6AEC6AEC6AEC6A1F0EC925E96EDB
:1050B000030ECA21EA6E030EEF6E10D00001CAC6BD
:1050C000CDF6C9C6CCF6CBC6CEF682EC18F0CAC671
:1050D000CDF6C9C6CCF6F6EC1DF0060187D0CAC6DF
:1050E000CDF6C9C6CCF6050E0601CE6F0001E3EC85
:1050F00022F01F0E0601C925E96E030ECA21EA6ED1
:10510000EF68CAC6CDF6C9C6CCF60001F6EC1DF0B4
:1051100006016CD0CAC6CDF6C9C6CCF6060E06018D
:10512000CE6F0001E3EC22F01F0E0601C925E96EE7
:10513000030ECA21EA6EEF68CAC6CDF6C9C6CCF620
:105140000001F6EC1DF0060151D0CAC6CDF6C9C665
:10515000CCF6070E0601CE6F0001E3EC22F01F0E25
:105160000601C925E96E030ECA21EA6EEF68CAC6B8
:10517000CDF6C9C6CCF60001F6EC1DF0060136D01E
:10518000CAC6CDF6C9C6CCF6080E0601CE6F000120
:10519000E3EC22F01F0E0601C925E96E030ECA21B9
:1051A000EA6EEF68CAC6CDF6C9C6CCF60001F6ECC9
:1051B0001DF006011BD000010601C935026ECA357B
:1051C000036E02360336FC0E021602500F0FE96E14
:1051D000030E0320EA6EEF6AEC6AEC6AEC6A1F0EBB
:1051E000C925E96E030ECA21EA6EEF6800011200BC
:1051F000036A0601CB51CF0FE96E010E0320EA6E60
:10520000EF3C33D0CE6BCE51080819E3CB51120DD1
:10521000F350E56BE46FD890CE35036AE425016E58
:10522000E55103220150750FE96E010E0320EA6E6D
:10523000CDC6ECFFED52CCC6EFFFCE2BE4D7036A10
:10524000CB51CF0FE96E010E0320EA6EEF6AD890C2
:10525000CB35036AD40FE96E010E0320EA6ECDC68A
:10526000ECFFED52CCC6EFFFE1D0CB51120DF35065
:10527000E56BE46F036ACB51CF0FE96E010E03209B
:10528000EA6ED890EF34036AE425016EE5510322FB
:105290000150750FE96E010E0320EA6ECDC6ECFFDA
:1052A000ED52CCC6EFFF036ACB51CF0FE96E010E72
:1052B0000320EA6EEF2AEF50080808E2036ACB5198
:1052C000CF0FE96E010E0320EA6EEF6ACE6BCE516E
:1052D00008082FE3D890CE35036AD20F016E060E70
:1052E000032201C0E4F603C0E5F6CB51120DF350E2
:1052F000E76BE66FD890CE35036AE625016EE7517D
:1053000003220150750FE96E010E0320EA6EECCF07
:1053100003F0ED52EFCFE6F603C0E7F6E5C6EAFF8D
:10532000E4C6E9FF03C0ECFFED52E6C6EFFFCE2B6B
:10533000CED7CF91CE6BCE51070869E3D890CE354A
:10534000036AD20FE96E060E0320EA6EECCFE5F693
:10535000ED52EFCFE4F6010ECE25006ED890003668
:105360000050036AD20FE96E060E0320EA6EECCFFE
:1053700003F0ED52EFCF01F00350E55D46E303E1AA
:10538000E451015C42E2D890CE35036AD20FE96E57
:10539000060E0320EA6EECCFD1F6ED52EFCFD0F639
:1053A000D890CE35036AD20F016E060E032203C0D9
:1053B000E5F6010ECE25006ED89000360050036A47
:1053C000D20FE96E060E0320EA6EECCF03F0ED5229
:1053D000EFCFE6F6E5C6EAFF01C0E9FF03C0ECFF48
:1053E000ED52E6C6EFFF010ECE25006ED8900036D6
:1053F0000050036AD20FE96E060E0320EA6ED1C692
:10540000ECFFED52D0C6EFFFCF81CE2B94D7CFB1BA
:1054100090D7D890CB35036AD40FE96E010E0320E4
:10542000EA6EDBC6ECFFED52DAC6EFFF00011200B8
:10543000CAC654F7C9C653F71FEC0BF003C0CEF62B
:1054400002C0CDF601C0CCF600C0CBF6CEC656F7F2
:10545000CDC655F7CCC654F7CBC653F707015A6BE8
:10546000F00E596F7F0E586F8A0E576F0001E0ECF7
:1054700013F003C0CEF602C0CDF601C0CCF600C0DA
:10548000CBF6CEC656F7CDC655F7CCC654F7CBC62D
:1054900053F707015A6B596B200E586F810E576FE7
:1054A0000001AFEC11F003C0CEF602C0CDF601C092
:1054B000CCF600C0CBF6CEC656F7CDC655F7CCC657
:1054C00054F7CBC653F7F10E07015A6F290E596FE7
:1054D000586B7C0E576F0001E0EC13F003C0CEF662
:1054E00002C0CDF601C0CCF600C0CBF6CEC656F752
:1054F000CDC655F7CCC654F7CBC653F707015A6B48
:10550000596B7A0E586F880E576F0001AFEC11F08F
:1055100003C0CEF602C0CDF601C0CCF600C0CBF67B
:10552000CEC6F1F6CDC6F0F6CCC6EFF6CBC6EEF69B
:105530002AEC12F00250FBEF2FF0CAC654F7C9C68E
:1055400053F71FEC0BF003C0CEF602C0CDF601C03E
:10555000CCF600C0CBF6CEC656F7CDC655F7CCC6B6
:1055600054F7CBC653F707015A6BF00E596F7F0EF5
:10557000586F8A0E576F0001E0EC13F003C0CEF6AF
:1055800002C0CDF601C0CCF600C0CBF6CEC656F7B1
:10559000CDC655F7CCC654F7CBC653F707015A6BA7
:1055A000596B200E586F810E576F0001AFEC11F050
:1055B00003C0CEF602C0CDF601C0CCF600C0CBF6DB
:1055C000CEC656F7CDC655F7CCC654F7CBC653F763
:1055D00007015A6B596B7A0E586F880E576F00018E
:1055E000AFEC11F003C0CEF602C0CDF601C0CCF690
:1055F00000C0CBF6CBC600F0CCC601F0CDC602F0A1
:10560000CEC603F01200C282C2B2FED7C4CF02F0EF
:10561000C3CF01F0C4CF54F7C3CF53F700011FEC41
:105620000BF003C0C8F602C0C7F601C0C6F600C042
:10563000C5F60701486B476B466B8E0E456FC8C6B3
:105640004CF7C7C64BF7C6C64AF7C5C649F70001AF
:1056500036EC10F006E30601C86BC76BC66BC56B72
:105660000001010174535FE00701546B74C153F7EB
:1056700000011FEC0BF003C048F702C047F701C060
:1056800046F700C045F7C8C64CF7C7C64BF7C6C6B5
:105690004AF7C5C649F736EC10F001E223E10701ED
:1056A000546B74C153F700011FEC0BF0D882C8C6CD
:1056B0005AF7C7C659F7C6C658F7C5C657F703C045
:1056C0005EF702C05DF701C05CF700C05BF773ECEA
:1056D00010F003C0C8F602C0C7F601C0C6F600C08D
:1056E000C5F606D00601C86BC76BC66BC56B00015B
:1056F000C8C656F7C7C655F7C6C654F7C5C653F74A
:1057000073C15AF772C159F771C158F770C157F791
:10571000AFEC11F003C0C8F602C0C7F601C0C6F670
:1057200000C0C5F601016F51F60FD8B0BBEF30F0E5
:105730000A0F00011BEF31F006019DB1E8D0C8C689
:10574000F1F6C7C6F0F6C6C6EFF6C5C6EEF600011E
:105750002AEC12F002C0DFF101C0DEF1F2CFC9F68F
:10576000F29E756A020E746E7F9C7F9E7F807350DE
:105770000601C9BFF28E030BFC0FD8B0C1D0040FD5
:105780000001D7EF30F0C8C6F1F6C7C6F0F6C6C6BE
:10579000EFF6C5C6EEF62AEC12F002C0E3F201C045
:1057A000E2F20601ADD0C8C6F1F6C7C6F0F6C6C62D
:1057B000EFF6C5C6EEF62AEC12F002C0CAF601C03A
:1057C000C9F6F2CFCBF6F29E756A030E746E7F9C1B
:1057D0007F9E7F8073500601CBBFF28ECC6FCD6B66
:1057E000CAC6CFF6C9C6CEF6CCC6D0F6000148EC84
:1057F00012F0060185D0C8C6F1F6C7C6F0F6C6C6D7
:10580000EFF6C5C6EEF62AEC12F002C0CAF601C0E9
:10581000C9F6F2CFCBF6F29E756A070E746E7F9CC6
:105820007F9E7F8073500601CBBFF28ECC6FCD6B15
:10583000CAC6CFF6C9C6CEF6CCC6D0F600018FECEC
:1058400014F0EDC2F1F6ECC2F0F6EBC2EFF6EAC2EC
:10585000EEF62AEC12F002C0E3F201C0E2F2060119
:105860004FD0C8C6F1F6C7C6F0F6C6C6EFF6C5C635
:10587000EEF62AEC12F002C0CAF601C0C9F6F2CF69
:10588000CBF6F29E756A030E746E7F9C7F9E7F80BE
:1058900073500601CBBFF28ECC6FCD6BCAC6CFF66C
:1058A000C9C6CEF6CCC6D0F6000148EC12F0F2CF55
:1058B000C9F6F29E756A070E746E7F9C7F9E7F808C
:1058C00073500601C9BFF28ECA6FCD6BE3C2CFF62B
:1058D000E2C2CEF6CAC6D0F600018FEC14F0EDC2DB
:1058E000F1F6ECC2F0F6EBC2EFF6EAC2EEF62AEC05
:1058F00012F002C0E3F201C0E2F2060101D006019B
:10590000CA6BC96B0001C6EC27F01BD00601C8C6E4
:10591000F1F6C7C6F0F6C6C6EFF6C5C6EEF600014C
:105920002AEC12F002C0CAF601C0C9F60601CD6B1E
:1059300002C0CFF601C0CEF6050ED06F000148ECD4
:1059400012F00101BBEF30F006019DB1F4D0C8C6E2
:10595000F1F6C7C6F0F6C6C6EFF6C5C6EEF600010C
:105960002AEC12F002C0E1F101C0E0F1F2CFC9F679
:10597000F29E756A020E746E7F9C7F9E7F807350CC
:105980000601C9BFF28EC00B006E003A0032003231
:10599000030E00160050FC0FD8B0C5D0040F000154
:1059A000E8EF30F0C8C6F1F6C7C6F0F6C6C6EFF6A7
:1059B000C5C6EEF62AEC12F002C0E9F201C0E8F228
:1059C0000601B1D0C8C6F1F6C7C6F0F6C6C6EFF6F6
:1059D000C5C6EEF62AEC12F002C0CAF601C0C9F63E
:1059E000F2CFCBF6F29E756A060E746E7F9C7F9E98
:1059F0007F8073500601CBBFF28ECC6F030ECD6F4C
:105A0000CAC6CFF6C9C6CEF6CCC6D0F6000148EC61
:105A100012F0060188D0C8C6F1F6C7C6F0F6C6C6B1
:105A2000EFF6C5C6EEF62AEC12F002C0CAF601C0C7
:105A3000C9F6F2CFCBF6F29E756A0A0E746E7F9CA1
:105A40007F9E7F8073500601CBBFF28ECC6F030E1A
:105A5000CD6FCAC6CFF6C9C6CEF6CCC6D0F6000109
:105A60008FEC14F0F9C2F1F6F8C2F0F6F7C2EFF6D7
:105A7000F6C2EEF62AEC12F002C0E9F201C0E8F23A
:105A8000060151D0C8C6F1F6C7C6F0F6C6C6EFF695
:105A9000C5C6EEF62AEC12F002C0CAF601C0C9F67D
:105AA000F2CFCBF6F29E756A060E746E7F9C7F9ED7
:105AB0007F8073500601CBBFF28ECC6F030ECD6F8B
:105AC000CAC6CFF6C9C6CEF6CCC6D0F6000148ECA1
:105AD00012F0F2CFC9F6F29E756A0A0E746E7F9CC0
:105AE0007F9E7F8073500601C9BFF28ECA6F030E7E
:105AF000CD6FE9C2CFF6E8C2CEF6CAC6D0F6000135
:105B00008FEC14F0F9C2F1F6F8C2F0F6F7C2EFF636
:105B1000F6C2EEF62AEC12F002C0E9F201C0E8F299
:105B2000060101D00601CA6B030EC96F0001C6EC65
:105B300027F01CD00601C8C6F1F6C7C6F0F6C6C6E7
:105B4000EFF6C5C6EEF600012AEC12F002C0CAF666
:105B500001C0C9F6030E0601CD6F02C0CFF601C029
:105B6000CEF6050ED06F000148EC12F0010103D310
:105B700006019DB1F2D0C8C6F1F6C7C6F0F6C6C69A
:105B8000EFF6C5C6EEF600012AEC12F002C0E3F112
:105B900001C0E2F1F2CFC9F6F29E756A020E746E90
:105BA0007F9C7F9E7F8073500601C9BFF28E300BB1
:105BB000006E003A0F0E00160050FC0FD8B0C5D092
:105BC000040F0001F9EF30F0C8C6F1F6C7C6F0F6D1
:105BD000C6C6EFF6C5C6EEF62AEC12F002C0E7F232
:105BE00001C0E6F20601B1D0C8C6F1F6C7C6F0F6AC
:105BF000C6C6EFF6C5C6EEF62AEC12F002C0CAF62B
:105C000001C0C9F6F2CFCBF6F29E756A050E746E2E
:105C10007F9C7F9E7F8073500601CBBFF28ECC6F3E
:105C2000020ECD6FCAC6CFF6C9C6CEF6CCC6D0F628
:105C3000000148EC12F0060188D0C8C6F1F6C7C6CC
:105C4000F0F6C6C6EFF6C5C6EEF62AEC12F002C0B4
:105C5000CAF601C0C9F6F2CFCBF6F29E756A090EFC
:105C6000746E7F9C7F9E7F8073500601CBBFF28E47
:105C7000CC6F020ECD6FCAC6CFF6C9C6CEF6CCC663
:105C8000D0F600018FEC14F0F5C2F1F6F4C2F0F694
:105C9000F3C2EFF6F2C2EEF62AEC12F002C0E7F21F
:105CA00001C0E6F2060151D0C8C6F1F6C7C6F0F64B
:105CB000C6C6EFF6C5C6EEF62AEC12F002C0CAF66A
:105CC00001C0C9F6F2CFCBF6F29E756A050E746E6E
:105CD0007F9C7F9E7F8073500601CBBFF28ECC6F7E
:105CE000020ECD6FCAC6CFF6C9C6CEF6CCC6D0F668
:105CF000000148EC12F0F2CFC9F6F29E756A090E67
:105D0000746E7F9C7F9E7F8073500601C9BFF28EA8
:105D1000CA6F020ECD6FE7C2CFF6E6C2CEF6CAC694
:105D2000D0F600018FEC14F0F5C2F1F6F4C2F0F6F3
:105D3000F3C2EFF6F2C2EEF62AEC12F002C0E7F27E
:105D400001C0E6F2060101D00601CA6B020EC96F5E
:105D50000001C6EC27F01CD00601C8C6F1F6C7C684
:105D6000F0F6C6C6EFF6C5C6EEF600012AEC12F054
:105D700002C0CAF601C0C9F6020E0601CD6F02C00C
:105D8000CFF601C0CEF6050ED06F000148EC12F040
:105D90000101F1D106019DB1F3D0C8C6F1F6C7C625
:105DA000F0F6C6C6EFF6C5C6EEF600012AEC12F014
:105DB00002C0E5F101C0E4F1F2CFC9F6F29E756AC6
:105DC000020E746E7F9C7F9E7F8073500601C9BF58
:105DD000F28E0C0B006E003200323F0E00160050A7
:105DE000FC0FD8B0C5D0040F00010AEF31F0C8C6CF
:105DF000F1F6C7C6F0F6C6C6EFF6C5C6EEF62AEC53
:105E000012F002C0E5F201C0E4F20601B1D0C8C64A
:105E1000F1F6C7C6F0F6C6C6EFF6C5C6EEF62AEC32
:105E200012F002C0CAF601C0C9F6F2CFCBF6F29E5C
:105E3000756A040E746E7F9C7F9E7F80735006018E
:105E4000CBBFF28ECC6F010ECD6FCAC6CFF6C9C6DE
:105E5000CEF6CCC6D0F6000148EC12F0060188D090
:105E6000C8C6F1F6C7C6F0F6C6C6EFF6C5C6EEF66A
:105E70002AEC12F002C0CAF601C0C9F6F2CFCBF686
:105E8000F29E756A080E746E7F9C7F9E7F807350B1
:105E90000601CBBFF28ECC6F010ECD6FCAC6CFF616
:105EA000C9C6CEF6CCC6D0F600018FEC14F0F1C214
:105EB000F1F6F0C2F0F6EFC2EFF6EEC2EEF62AEC23
:105EC00012F002C0E5F201C0E4F2060151D0C8C6EA
:105ED000F1F6C7C6F0F6C6C6EFF6C5C6EEF62AEC72
:105EE00012F002C0CAF601C0C9F6F2CFCBF6F29E9C
:105EF000756A040E746E7F9C7F9E7F8073500601CE
:105F0000CBBFF28ECC6F010ECD6FCAC6CFF6C9C61D
:105F1000CEF6CCC6D0F6000148EC12F0F2CFC9F6AE
:105F2000F29E756A080E746E7F9C7F9E7F80735010
:105F30000601C9BFF28ECA6F010ECD6FE5C2CFF662
:105F4000E4C2CEF6CAC6D0F600018FEC14F0F1C25E
:105F5000F1F6F0C2F0F6EFC2EFF6EEC2EEF62AEC82
:105F600012F002C0E5F201C0E4F2060101D0060120
:105F7000CA6B010EC96F0001C6EC27F01CD00601E8
:105F8000C8C6F1F6C7C6F0F6C6C6EFF6C5C6EEF649
:105F900000012AEC12F002C0CAF601C0C9F6010ED7
:105FA0000601CD6F02C0CFF601C0CEF6050ED06F50
:105FB000000148EC12F00101DED0C8C6F1F6C7C6F8
:105FC000F0F6C6C6EFF6C5C6EEF62AEC12F002C031
:105FD000CAF601C0C9F6040E0601CB6F02C0CDF6A9
:105FE00001C0CCF60001F8EC28F0DDC1CAF6DCC136
:105FF000C9F618EF2AF002C004F301C003F301014F
:10600000BAD00101B8D0C8C6F1F6C7C6F0F6C6C608
:10601000EFF6C5C6EEF62AEC12F002C0CAF601C0D1
:10602000C9F6010E0601CB6F02C0CDF601C0CCF659
:106030000001F8EC28F0D7C1CAF6D6C1C9F69DEC2C
:106040002AF003C0F1F602C0F0F601C0EFF600C07E
:10605000EEF62AEC12F002C008F301C007F30101CA
:106060008AD0C8C6F1F6C7C6F0F6C6C6EFF6C5C6F2
:10607000EEF62AEC12F002C0CAF601C0C9F606011B
:10608000CB6B02C0CDF601C0CCF60001F8EC28F0D5
:10609000D5C1CAF6D4C1C9F69DEC2AF003C0F1F609
:1060A00002C0F0F601C0EFF600C0EEF62AEC12F0E6
:1060B00002C006F301C005F301015DD0C8C6F1F6C8
:1060C000C7C6F0F6C6C6EFF6C5C6EEF62AEC12F065
:1060D00002C0CAF601C0C9F6030E0601CB6F02C0AA
:1060E000CDF601C0CCF60001F8EC28F0DBC1CAF611
:1060F000DAC1C9F69DEC2AF003C0F1F602C0F0F651
:1061000001C0EFF600C0EEF62AEC12F002C00CF36C
:1061100001C00BF301012FD0C8C6F1F6C7C6F0F6D7
:10612000C6C6EFF6C5C6EEF62AEC12F002C0CAF6F5
:1061300001C0C9F6020E0601CB6F02C0CDF601C048
:10614000CCF60001F8EC28F0D9C1CAF6D8C1C9F6DE
:106150009DEC2AF003C0F1F602C0F0F601C0EFF6A4
:1061600000C0EEF62AEC12F002C00AF301C009F3F7
:10617000010101D001016F2B6F51050802E16F2B66
:1061800004D06F51090801E26F6B6F35006E003665
:10619000FC0E0016C250830B0010C26E000E016E82
:1061A000C150F80B0110C16E000123EF5DF0E8242F
:1061B000F76AF736C90FF66E610EF7220A00F5503E
:1061C000FA6E0800F550F96E8657A657F6576258D2
:1061D000E824F76AF736EB0FF66E610EF7220A0035
:1061E000F550FA6E0800F550F96EA459C459165AC4
:1061F000845AE824F76AF7360D0FF66E620EF7221E
:106200000A00F550FA6E0800F550F96EC85BE85BBD
:106210003A5CA85CE824F76AF7362F0FF66E620E38
:10622000F7220A00F550FA6E0800F550F96EEE5D9F
:106230000E5E605ECE5EE824F76AF736510FF66EAA
:10624000620EF7220A00F550FA6E0800F550F96E5A
:1062500038574859705B945DBA5F026006606260AF
:10626000BC60186104C354F703C353F71FEC0BF071
:1062700003C0D0F602C0CFF601C0CEF600C0CDF606
:10628000D0C656F7CFC655F7CEC654F7CDC653F78E
:1062900007015A6B596B7A0E586F880E576F0001C1
:1062A000E0EC13F003C0D0F602C0CFF601C0CEF68A
:1062B00000C0CDF606018F69F2CFD1F6F29E020E34
:1062C000756EF40E746E7F9C7F9E7F807350D1BF7D
:1062D000F28ECC6FCC53D8B48FD1F2CFD1F6F29EE0
:1062E000020E756EF90E746E7F9C7F9E7F807350D8
:1062F000D1BFF28EC56F020E0701446FF50E436FDA
:106300000001B2EC15F003C0C9F602C0C8F601C026
:10631000C7F600C0C6F6F2CFD1F6F29E020E756E39
:10632000FB0E746E7F9C7F9E7F8073500601D1BFF1
:10633000F28ECA6FC551070BFB0F3CE2050F00013F
:10634000FFEF32F00601CB9135D0D0C648F7CFC66B
:1063500047F7CEC646F7CDC645F7C9C64CF7C8C6FF
:106360004BF7C7C64AF7C6C649F736EC10F004E348
:106370000601CB8103D000010601CB911BD0C9C619
:1063800048F7C8C647F7C7C646F7C6C645F7D0C6DA
:106390004CF7CFC64BF7CEC64AF7CDC649F736EC19
:1063A00010F004E30601CB8103D000010601CB917C
:1063B00001D00601CBA138D0C5A92FD001016C5363
:1063C0000BE16D5309E10601905304E1915302E1A1
:1063D000CAC68FF621D00101F2CFD1F6F29E020E8D
:1063E000756EFA0E746E7F9C7F9E7F8073500601DF
:1063F000D1BFF28E916B906F91C642F790C641F774
:106400000701446B630E436F0001A9EC06F002C064
:1064100091F601C090F6060106D0905304E1915325
:1064200002E1CAC68FF61FD0F2CFD1F6F29E020E5D
:10643000756EFA0E746E7F9C7F9E7F807350D1BF05
:10644000F28E916B906F91C642F790C641F70701AB
:10645000446B630E436F0001A9EC06F002C091F695
:1064600001C090F60601F2CFD1F6F29E030E756ED2
:10647000746A7F9C7F9E7F807350D1BFF28EC56F00
:10648000020E0701446FFC0E436F0001B2EC15F0E1
:1064900003C0C9F602C0C8F601C0C7F600C0C6F600
:1064A000F2CFD1F6F29E030E756E020E746E7F9CD3
:1064B0007F9E7F8073500601D1BFF28ECA6F8F51CD
:1064C000CA5DD8B099D0C551070BFB0F3CE2050F50
:1064D000000111EF33F00601CB9135D0D0C648F75B
:1064E000CFC647F7CEC646F7CDC645F7C9C64CF767
:1064F000C8C64BF7C7C64AF7C6C649F736EC10F010
:1065000004E30601CB8103D000010601CB911BD02F
:10651000C9C648F7C8C647F7C7C646F7C6C645F74F
:10652000D0C64CF7CFC64BF7CEC64AF7CDC649F713
:1065300036EC10F004E30601CB8103D00001060124
:10654000CB9101D00601CBA138D0C5A92FD0010134
:106550006C530BE16D5309E10601925304E193532F
:1065600002E1CAC68FF621D00101F2CFD1F6F29E28
:10657000030E756E010E746E7F9C7F9E7F8073503C
:106580000601D1BFF28E936B926F93C642F792C60B
:1065900041F70701446B630E436F0001A9EC06F05D
:1065A00002C093F601C092F6060106D0925304E1B0
:1065B000935302E1CAC68FF61FD0F2CFD1F6F29EF6
:1065C000030E756E010E746E7F9C7F9E7F807350EC
:1065D000D1BFF28E936B926F93C642F792C641F78A
:1065E0000701446B630E436F0001A9EC06F002C083
:1065F00093F601C092F60601000125EF5DF0E82454
:10660000F76AF736190FF66E660EF7220A00F55094
:10661000FA6E0800F550F96E44634A634A637E637C
:106620007E63E824F76AF7363D0FF66E660EF722B2
:106630000A00F550FA6E0800F550F96ED664DC6475
:10664000DC6410651065B60E006E036A026A016AAA
:106650000601EE51EF11F011F11102E1006A0DD0C7
:10666000D89001BE09D0EE37EF37F037F137033657
:1066700002360136002EF4D7019E00011200F2CF3F
:10668000CEF6F29E020E756E8C0E746E7F9C7F9E0F
:106690007F8073500601CEBFF28EC76FF2CFCEF669
:1066A000F29E020E756EB30E746E7F9C7F9E7F808D
:1066B0007350CEBFF28ECF6FF2CFD0F6F29E020EA5
:1066C000756EB20E746E7F9C7F9E7F807350D0BFBC
:1066D000F28ED16FCFC6CDF6D1C6CCF6C751000A27
:1066E000000101E006D0FE0E0101686F67697AD0F3
:1066F0000001C6C654F7C5C653F71FEC0BF003C024
:10670000CBF602C0CAF601C0C9F600C0C8F6CDC6B5
:1067100054F7CCC653F71FEC0BF0CBC656F7CAC6DE
:1067200055F7C9C654F7C8C653F703C05AF702C095
:1067300059F701C058F700C057F7E0EC13F003C059
:10674000CBF602C0CAF601C0C9F600C0C8F6CBC677
:1067500056F7CAC655F7C9C654F7C8C653F7070156
:106760005A6B596B700E586F840E576F0001AFEC67
:1067700011F003C0CBF602C0CAF601C0C9F600C0D2
:10678000C8F6020E0701446F8D0E436F0001B2EC94
:1067900015F0CBC656F7CAC655F7C9C654F7C8C6D2
:1067A00053F703C05AF702C059F701C058F700C0A9
:1067B00057F7AFEC11F003C0CBF602C0CAF601C028
:1067C000C9F600C0C8F6CBC6F1F6CAC6F0F6C9C60F
:1067D000EFF6C8C6EEF62AEC12F002C068F101C06E
:1067E00067F10101000166EF5DF001016E69F2CF12
:1067F000CDF6F29E020E756E8C0E746E7F9C7F9E9F
:106800007F8073500601CDBFF28ECC6FCC53D8B4CD
:10681000CAD1F2CFCDF6F29E020E756EA80E746E3E
:106820007F9C7F9E7F807350CDBFF28EC56F020E1E
:106830000701446FA40E436F0001B2EC15F003C0D2
:10684000C9F602C0C8F601C0C7F600C0C6F6F2CF4E
:10685000CDF6F29E020E756EAA0E746E7F9C7F9E20
:106860007F8073500601CDBFF28ECA6FC551070BF2
:10687000FB0F58E2050F0001D6EF35F00601CB9172
:1068800051D068C154F767C153F71FEC0BF003C038
:10689000D0F602C0CFF601C0CEF600C0CDF603C0E0
:1068A00048F702C047F701C046F700C045F7C9C620
:1068B0004CF7C8C64BF7C7C64AF7C6C649F736EC09
:1068C00010F004E30601CB8103D000010601CB9157
:1068D00029D068C154F767C153F71FEC0BF003C010
:1068E000D0F602C0CFF601C0CEF600C0CDF6C9C6C4
:1068F00048F7C8C647F7C7C646F7C6C645F703C038
:106900004CF702C04BF701C04AF700C049F736EC1C
:1069100010F004E30601CB8103D000010601CB9106
:1069200001D00601CBA138D0C5A92FD001016C53ED
:106930000BE16D5309E10601685304E1695302E17B
:10694000CAC66EF121D00101F2CFCDF6F29E020E41
:10695000756EA90E746E7F9C7F9E7F8073500601BA
:10696000CDBFF28E696B686F69C642F768C641F7A2
:106970000701446B630E436F0001A9EC06F002C0EF
:1069800069F601C068F6060106D0685304E1695350
:1069900002E1CAC66EF11FD0F2CFCDF6F29E020E12
:1069A000756EA90E746E7F9C7F9E7F807350CDBFE5
:1069B000F28E696B686F69C642F768C641F70701D6
:1069C000446B630E436F0001A9EC06F002C069F648
:1069D00001C068F60601F2CFCDF6F29E020E756E8A
:1069E000AF0E746E7F9C7F9E7F807350CDBFF28E02
:1069F000C56F020E0701446FAB0E436F0001B2EC8E
:106A000015F003C0C9F602C0C8F601C0C7F600C041
:106A1000C6F6F2CFCDF6F29E020E756EB10E746E12
:106A20007F9C7F9E7F8073500601CDBFF28ECA6F20
:106A300001016E510601CA5DD8B0B5D0C551070B32
:106A4000FB0F58E2050F0001E8EF35F00601CB918E
:106A500051D068C154F767C153F71FEC0BF003C066
:106A6000D0F602C0CFF601C0CEF600C0CDF603C00E
:106A700048F702C047F701C046F700C045F7C9C64E
:106A80004CF7C8C64BF7C7C64AF7C6C649F736EC37
:106A900010F004E30601CB8103D000010601CB9185
:106AA00029D068C154F767C153F71FEC0BF003C03E
:106AB000D0F602C0CFF601C0CEF600C0CDF6C9C6F2
:106AC00048F7C8C647F7C7C646F7C6C645F703C066
:106AD0004CF702C04BF701C04AF700C049F736EC4B
:106AE00010F004E30601CB8103D000010601CB9135
:106AF00001D00601CBA138D0C5A92FD001016C531C
:106B00000BE16D5309E106016A5304E16B5302E1A5
:106B1000CAC66EF121D00101F2CFCDF6F29E020E6F
:106B2000756EA90E746E7F9C7F9E7F8073500601E8
:106B3000CDBFF28E6B6B6A6F6BC642F76AC641F7C8
:106B40000701446B630E436F0001A9EC06F002C01D
:106B50006BF601C06AF6060106D06A5304E16B5376
:106B600002E1CAC66EF11FD0F2CFCDF6F29E020E40
:106B7000756EB00E746E7F9C7F9E7F807350CDBF0C
:106B8000F28E6B6B6A6F6BC642F76AC641F70701FC
:106B9000446B630E436F0001A9EC06F002C06BF674
:106BA00001C06AF60601000168EF5DF0E824F76AAB
:106BB000F736C70FF66E6B0EF7220A00F550FA6E25
:106BC0000800F550F96E7C6882688268D268D268E5
:106BD000E824F76AF736EB0FF66E6B0EF7220A0021
:106BE000F550FA6E0800F550F96E4C6A526A526A16
:106BF000A26AA26AF2CFC7F6F29E756A3F0E746E61
:106C00007F9C7F9E7F8073500601C7BFF28EC56F49
:106C1000C551000A00011DE0010A1EE0030A5CE004
:106C2000010AD8B4A2D0070AD8B4E6D0010AD8B471
:106C30002AD1030AD8B46ED1010AD8B4B2D10F0A4E
:106C4000D8B4EFD1010AD8B42DD2030AD8B46BD28C
:106C5000ACD20601C681ABD20701446B400E436F34
:106C60000001B2EC15F003C0F1F602C0F0F601C06D
:106C7000EFF600C0EEF62AEC12F00250036E0101AE
:106C8000685D08E303E16751015C04E20601C68127
:106C900022D001010601C691F2CFC7F6F29E756AB5
:106CA000440E746E7F9C7F9E7F807350C7BFF28EB0
:106CB00001016D6B6C6F6DC142F76CC141F707014B
:106CC000446B630E436F0001A9EC06F002C06DF146
:106CD00001C06CF106016BD20101693D06D06A5119
:106CE000FE0803E10601C6813FD00701446B400E58
:106CF000436F0001B2EC15F003C0F1F602C0F0F6EC
:106D000001C0EFF600C0EEF62AEC12F00250036E5E
:106D100001016A5D08E303E16951015C04E20601D7
:106D2000C68122D001010601C691F2CFC7F6F29EBC
:106D3000756A440E746E7F9C7F9E7F807350C7BFC0
:106D4000F28E01016D6B6C6F6DC142F76CC141F742
:106D50000701446B630E436F0001A9EC06F002C00B
:106D60006DF101C06CF1060122D203011F3D41D03B
:106D70000701446B400E436F0001B2EC15F003C0F5
:106D800048F702C047F701C046F700C045F712C3F5
:106D90004CF711C34BF710C34AF70FC349F736EC52
:106DA00010F004E30601C68122D000010601C6915D
:106DB000F2CFC7F6F29E756A440E746E7F9C7F9E7A
:106DC0007F807350C7BFF28E01016D6B6C6F6DC118
:106DD00042F76CC141F70701446B630E436F00013A
:106DE000A9EC06F002C06DF101C06CF1060103D000
:106DF00003010601C681DBD10301203D41D007011B
:106E0000446B400E436F0001B2EC15F003C048F72D
:106E100002C047F701C046F700C045F716C34CF75C
:106E200015C34BF714C34AF713C349F736EC10F0F8
:106E300004E30601C68122D000010601C691F2CF0B
:106E4000C7F6F29E756A440E746E7F9C7F9E7F80AB
:106E50007350C7BFF28E01016D6B6C6F6DC142F74D
:106E60006CC141F70701446B630E436F0001A9EC4D
:106E700006F002C06DF101C06CF1060103D0030100
:106E80000601C68194D10301213D41D00701446B25
:106E9000400E436F0001B2EC15F003C048F702C08A
:106EA00047F701C046F700C045F71AC34CF719C3AE
:106EB0004BF718C34AF717C349F736EC10F004E351
:106EC0000601C68122D000010601C691F2CFC7F6A5
:106ED000F29E756A440E746E7F9C7F9E7F80735015
:106EE000C7BFF28E01016D6B6C6F6DC142F76CC153
:106EF00041F70701446B630E436F0001A9EC06F0F4
:106F000002C06DF101C06CF1060103D0030106015E
:106F1000C6814DD10301223D41D00701446B400E93
:106F2000436F0001B2EC15F003C048F702C047F709
:106F300001C046F700C045F71EC34CF71DC34BF711
:106F40001CC34AF71BC349F736EC10F004E30601F3
:106F5000C68122D000010601C691F2CFC7F6F29E8B
:106F6000756A440E746E7F9C7F9E7F807350C7BF8E
:106F7000F28E01016D6B6C6F6DC142F76CC141F710
:106F80000701446B630E436F0001A9EC06F002C0D9
:106F90006DF101C06CF1060103D003010601C68149
:106FA00006D10701446BA70E436F0001B2EC15F048
:106FB00012C348F711C347F710C346F70FC345F78D
:106FC00003C04CF702C04BF701C04AF700C049F7B5
:106FD00036EC10F004E10601C68122D00001060162
:106FE000C691F2CFC7F6F29E756A440E746E7F9C0E
:106FF0007F9E7F807350C7BFF28E01016D6B6C6FF7
:107000006DC142F76CC141F70701446B630E436FDA
:107010000001A9EC06F002C06DF101C06CF106019F
:10702000C6D0010E0701446F360E436F0001B2EC6B
:1070300015F016C348F715C347F714C346F713C333
:1070400045F703C04CF702C04BF701C04AF700C038
:1070500049F736EC10F004E10601C68122D00001A8
:107060000601C691F2CFC7F6F29E756A440E746EA1
:107070007F9C7F9E7F807350C7BFF28E01016D6B36
:107080006C6F6DC142F76CC141F70701446B630E31
:10709000436F0001A9EC06F002C06DF101C06CF174
:1070A000060185D0010E0701446FC50E436F000134
:1070B000B2EC15F01AC348F719C347F718C346F7DF
:1070C00017C345F703C04CF702C04BF701C04AF79E
:1070D00000C049F736EC10F004E10601C68122D069
:1070E00000010601C691F2CFC7F6F29E756A440E02
:1070F000746E7F9C7F9E7F807350C7BFF28E0101AC
:107100006D6B6C6F6DC142F76CC141F70701446B49
:10711000630E436F0001A9EC06F002C06DF101C0DF
:107120006CF1060144D0020E0701446F540E436F08
:107130000001B2EC15F01EC348F71DC347F71CC38E
:1071400046F71BC345F703C04CF702C04BF701C01D
:107150004AF700C049F736EC10F004E10601C68199
:1071600022D000010601C691F2CFC7F6F29E756AE1
:10717000440E746E7F9C7F9E7F807350C7BFF28EDB
:1071800001016D6B6C6F6DC142F76CC141F7070176
:10719000446B630E436F0001A9EC06F002C06DF171
:1071A00001C06CF1060103D000010601C681000E8A
:1071B000C6B1010E016E00016AEF5DF00601C591D6
:1071C00019AE01D1199EF2CFCAF6F29E030E756E6A
:1071D0001C0E746E7F9C7F9E7F807350CABFF28EA0
:1071E000F60FD8B0DDD00A0F0001E6EF39F0060146
:1071F000C591D6D00101673D03D06851FE082DE04E
:10720000030E0701446F1D0E436F0001B2EC15F031
:1072100003C0C9F602C0C8F601C0C7F600C0C6F672
:1072200068C154F767C153F71FEC0BF0C9C648F7A4
:10723000C8C647F7C7C646F7C6C645F703C04CF7EA
:1072400002C04BF701C04AF700C049F736EC10F016
:1072500003E30601C581000101010601A1D0030E6F
:107260000701446F1D0E436F0001B2EC15F003C01F
:10727000C9F602C0C8F601C0C7F600C0C6F6C9C646
:1072800048F7C8C647F7C7C646F7C6C645F712C38C
:107290004CF711C34BF710C34AF70FC349F736EC4D
:1072A00010F003E30601C5810001060179D0030E49
:1072B0000701446F1D0E436F0001B2EC15F003C0CF
:1072C000C9F602C0C8F601C0C7F600C0C6F6C9C6F6
:1072D00048F7C8C647F7C7C646F7C6C645F716C338
:1072E0004CF715C34BF714C34AF713C349F736ECF1
:1072F00010F003E30601C5810001060151D0030E21
:107300000701446F1D0E436F0001B2EC15F003C07E
:10731000C9F602C0C8F601C0C7F600C0C6F6C9C6A5
:1073200048F7C8C647F7C7C646F7C6C645F71AC3E3
:107330004CF719C34BF718C34AF717C349F736EC94
:1073400010F003E30601C5810001060129D0030EF8
:107350000701446F1D0E436F0001B2EC15F003C02E
:10736000C9F602C0C8F601C0C7F600C0C6F6C9C655
:1073700048F7C8C647F7C7C646F7C6C645F71EC38F
:107380004CF71DC34BF71CC34AF71BC349F736EC38
:1073900010F003E30601C5810001060101D00601DA
:1073A000C5A111D0942B9451B3080DE2946B952B89
:1073B00006E1962B965303E1972B01E1982B0001F0
:1073C00087EC0FF00601000171EF5DF0E824F76A29
:1073D000F736E70FF66E730EF7220A00F550FA6ED5
:1073E0000800F550F96EEE71F4715E72AE72FE72C5
:1073F0004E735E72AE72FE724E730601D76BD66B21
:10740000D56BD46BD2C6D9F6D1C6D8F6D353D8B47F
:107410009BD0D9C603F0D8C6E9FF03C0EAFFD76BFB
:10742000D66BD56BEFCFD4F6D851D8B4D907D807DF
:10743000D9C603F0D8C6E9FF03C0EAFFEF50DC6B02
:10744000DB6BDCC603F0DBC602F0016E006A0050A5
:10745000D4130150D5130250D6130350D713D8516B
:10746000D8B4D907D807D9C603F0D8C6E9FF03C0F6
:10747000EAFFEF50DD6BDC6BDB6BDA6F030EDA17C4
:10748000DB6BDC6BDD6BDBC603F0DAC602F0006A97
:10749000016A0050D4130150D5130250D613035083
:1074A000D713D9C603F0D8C6E9FF03C0EAFFEF50EF
:1074B000DD6BDC6BDB6BDA6FE00EDA17DB6BDC6B42
:1074C000DD6B006ADA35016EDB35026EDC35036E8A
:1074D00001360236033601360236033601360236ED
:1074E0000336013602360336E00E01160050D4137F
:1074F0000150D5130250D6130350D713D851D8B426
:10750000D907D807D9C603F0D8C6E9FF03C0EAFFF8
:10751000EF50DB6BDA6F006A016ADA35026EDB3539
:10752000036E02360336023603360236033602365F
:107530000336E00E02160050D4130150D51302504A
:10754000D6130350D71357D0020ED85F000ED95B65
:10755000D9C603F0D8C6E9FF03C0EAFFEF50DD6BE0
:10756000DC6BDB6BDA6FE00EDA17DB6BDC6BDD6B91
:10757000DD31D76FDC31D66FDB31D56FDA31D46FC7
:10758000D733D633D533D433D733D633D533D433B7
:10759000D733D633D533D433D733D633D533D433A7
:1075A000070ED717D851D8B4D907D807D9C603F0D2
:1075B000D8C6E9FF03C0EAFFEF50DD6BDC6BDB6B85
:1075C000DA6FDA35006EDB35016EDC35026EDD35E3
:1075D000036E0036013602360336003601360236B7
:1075E0000336F80E00160050D4130150D513025084
:1075F000D6130350D713D4C600F0D5C601F0D6C6B3
:1076000002F0D7C603F0000189EF5EF003012851B4
:10761000F0080FE1293D0DD02A530BE12B5309E16E
:107620001986010E2C6F19880601566B556B07D011
:107630000301199619980601566B556B198C0001B8
:10764000B6EF5FF00601C86BC76BC66BC56B020E69
:107650000301255D006E000E2659036E00C001F087
:107660000601C651035C12E303E10150C55D0EE261
:107670002D0EC525E96E030EC621EA6EEF50C72711
:10768000000EC823C52BD8B4C62BE1D7C71FC81F0F
:10769000010EC727000EC823010E0301255D060158
:1076A000C96F000E030126590601CA6F2D0EC925A8
:1076B000E96E030ECA21EA6EEFCF03F0020E03015A
:1076C000255D0601CC6F000E030126590601CD6F22
:1076D0002D0ECC25E96E030ECD21EA6EEFCFCEF64E
:1076E000CE51C75DD8A487D00350C85DD8A483D03D
:1076F000C66BC56B020E0301255D006E000E265998
:10770000036E00C001F00601C651035C29E303E1EA
:107710000150C55D25E22D0EC525E96E030EC6217B
:10772000EA6EEFCFC9F6F250006EF29EC6C675FF44
:10773000C5C674FFC9C673FF7F9C7F9E7F840F01FF
:10774000550E7E6EAA0E7E6E7F827FB2FED77F942C
:107750000050F21204000601C52BD8B4C62BCAD7BC
:10776000020E0301255D0601C96F000E03012659B3
:107770000601CA6FC7C6CBF6F250006EF29ECAC6AB
:1077800075FFC9C674FFCBC673FF7F9C7F9E7F8445
:107790000F01550E7E6EAA0E7E6E7F827FB2FED7DF
:1077A0007F940050F212010E0301255D0601C96F9E
:1077B000000E030126590601CA6FC8C6CBF6F25067
:1077C000006EF29ECAC675FFC9C674FFCBC673FFB2
:1077D0007F9C7F9E7F840F01550E7E6EAA0E7E6E6B
:1077E0007F827FB2FED77F940050F212010E016EAD
:1077F00005D004D00601000E016E0F010001FEEF5E
:107800005FF02E50000A06E0010A52E0030AD8B4E5
:1078100079D089D02F50010A05E0030A14E0060A46
:1078200023E034D0010E0601C56FC55104080AE3F8
:10783000C5C6CFF6010ED06F0001AEEC09F006010F
:10784000C52BF3D733D0010E0601C56FC55104080F
:107850000AE3C5C6CFF6020ED06F0001AEEC09F008
:107860000601C52BF3D722D0010E0601C56FC55105
:1078700004080AE3C5C6CFF6040ED06F0001AEECD3
:1078800009F00601C52BF3D711D00001010E060146
:10789000C56FC55104080AE3C5C6CFF6030ED06F05
:1078A0000001AEEC09F00601C52BF3D700013BD077
:1078B00030C0C7F62FC0C6F60601C733C633C7337C
:1078C000C633C733C6C6BCFFC733C731300B006EE3
:1078D000BB50CF0B0010BB6E32C0C7F631C0C6F62E
:1078E000C733C633C733C633C733C6C651FFC733E2
:1078F000C731300B006E0F015051CF0B0010506F8D
:10790000000111D02F5209E1959C8C8C010E0601CB
:107910009F6FF40E9E6F06D000012F2C02D0959C15
:107920008C9C0601000116EF61F0010E0601F26F5A
:10793000E16BE06BE15344E1E051030841E3E1C650
:1079400042F7E0C641F70701446B8F0E436F000119
:10795000A9EC06F002C003F00150500F0601F36FCE
:10796000000E0320F46FF2CFF5F6F29EF4C675FF19
:10797000F3C674FF7F9C7F9E7F807350F5BFF28EAD
:10798000000A0EE0E0C6FEF6010EFF6F030E0701CF
:10799000016F230E006F0001BDEC13F00CD0060147
:1079A000E0C6FEF6FF6B030E0701016F230E006FAA
:1079B0000001BDEC13F00601E02BD8B4E12BBAD7DF
:1079C000E16BE06BE153D8A443D1E0510308D8A0A8
:1079D0003FD1E035026EE135036E02360336FC0E10
:1079E00002160250E20FE96E060E0320EA6EE1C6AF
:1079F00042F7E0C641F70701446B8F0E436F000169
:107A0000A9EC06F002C003F00150500F0601F56F1B
:107A1000000E0320F66F040EF527000EF623020E6B
:107A2000F527000EF623F2CFF7F6F29EF6C675FFA5
:107A3000F5C674FF7F9C7F9E7F807350F7BFF28EE8
:107A4000010BEE52EE52EC6AED52EF6AED52EF6A24
:107A5000ED52EF6EE035026EE135036E023603360D
:107A6000FC0E02160250E20FE96E060E0320EA6ECB
:107A7000EE52ECCF03F0ED52EFCF02F0ED52EFCF2C
:107A800001F0006A00C0EFFF01C0ECFF02C0ECFF94
:107A900003C0ECFFE035026EE135036E02360336BB
:107AA000FC0E02160250E20FE96E060E0320EA6E8B
:107AB000E1C642F7E0C641F70701446B8F0E436F02
:107AC0000001A9EC06F002C003F00150500F0601BE
:107AD000F96F000E0320FA6F040EF927000EFA2347
:107AE000010EF927000EFA23F2CFFBF6F29EFAC63A
:107AF00075FFF9C674FF7F9C7F9E7F807350FBBF2C
:107B0000F28EEF24006E000EEC20016E000EEC20D1
:107B1000026E000EEC20036EED52ED52ED5200C0ED
:107B2000EFFF01C0ECFF02C0ECFF03C0ECFFED5221
:107B3000ED52ED52E035026EE135036E023603364A
:107B4000FC0E02160250E20FE96E060E0320EA6EEA
:107B5000EE52ECCF03F0ED52EFCF02F0ED52EFCF4B
:107B600001F0006A00C0EFFF01C0ECFF02C0ECFFB3
:107B700003C0ECFFE035026EE135036E02360336DA
:107B8000FC0E02160250E20FE96E060E0320EA6EAA
:107B9000E1C642F7E0C641F70701446B8F0E436F21
:107BA0000001A9EC06F002C003F00150500F0601DD
:107BB000F96F000E0320FA6F040EF927000EFA2366
:107BC000F2CFFBF6F29EFAC675FFF9C674FF7F9CF2
:107BD0007F9E7F807350FBBFF28EEF24006E000EFD
:107BE000EC20016E000EEC20026E000EEC20036E05
:107BF000ED52ED52ED5200C0EFFF01C0ECFF02C0AC
:107C0000ECFF03C0ECFFED52ED52ED52E0C6F3F68F
:107C1000030EF56F230EF46F0001A2EC13F001A028
:107C20000BD04A0E0601E025E96E000EE121EA6E56
:107C3000010EEF6E09D000014A0E0601E025E96E43
:107C4000000EE121EA6EEF6AE02BD8B4E12BBAD640
:107C5000E651E25D12E1E751E35D0FE1E851E45DD9
:107C60000CE1E951E55D09E1030123B302D006010E
:107C700004D04A2A0601F2834B6AEA51E25D12E11E
:107C8000EB51E35D0FE1EC51E45D0CE1ED51E55D9D
:107C900009E1030123B502D0060104D04A2A0601F6
:107CA000F2854C6AEE51E25D12E1EF51E35D0FE1C6
:107CB000F051E45D0CE1F151E55D09E1030123B709
:107CC00002D0060104D04A2A0601F2874D6AF2B3B7
:107CD0002ED0F2B515D0EA51E65D12E1EB51E75D29
:107CE0000FE1EC51E85D0CE1ED51E95D09E10301C3
:107CF00023B502D0060104D04B2A0601F2854C6A56
:107D0000F2B715D0EE51E65D12E1EF51E75D0FE1FC
:107D1000F051E85D0CE1F151E95D09E1030123B7A0
:107D200002D0060104D04B2A0601F2874D6AF2B553
:107D300017D0F2B715D0EE51EA5D12E1EF51EB5DCD
:107D40000FE1F051EC5D0CE1F151ED5D09E1030152
:107D500023B702D0060104D04C2A0601F2874D6AEF
:107D60000001B9EF3FF00601E551010A000117E0FB
:107D7000030A1AE0010A1DE0070A20E0010A23E0D5
:107D8000030A26E0010A29E00F0A2CE0010A2FE08D
:107D9000030A33E0010A37E0070A3BE041D006015D
:107DA000E76B010EE66F3FD00601E76B020EE66F50
:107DB0003AD00601E76B050EE66F35D00601E76B9A
:107DC0000A0EE66F30D00601E76B140EE66F2BD07B
:107DD0000601E76B320EE66F26D00601E76B640EF4
:107DE000E66F21D00601E76BC80EE66F1CD0010ECE
:107DF0000601E76FF40EE66F16D0030E0601E76F7B
:107E0000E80EE66F10D0070E0601E76FD00EE66FA2
:107E10000AD00B0E0601E76FB80EE66F04D0000122
:107E20000601E769E669E6C601F0E7C602F000016F
:107E300012000601E051B608E06F036AE1C6E4F6FD
:107E4000E18FD890E133E233E3330332023201327F
:107E50000032E02FF6D7E4AF0BD0001E011E021E49
:107E6000031E002AD8B4012AD8B4022AD8B4032A9F
:107E7000000112004E50040DF350036A500FE96EDA
:107E8000000E0320EA6EF3C6EFFFF4C6ECFFF5C662
:107E9000ECFFF6C6ECFF0601FD6BFD51070827E37A
:107EA0004E50080DF350FF6BFE6F036AFD51FE2527
:107EB000016EFF5103220150900F016E000E03224C
:107EC00003C0FFF6F8C603F0F7C6E9FF03C0EAFFF8
:107ED000EFCF00F70701FFC6EAFF01C0E9FF00C7C7
:107EE000EFFF0601F72BD8B4F82BFD2BD6D7036A8A
:107EF0004E50100FE96E010E0320EA6EF9C6EFFF37
:107F0000036A4E50200FE96E010E0320EA6EFAC696
:107F1000EFFF4EC0FEF6FBC6FFF6010E0701016F34
:107F2000300E006F0001BDEC13F04EC0FEF6FCC633
:107F3000FFF6010E0701016F320E006F0001BDEC6C
:107F400013F04E2A4E500F0801E24E6A120006014D
:107F5000EF6BEF5107080AE3036AEF51240FE96E54
:107F6000000E0320EA6EEF68EF2BF3D7000112003A
:107F7000DCD40601C66BC56BC653D8A447EF45F0E9
:107F8000C5510308D8A047EF45F0C6C642F7C5C69D
:107F900041F70701446B8F0E436F0001A9EC06F017
:107FA00002C003F00150500F0601E06F000E0320E5
:107FB000E16FF2CFE2F6F29EE1C675FFE0C674FF14
:107FC0007F9C7F9E7F807350E2BFF28EC76FC75346
:107FD000D8B442EF45F0C7510808D8A042EF45F0A9
:107FE0004A0EC525E96E000EC621EA6EEF52D8B4DE
:107FF00042EF45F0D890C535026EC635036E02508B
:10800000340FE96E000E0320EA6EECCFE1F6ED527C
:10801000EFCFE0F6E053D8A442EF45F0E153D8A407
:1080200042EF45F0D890C535026EC635036E02505A
:10803000340F016E000E03220150E06F03C0E1F621
:10804000C6C642F7C5C641F70701446B8F0E436FA2
:108050000001A9EC06F002C003F00150500F060128
:10806000E26F000E0320E36F0A0EE227000EE32307
:10807000F2CFE4F6F29EE3C675FFE2C674FF7F9C82
:108080007F9E7F807350E4BFF28EE26FE2C6E5F61A
:10809000000169DEE1C6EAFFE0C6E9FF02C0ECFFCD
:1080A000ED5201C0EFFFC6C642F7C5C641F7070152
:1080B000446B8F0E436F0001A9EC06F002C003F081
:1080C0000150500F0601E06F000E0320E16F090E12
:1080D000E027000EE123F2CFE2F6F29EE1C675FF43
:1080E000E0C674FF7F9C7F9E7F807350E2BFF28E5C
:1080F0001F6A1E6A1D6A1C6E070E1C161D6A1E6A08
:108100001F6A1C361D361E361F361C361D361E369F
:108110001F36FC0E1C16C6C642F7C5C641F707013E
:10812000446B8F0E436F0001A9EC06F002C003F010
:108130000150500F0601E06F000E0320E16F040EA6
:10814000E027000EE123020EE027000EE123F2CF2C
:10815000E2F6F29EE1C675FFE0C674FF7F9C7F9E4B
:108160007F807350E2BFF28E010B1C26000E1D2291
:10817000000E1E22000E1F221EC01FF01DC01EF08A
:108180001CC01DF01C6AC6C642F7C5C641F70701F0
:10819000446B8F0E436F0001A9EC06F002C003F0A0
:1081A0000150500F0601E06F000E0320E16F040E36
:1081B000E027000EE123010EE027000EE123F2CFBD
:1081C000E2F6F29EE1C675FFE0C674FF7F9C7F9EDB
:1081D0007F807350E2BFF28E1C26000E1D22000E1F
:1081E0001E22000E1F221EC01FF01DC01EF01CC04C
:1081F0001DF01C6AC6C642F7C5C641F70701446BAD
:108200008F0E436F0001A9EC06F002C003F001508D
:10821000500F0601E06F000E0320E16F040EE0270F
:10822000000EE123F2CFE2F6F29EE1C675FFE0C652
:1082300074FF7F9C7F9E7F807350E2BFF28E1C266E
:10824000000E1D22000E1E22000E1F221EC01FF057
:108250001DC01EF01CC01DF01C6A1B501C26000E09
:108260001D221E221F22CA6BCA5107080AE3036A95
:10827000CA51240FE96E000E0320EA6EEF68CA2B84
:10828000F3D7DB6BDA6B030ED880C555006E000E9A
:10829000C655036E00C001F0DB51035CD8A02CEF83
:1082A00045F005E1DA51015CD8A02CEF45F0DA5138
:1082B000C525E06FDB51C621E16FE1C642F7E0C69C
:1082C00041F70701446B8F0E436F0001A9EC06F0E4
:1082D00002C003F00150500F0601E06F000E0320B2
:1082E000E16F040EE027000EE123020EE027000EEE
:1082F000E123F2CFE2F6F29EE1C675FFE0C674FF1D
:108300007F9C7F9E7F807350E2BFF28E010BDC6FFB
:10831000DD6BDE6BDF6BDEC6DFF6DDC6DEF6DCC6F0
:10832000DDF6DC6BDA51C525E06FDB51C621E16F6C
:10833000E1C642F7E0C641F70701446B8F0E436F79
:108340000001A9EC06F002C003F00150500F060135
:10835000E06F000E0320E16F040EE027000EE12322
:10836000010EE027000EE123F2CFE2F6F29EE1C615
:1083700075FFE0C674FF7F9C7F9E7F807350E2BFD5
:10838000F28EDC27000EDD23000EDE23000EDF233D
:10839000DEC6DFF6DDC6DEF6DCC6DDF6DC6BDA5106
:1083A000C525E06FDB51C621E16FE1C642F7E0C6AB
:1083B00041F70701446B8F0E436F0001A9EC06F0F3
:1083C00002C003F00150500F0601E06F000E0320C1
:1083D000E16F040EE027000EE123F2CFE2F6F29EF9
:1083E000E1C675FFE0C674FF7F9C7F9E7F8073505F
:1083F000E2BFF28EDC27000EDD23000EDE23000E2E
:10840000DF23DEC6E3F6DDC6E2F6DCC6E1F6E06BAE
:10841000010EE317006A1DC001F01EC002F01F50DC
:10842000010B036E0050E05DD8A412D30150E15D52
:10843000D8A40ED30250E25DD8A40AD30350E35D62
:10844000D8A406D3DA51C525E06FDB51C621E16F10
:10845000E0C6F3F6030EF56F230EF46F0001A2ECF5
:1084600013F00150010B0108D8B402D00601F0D27C
:108470000601DA51C525E06FDB51C621E16FE1C687
:1084800042F7E0C641F70701446B8F0E436F0001CE
:10849000A9EC06F002C003F00150500F0601E06F96
:1084A000000E0320E16F070EE027000EE123F2CF5C
:1084B000E2F6F29EE1C675FFE0C674FF7F9C7F9EE8
:1084C0007F807350E2BFF28EC86FDA51C525E06F2E
:1084D000DB51C621E16FE1C642F7E0C641F7070173
:1084E000446B8F0E436F0001A9EC06F002C003F04D
:1084F0000150500F0601E06F000E0320E16F080EDF
:10850000E027000EE123F2CFE2F6F29EE1C675FF0E
:10851000E0C674FF7F9C7F9E7F807350E2BFF28E27
:10852000C96FDA51C525E06FDB51C621E16F1F0E1F
:10853000E025E96E030EE121EA6EEF5003080FE03B
:10854000DA51C525E26FDB51C621E36F1F0EE2252C
:10855000E96E030EE321EA6EEF5004082EE1C951E3
:10856000080A000107E0180A0CE0080A11E0380ABE
:1085700016E01DD00601D16BD06BCF6BFE0ECE6F17
:108580001BD00601D16BD06BFE0ECF6FCE6914D01D
:108590000601D16BFE0ED06FCF69CE690DD0FE0EF5
:1085A0000601D16FD069CF69CE6906D000010601FE
:1085B000D169D069CF69CE690BD2DA51C525E06F98
:1085C000DB51C621E16FE1C642F7E0C641F7070182
:1085D000446B8F0E436F0001A9EC06F002C003F05C
:1085E0000150500F0601E06F000E0320E16F100EE6
:1085F000E027000EE123030EE027000EE123F2CF77
:10860000E2F6F29EE1C675FFE0C674FF7F9C7F9E96
:108610007F807350E2BFF28EE06FDA51C525E36FC1
:10862000DB51C621E46FE4C642F7E3C641F7070118
:10863000446B8F0E436F0001A9EC06F002C003F0FB
:108640000150500F0601E36F000E0320E46F100E7F
:10865000E327000EE423020EE327000EE423F2CF0B
:10866000E1F6F29EE4C675FFE3C674FF7F9C7F9E31
:108670007F807350E1BFF28EE36FDA51C525E46F5E
:10868000DB51C621E56FE5C642F7E4C641F70701B5
:10869000446B8F0E436F0001A9EC06F002C003F09B
:1086A0000150500F0601E46F000E0320E56F100E1D
:1086B000E427000EE523010EE427000EE523F2CFA8
:1086C000E6F6F29EE5C675FFE4C674FF7F9C7F9ECA
:1086D0007F807350E6BFF28EE46FDA51C525E76FF5
:1086E000DB51C621E86FE8C642F7E7C641F707014C
:1086F000446B8F0E436F0001A9EC06F002C003F03B
:108700000150500F0601E76F000E0320E86F100EB6
:10871000E727000EE823F2CFE5F6F29EE8C675FFE4
:10872000E7C674FF7F9C7F9E7F807350E5BFF28E0B
:10873000E76FE0C6D9F6E3C6D8F6E4C6D7F6E7C6D3
:10874000D6F6DA51C525E06FDB51C621E16FE03581
:10875000026EE135036E02360336FC0E021602503D
:108760000F0FE96E030E0320EA6EEFCFD2F6ECCFC7
:10877000D3F6ECCFD4F6ECCFD5F6D9C623F0D8C6D5
:1087800022F0D7C621F0D6C620F000018FEC15F0FC
:10879000EACFE1F6E9CFE0F6D882D5C65AF7D4C6DB
:1087A00059F7D3C658F7D2C657F703C05EF702C0D1
:1087B0005DF701C05CF700C05BF773EC10F0E1C639
:1087C000EAFFE0C6E9FF03C0D5F602C0D4F601C057
:1087D000D3F600C0D2F60601DA51C525E06FDB51B1
:1087E000C621E16FE1C642F7E0C641F70701446BDD
:1087F0008F0E436F0001A9EC06F002C003F0015098
:10880000500F0601E06F000E0320E16F0C0EE02711
:10881000000EE123030EE027000EE123F2CFE2F683
:10882000F29EE1C675FFE0C674FF7F9C7F9E7F804D
:108830007350E2BFF28EE06FDA51C525E36FDB5172
:10884000C621E46FE4C642F7E3C641F70701446B73
:108850008F0E436F0001A9EC06F002C003F0015037
:10886000500F0601E36F000E0320E46F0C0EE327A8
:10887000000EE423020EE327000EE423F2CFE1F61C
:10888000F29EE4C675FFE3C674FF7F9C7F9E7F80E7
:108890007350E1BFF28EE36FDA51C525E46FDB510F
:1088A000C621E56FE5C642F7E4C641F70701446B10
:1088B0008F0E436F0001A9EC06F002C003F00150D7
:1088C000500F0601E46F000E0320E56F0C0EE42745
:1088D000000EE523010EE427000EE523F2CFE6F6B5
:1088E000F29EE5C675FFE4C674FF7F9C7F9E7F8085
:1088F0007350E6BFF28EE46FDA51C525E76FDB51A6
:10890000C621E86FE8C642F7E7C641F70701446BA6
:108910008F0E436F0001A9EC06F002C003F0015076
:10892000500F0601E76F000E0320E86F0C0EE727DB
:10893000000EE823F2CFE5F6F29EE8C675FFE7C623
:1089400074FF7F9C7F9E7F807350E5BFF28EE76F40
:10895000E0C6D9F6E3C6D8F6E4C6D7F6E7C6D6F63B
:10896000D9C623F0D8C622F0D7C621F0D6C620F04B
:1089700000018FEC15F0D5C656F7D4C655F7D3C60F
:1089800054F7D2C653F703C05AF702C059F701C0D3
:1089900058F700C057F7E0EC13F003C0D5F602C05B
:1089A000D4F601C0D3F600C0D2F6D5C6E3F6D4C6DD
:1089B000E2F6D3C6E1F6D2C6E0F619EC3FF003C00A
:1089C000D1F602C0D0F601C0CFF600C0CEF6060147
:1089D000CC6BCD6BCB6BCB5107083AE3CA6BCA515A
:1089E000070834E3C851CC5D2EE3C951CD5D2BE2BD
:1089F000D1C603F0D0C602F0CFC601F0CEC600F05B
:108A0000CD51E06F07E0D8900332023201320032DC
:108A1000E02FF9D700B016D0036ACB51240F016EB6
:108A2000000E032201C0E9FF03C0EAFF010E006E41
:108A3000CA51016E04E0D8900036012EFCD70050D8
:108A4000FF0AEF16CD2BCC2BCA2BC9D7CB2BC3D704
:108A5000DA2BD8B4DB2B17D41FC0F6F61EC0F5F600
:108A60001DC0F4F61CC0F3F6F86B240EF76F080E69
:108A7000F96F020EFA6F010EFB6FFC6B00013AEC0E
:108A80003FF00601C52BD8B4C62BBCEF3FF0F2CFA8
:108A9000E0F6F29E020E756E8C0E746E7F9C7F9EC9
:108AA0007F807350E0BFF28EC76FC753D8B480D1B8
:108AB0003C52D8A47DD13D52D8A47AD1F2CFE0F671
:108AC000F29E020E756E9A0E746E7F9C7F9E7F8062
:108AD0007350E0BFF28EE16FE1C6E5F60001B3EC42
:108AE0003EF002C03DF001C03CF0F2CFE0F6F29E55
:108AF000020E756E990E746E7F9C7F9E7F80735000
:108B00000601E0BFF28E1F6A1E6A1D6A1C6E1C36CB
:108B10001D361E361F361C361D361E361F36FC0E01
:108B20001C16F2CFE0F6F29E020E756E960E746E73
:108B30007F9C7F9E7F807350E0BFF28E010B1C26CE
:108B4000000E1D22000E1E22000E1F221EC01FF04E
:108B50001DC01EF01CC01DF01C6AF2CFE0F6F29E94
:108B6000020E756E950E746E7F9C7F9E7F80735093
:108B7000E0BFF28E1C26000E1D22000E1E22000EEB
:108B80001F221EC01FF01DC01EF01CC01DF01C6A5D
:108B9000F2CFE0F6F29E020E756E940E746E7F9C1C
:108BA0007F9E7F807350E0BFF28E1C26000E1D2238
:108BB000000E1E22000E1F221EC01FF01DC01EF040
:108BC0001CC01DF01C6A1B501C26000E1D221E22FC
:108BD0001F22CA6BCA5107080AE3036ACA51240F4D
:108BE000E96E000E0320EA6EEF68CA2BF3D7F2CFCE
:108BF000E0F6F29E020E756E970E746E7F9C7F9E5D
:108C00007F807350E0BFF28EC86FF2CFE0F6F29E25
:108C1000020E756E980E746E7F9C7F9E7F807350DF
:108C2000E0BFF28EC96F68C154F767C153F7000106
:108C30001FEC0BF003C0D5F602C0D4F601C0D3F68A
:108C400000C0D2F6020E0701446FA00E436F000170
:108C5000B2EC15F0EACFE1F6E9CFE0F6D882D5C65E
:108C60005AF7D4C659F7D3C658F7D2C657F703C038
:108C70005EF702C05DF701C05CF700C05BF773EC04
:108C800010F0E1C6EAFFE0C6E9FF03C0D5F602C076
:108C9000D4F601C0D3F600C0D2F6020E0701446F2D
:108CA0009C0E436F0001B2EC15F0D5C656F7D4C642
:108CB00055F7D3C654F7D2C653F703C05AF702C0CC
:108CC00059F701C058F700C057F7E0EC13F003C0A4
:108CD000D5F602C0D4F601C0D3F600C0D2F6D5C690
:108CE000E3F6D4C6E2F6D3C6E1F6D2C6E0F619EC56
:108CF0003FF003C0D1F602C0D0F601C0CFF600C0ED
:108D0000CEF60601CC6BCD6BCB6BCB5107083AE3AB
:108D1000CA6BCA51070834E3C851CC5D2EE3C95170
:108D2000CD5D2BE2D1C603F0D0C602F0CFC601F074
:108D3000CEC600F0CD51E06F07E0D890033202328A
:108D400001320032E02FF9D700B016D0036ACB51C0
:108D5000240F016E000E032201C0E9FF03C0EAFFE9
:108D6000010E006ECA51016E04E0D8900036012E4B
:108D7000FCD70050FF0AEF16CD2BCC2BCA2BC9D73E
:108D8000CB2BC3D71FC0F6F61EC0F5F61DC0F4F6F8
:108D90001CC0F3F6F86B240EF76F080EF96F020E85
:108DA000FA6F010EFB6FFC6B00013AEC3FF006011D
:108DB0004052D8A4A2D14152D8A49FD10001A7EC1F
:108DC0003FF0F2CFE0F6F29E020E756EF40E746E76
:108DD0007F9C7F9E7F8073500601E0BFF28E000A69
:108DE000000103E0010A02E087D186D1F2CFE0F66C
:108DF000F29E030E756E0C0E746E7F9C7F9E7F80BC
:108E000073500601E0BFF28EE16FE1C6E5F60001A6
:108E1000B3EC3EF002C041F001C040F0F2CFE0F60A
:108E2000F29E030E756E0B0E746E7F9C7F9E7F808C
:108E300073500601E0BFF28E1F6A1E6A1D6A1C6E27
:108E40001C361D361E361F361C361D361E361F3686
:108E5000FC0E1C16F2CFE0F6F29E030E756E080EA5
:108E6000746E7F9C7F9E7F807350E0BFF28E010BFB
:108E70001C26000E1D22000E1E22000E1F221EC0E8
:108E80001FF01DC01EF01CC01DF01C6AF2CFE0F6E2
:108E9000F29E030E756E070E746E7F9C7F9E7F8020
:108EA0007350E0BFF28E1C26000E1D22000E1E2203
:108EB000000E1F221EC01FF01DC01EF01CC01DF0A2
:108EC0001C6AF2CFE0F6F29E030E756E060E746E0B
:108ED0007F9C7F9E7F807350E0BFF28E1C26000E29
:108EE0001D22000E1E22000E1F221EC01FF01DC0DC
:108EF0001EF01CC01DF01C6A1B501C26000E1D22FB
:108F00001E221F22F2CFE0F6F29E030E756E090EAE
:108F1000746E7F9C7F9E7F807350E0BFF28EC86F1F
:108F2000F2CFE0F6F29E030E756E0A0E746E7F9C11
:108F30007F9E7F807350E0BFF28EC96F04C354F7E9
:108F400003C353F700011FEC0BF003C0D5F602C0BA
:108F5000D4F601C0D3F600C0D2F6D5C656F7D4C6B3
:108F600055F7D3C654F7D2C653F707015A6B596B5E
:108F70007A0E586F880E576F0001E0EC13F003C0B3
:108F8000D5F602C0D4F601C0D3F600C0D2F6030E67
:108F90000701446F0D0E436F0001B2EC15F0EACFEC
:108FA000E1F6E9CFE0F6D882D5C65AF7D4C659F72C
:108FB000D3C658F7D2C657F703C05EF702C05DF7B5
:108FC00001C05CF700C05BF773EC10F0E1C6EAFF8C
:108FD000E0C6E9FF03C0D5F602C0D4F601C0D3F65F
:108FE00000C0D2F6030E0701446F110E436F00015B
:108FF000B2EC15F0D5C656F7D4C655F7D3C654F71C
:10900000D2C653F703C05AF702C059F701C058F748
:1090100000C057F7E0EC13F003C0D5F602C0D4F659
:1090200001C0D3F600C0D2F6D5C6E3F6D4C6E2F648
:10903000D3C6E1F6D2C6E0F619EC3FF003C0D1F694
:1090400002C0D0F601C0CFF600C0CEF60601CC6B50
:10905000CD6BCB6BCB5107083AE3CA6BCA510708FB
:1090600034E3C851CC5D2EE3C951CD5D2BE2D1C6AE
:1090700003F0D0C602F0CFC601F0CEC600F0CD514D
:10908000E06F07E0D8900332023201320032E02F65
:10909000F9D700B016D0036ACB51240F016E000E31
:1090A000032201C0E9FF03C0EAFF010E006ECA51AE
:1090B000016E04E0D8900036012EFCD70050FF0A64
:1090C000EF16CD2BCC2BCA2BC9D7CB2BC3D71FC0A8
:1090D000F6F61EC0F5F61DC0F4F61CC0F3F6F86BEC
:1090E000240EF76F080EF96F020EFA6F010EFB6F78
:1090F000FC6B00013AEC3FF00601425256E143524C
:1091000054E1436A640E426EF2CFE0F6F29E030E23
:10911000756E1C0E746E7F9C7F9E7F807350E0BFC7
:10912000F28E000A42E00001A7EC3FF01BC01CF0E9
:10913000E50E1D6EFE0E1E6E180E1F6E0601CA6B2A
:10914000CA5103081CE3036ACA51240F016E000EC2
:10915000032201C0E0F603C0E1F6010ECA25036A4E
:10916000940FE96E060E0320EA6EEFCFE2F6E1C639
:10917000EAFF01C0E9FFE2C6EFFFCA2BE1D71FC03B
:10918000F6F61EC0F5F61DC0F4F61CC0F3F6F86B3B
:10919000240EF76F080EF96F020EFA6F010EFB6FC7
:1091A000FC6B00013AEC3FF00601000158EF61F062
:1091B0000601D291D16BD151070829E3D151040D99
:1091C000F350036A340FE96E010E0320EA6EEFCF0D
:1091D000D3F6ECCFD4F6ECCFD5F6ECCFD6F6CC5117
:1091E000D35D13E1CD51D45D10E1CE51D55D0DE1DC
:1091F000CF51D65D0AE1D281036AD151540FE96E95
:10920000010E0320EA6ED0C6EFFFD12BD4D7D2B126
:1092100039D0D16BD151040DF350036A340FE96E8C
:10922000010E0320EA6EEFCFD3F6ECCFD4F6ECCFED
:10923000D5F6ECCFD6F6D35307E1D45305E1D55399
:1092400003E1D65301E104D0D12BD1510708E2E26A
:10925000D151040DF350036A340FE96E010E03205F
:10926000EA6ECCC6EFFFCDC6ECFFCEC6ECFFCFC694
:10927000ECFF036AD151540FE96E010E0320EA6E30
:10928000D0C6EFFF000112000601CF6BCF51040DD5
:10929000F350036A340FE96E010E0320EA6EEFCF3C
:1092A000D0F6ECCFD1F6ECCFD2F6ECCFD3F6CB5153
:1092B000D05D1EE1CC51D15D1BE1CD51D25D18E1F5
:1092C000CE51D35D15E1CF51040DF350036A340F35
:1092D000E96E010E0320EA6EEF6AEC6AEC6AEC6A52
:1092E000036ACF51540FE96E010E0320EA6EEF6856
:1092F000CF2BCF510708CAE2000112000601C66B4E
:10930000C56BC653D8A4BFD0C5510308D8A0BBD0E5
:10931000C5C6F3F6030EF56F230EF46F0001A2EC41
:1093200013F00150010B0108D8A4A8D0C6C642F71B
:10933000C5C641F70701446B8F0E436F0001A9ECCE
:1093400006F002C003F00150500F0601CB6F000E73
:109350000320CC6F010ECB27000ECC23020ECB27AF
:10936000000ECC23F2CFCDF6F29ECCC675FFCBC655
:1093700074FF7F9C7F9E7F807350CDBFF28ECB6F3A
:10938000C6C642F7C5C641F70701446B8F0E436F4F
:109390000001A9EC06F002C003F00150500F0601D5
:1093A000CE6F000E0320CF6F010ECE27000ECF230D
:1093B000010ECE27000ECF23F2CFCCF6F29ECFC601
:1093C00075FFCEC674FF7F9C7F9E7F807350CCBF9D
:1093D000F28ECE6FC6C642F7C5C641F70701446B91
:1093E0008F0E436F0001A9EC06F002C003F001509C
:1093F000500F0601CF6F000E0320D06F010ECF2754
:10940000000ED023F2CFD1F6F29ED0C675FFCFC6A4
:1094100074FF7F9C7F9E7F807350D1BFF28ECF6F91
:10942000CA6BCBC6C9F6CEC6C8F6CFC6C7F61F0EE6
:10943000C525E96E030EC621EA6EEF3C01D014D0BB
:109440001F0EC525E96E030EC621EA6EEFCFD0F6DA
:10945000CAC6CFF6C9C6CEF6C8C6CDF6C7C6CCF6C4
:109460000001A6DE0BD00601CAC6CEF6C9C6CDF6EF
:10947000C8C6CCF6C7C6CBF6000106DF0601C52B71
:10948000D8B4C62B3ED7F2CFCBF6F29E020E756E45
:10949000930E746E7F9C7F9E7F807350CBBFF28E45
:1094A000CC6FF2CFCDF6F29E020E756E920E746EF8
:1094B0007F9C7F9E7F807350CDBFF28ECE6FF2CFA8
:1094C000CFF6F29E020E756E910E746E7F9C7F9E9B
:1094D0007F807350CFBFF28ED06FCA6BCCC6C9F6F7
:1094E000CEC6C8F6D0C6C7F601016E3D01D00ED07B
:1094F000CAC6CFF6C9C6CEF6C8C6CDF6C7C6CCF624
:109500006EC1D0F6000154DE0BD00101CAC6CEF602
:10951000C9C6CDF6C8C6CCF6C7C6CBF60001B4DEC8
:10952000F2CFCBF6F29E020E756EF40E746E7F9C37
:109530007F9E7F8073500601CBBFF28E000A000130
:1095400003E0010A08E03AD00601CA6BC96BC86B98
:10955000C76B000133D0F2CFCBF6F29E030E756ECF
:10956000050E746E7F9C7F9E7F8073500601CBBF7B
:10957000F28ECC6FF2CFCDF6F29E030E756E040E16
:10958000746E7F9C7F9E7F807350CDBFF28ECE6FB6
:10959000F2CFCFF6F29E030E756E030E746E7F9CB3
:1095A0007F9E7F807350CFBFF28ED06FCA6BCCC6C8
:1095B000C9F6CEC6C8F6D0C6C7F6000106018F3D73
:1095C00001D00ED0CAC6CFF6C9C6CEF6C8C6CDF6F3
:1095D000C7C6CCF68FC6D0F60001EADD0BD0060177
:1095E000CAC6CEF6C9C6CDF6C8C6CCF6C7C6CBF637
:1095F00000014ADE61EF61F00601C56B0001A7ECD6
:109600003FF00601C66BC65107081CE3C651040DA6
:10961000F350036A340FE96E010E0320EA6EEFCFB8
:10962000EFF6ECCFF0F6ECCFF1F6ECCFF2F6EF532D
:1096300006E1F05304E1F15302E1F25301E0C52BDE
:10964000C62BE1D7C52D92D0C66BC6510708D8A04E
:109650008CD0C651040DF350036A340FE96E010E2D
:109660000320EA6EEFCFEFF6ECCFF0F6ECCFF1F699
:10967000ECCFF2F6EF5306E1F05304E1F15302E1CF
:10968000F25371E0036AC651540FE96E010E0320D4
:10969000EA6EEF50010803E2C70E246E02D0D30E2B
:1096A000246EC651040DF350036A340FE96E010EA7
:1096B0000320EA6EEFCF26F0ECCFF0F6ECCFF1F618
:1096C000ECCFF2F6C651040DF350036A340FE96E85
:1096D000010E0320EA6EEFCFEFF6ECCF27F0ECCFD0
:1096E000F1F6ECCFF2F6C651040DF350036A340FD5
:1096F000E96E010E0320EA6EEFCFEFF6ECCFF0F645
:10970000ECCFF1F6ECCFF2F6F151070B200DF3CFD1
:1097100028F0036AC651540FE96E010E0320EA6E69
:10972000EF501F0B28267F0E296E1BC0EFF6CA0EC6
:10973000F06FFE0EF16F180EF26FF66FF1C6F5F6D0
:10974000F0C6F4F61BC0F3F6F86B240EF76F080EA4
:10975000F96F020EFA6F010EFB6FFC6B00013AEC21
:109760003FF0060102D0C62B70D765D1C553D8B4DF
:1097700062D1C30ECB6FCC69CA6B020EC96FC66BC8
:10978000C6510708D8A0C9D0C651040DF350036ACA
:10979000340FE96E010E0320EA6EEFCFEFF6ECCF47
:1097A000F0F6ECCFF1F6ECCFF2F6EF5307E1F05321
:1097B00005E1F15303E1F253D8B4ADD0CAC603F0CA
:1097C000C951C92BD8B4CA2BEF6F03C0F0F6CB0E2A
:1097D000EF25016E060E0320036EF26FC651040DD5
:1097E000F350036A340FE96E010E0320EA6EEFCFE7
:1097F000F3F6ECCFF4F6ECCFF5F6ECCFF6F6F2C6D6
:10980000EAFF01C0E9FFF3C6EFFFCAC6F0F6C9518F
:10981000C92BD8B4CA2BEF6FCB0EEF25016E060E05
:10982000F021036EF26FC651040DF350036A340F3A
:10983000E96E010E0320EA6EEFCFF3F6ECCFF4F6FB
:10984000ECCFF5F6ECCFF6F6F2C6EAFF01C0E9FF81
:10985000F4C6EFFFCB0EC925016E060ECA21036EBA
:10986000F06FC651040DF350036A340FE96E010E18
:109870000320EA6EEFCFF1F6ECCFF2F6ECCFF3F681
:10988000ECCFF4F6F351070B200DF3CFF5F6F0C64D
:10989000EAFF01C0E9FFF5C6EFFFCAC6F0F6C951FD
:1098A000C92BD8B4CA2BEF6FCB0EEF25016E060E75
:1098B000F021036EF26FEA6E01C0E9FFEFCFF3F61D
:1098C000036AC651540FE96E010E0320EA6EEF5091
:1098D0001F0BF325F2C6EAFF01C0E9FFEF6E036A32
:1098E000C651540FE96E010E0320EA6EEF500108D5
:1098F00002E3CB8901D0CB85CAC603F0C951C92B7D
:10990000D8B4CA2BEF6FCB0EEF25E96E060E0320FD
:10991000EA6E7F0EEF6EC62B33D7010EC95DEF6F77
:10992000000ECA59F06FF26FEFC6F1F6F46B070E36
:10993000F36F0001FCEC0AF0010E06010124C86F70
:10994000200E246EC9C625F0CAC626F0C8C627F068
:109950002868CA0E296EFE0E2A6E2B6A1BC0EFF60F
:10996000FF0EF06FEC0EF16F180EF26FF66FF1C68E
:10997000F5F6F0C6F4F61BC0F3F6F86B240EF76F9D
:10998000080EF96F020EFA6F010EFB6FFC6B0001FF
:109990003AEC3FF00601EE6BED6B0001A7EC3FF0F7
:1099A000010E0601C66FC651C85D45E3C6C624F068
:1099B000010EC76FC75107081FE3036AC751240F81
:1099C000016E000E032203C0F0F6EEC603F0ED5167
:1099D000ED2BD8B4EE2BF16FCB0EF125E96E060E10
:1099E0000320EA6EEFCFF3F6F0C6EAFF01C0E9FF0D
:1099F000F3C6EFFFC72BDED71BC0EFF6FF0EF06FED
:109A0000EB0EF16F180EF26FF66FF1C6F5F6F0C6B9
:109A1000F4F61BC0F3F6F86B240EF76F080EF96F1F
:109A2000020EFA6F010EFB6FFC6B00013AEC3FF087
:109A30000601C62BB8D7000163EF61F00601A05301
:109A4000D8A41FD20A0EA06FA151FB0FD8B014D218
:109A5000050F000144EF4FF0010165C124F066C11C
:109A600025F004C3F2F603C3F1F60601F46B0A0E07
:109A7000F36F0001FCEC0AF0060101C026F004C3FC
:109A8000F2F603C3F1F6F46B0A0EF36F0001FCEC7F
:109A90000AF0060102C027F0180EF66FF569FE0EF7
:109AA000F46FF36BF86B240EF76F040EF96F020E70
:109AB000FA6F010EFB6FFC6B00013AEC3FF0060100
:109AC000DBD10601C56BC55103084CE3D890C53501
:109AD000036AE20FE96E020E0320EA6EECCF46F74E
:109AE000ED52EFCF45F70701446BC5C643F70001C0
:109AF00010EC16F003C0C9F602C0C8F601C0C7F6E4
:109B000000C0C6F6D8900601C535036A240FE96E79
:109B1000000E0320EA6EC9C6F1F6C8C6F0F6C7C645
:109B2000EFF6C6C6EEF600012AEC12F0060101C0FF
:109B3000EFFFD890C535010F036A240FE96E000EC0
:109B40000320EA6EC9C6F1F6C8C6F0F6C7C6EFF63E
:109B5000C6C6EEF600012AEC12F0060102C0EFFFC5
:109B6000C52BB1D7180EF66FF569FD0EF46FF36BC8
:109B7000F86B240EF76F080EF96F020EFA6F010EE4
:109B8000FB6FFC6B00013AEC3FF0060175D106015A
:109B9000C56BC551030862E3D890C535036AE20F6F
:109BA000E96E020E0320EA6EECCF44F7ED52EFCFE0
:109BB00043F7000150EC17F003C0C9F602C0C8F625
:109BC00001C0C7F600C0C6F6C9C656F7C8C655F7E5
:109BD000C7C654F7C6C653F707015A6B596B480EF0
:109BE000586F850E576F0001AFEC11F003C0C9F636
:109BF00002C0C8F601C0C7F600C0C6F6D89006017C
:109C0000C535036A240FE96E000E0320EA6EC9C64B
:109C1000F1F6C8C6F0F6C7C6EFF6C6C6EEF6000106
:109C20002AEC12F0060101C0EFFFD890C535010FF4
:109C3000036A240FE96E000E0320EA6EC9C6F1F62E
:109C4000C8C6F0F6C7C6EFF6C6C6EEF600012AECA7
:109C500012F0060102C0EFFFC52B9BD7180EF66F5E
:109C6000F569FC0EF46FF36BF86B240EF76F080EBA
:109C7000F96F020EFA6F010EFB6FFC6B00013AECFC
:109C80003FF00601F9D00601C56BC551030862E338
:109C9000D890C535036AE20FE96E020E0320EA6E22
:109CA000ECCF44F7ED52EFCF43F700019BEC17F0F8
:109CB00003C0C9F602C0C8F601C0C7F600C0C6F6A8
:109CC000C9C656F7C8C655F7C7C654F7C6C653F730
:109CD00007015A6B596B480E586F850E576F00017C
:109CE000AFEC11F003C0C9F602C0C8F601C0C7F658
:109CF00000C0C6F6D8900601C535036A240FE96E88
:109D0000000E0320EA6EC9C6F1F6C8C6F0F6C7C653
:109D1000EFF6C6C6EEF600012AEC12F0060101C00D
:109D2000EFFFD890C535010F036A240FE96E000ECE
:109D30000320EA6EC9C6F1F6C8C6F0F6C7C6EFF64C
:109D4000C6C6EEF600012AEC12F0060102C0EFFFD3
:109D5000C52B9BD7180EF66FF569FB0EF46FF36BEE
:109D6000F86B240EF76F080EF96F020EFA6F010EF2
:109D7000FB6FFC6B00013AEC3FF006017DD0060161
:109D8000C56BC551030862E3D890C535036AE20F7D
:109D9000E96E020E0320EA6EECCF44F7ED52EFCFEE
:109DA00043F7000102EC18F003C0C9F602C0C8F680
:109DB00001C0C7F600C0C6F6C9C656F7C8C655F7F3
:109DC000C7C654F7C6C653F707015A6B596B480EFE
:109DD000586F850E576F0001AFEC11F003C0C9F644
:109DE00002C0C8F601C0C7F600C0C6F6D89006018A
:109DF000C535036A240FE96E000E0320EA6EC9C65A
:109E0000F1F6C8C6F0F6C7C6EFF6C6C6EEF6000114
:109E10002AEC12F0060101C0EFFFD890C535010F02
:109E2000036A240FE96E000E0320EA6EC9C6F1F63C
:109E3000C8C6F0F6C7C6EFF6C6C6EEF600012AECB5
:109E400012F0060102C0EFFFC52B9BD7180EF66F6C
:109E5000F569FA0EF46FF36BF86B240EF76F080ECA
:109E6000F96F020EFA6F010EFB6FFC6B00013AEC0A
:109E70003FF0060101D00601A12BA151040801E227
:109E8000A16B000168EF61F0E824F76AF736A30FD1
:109E9000F66E9E0EF7220A00F550FA6E0800F55095
:109EA000F96E869C8E9B7E9DC29A589A0F0E060173
:109EB000F66F660EF56F0F0120B70FD00601A353A2
:109EC00005E1F10E6F1408096F6E04D0E00E7214F4
:109ED0000309726EF76B77D00F0110B710D006012F
:109EE000A35305E1F10E6F1406096F6E04D0E00E66
:109EF00072140409726E010EF76F65D00F0100B77E
:109F00000FD00601A35305E1F10E6F1404096F6E23
:109F100004D0E00E72140509726E020EF76F53D072
:109F20000E0180B70BD07DA509D0E00E7214120986
:109F3000726E030E0601F76F46D00E0190B70BD07C
:109F40007DA709D0E00E72141309726E040E06018B
:109F5000F76F39D00E01A0B70BD07DA909D0E00E64
:109F600072141409726E050E0601F76F2CD00E01E3
:109F7000B0B70BD07DAB09D0E00E72141509726E2C
:109F8000060E0601F76F1FD00E01C0B70BD07DADD6
:109F900009D0E00E72141609726E070E0601F76FF3
:109FA00012D00E01D0B70BD07DAF09D0E00E7214E5
:109FB0001709726E080E0601F76F05D00E01000E2C
:109FC000016E49D00601F151030B006EFC0E6014C6
:109FD0000010606E0F0EF96F640EF86FEDC6FDF69F
:109FE000ECC6FCF6EBC6FBF6EAC6FAF6F2C6FEF6DF
:109FF0000001FEEC0BF0F0C665FF659C0601F3B1B5
:10A00000658CF46BF051F45D18E2F6C6F9F6EFC614
:10A0100003F0EEC6E9FF03C0EAFFEFCFFAF6F9C698
:10A02000EAFFF5C6E9FFFAC6EFFFF52BD8B4F62B29
:10A03000EE2BD8B4EF2BF42BE5D76086A35304E1C5
:10A04000F10E6F146F6E04D0E00E72141009726E70
:10A05000010E016E0E01000112004E504F5CD8B48B
:10A06000C2D00F0120A72CD010A72AD000A728D03B
:10A070000E0180B704D07DA502D00F0121D090B78A
:10A0800004D07DA702D00F011BD0A0B704D07DA9BA
:10A0900002D00F0115D0B0B704D07DAB02D00F01B4
:10A0A0000FD0C0B704D07DAD02D00F0109D0D0A72A
:10A0B00002D0000198D07DBF02D0000194D00F01E2
:10A0C0000601C56BC551070825E3036AC551240F76
:10A0D000016E000E032201C0C6F603C0C7F64F5042
:10A0E000080DF350C96BC86F036AC551C825016ECE
:10A0F000C95103220150900FE96E000E0320EA6E51
:10A10000EFCFC8F6C7C6EAFFC6C6E9FFC8C6EFFF6D
:10A11000C52BD8D74F50040DF350036A500FE96E8A
:10A12000000E0320EA6EEFCFC6F6ECCFC7F6ECCFF9
:10A13000C8F6ECCFC9F6036A4F50100FE96E010E56
:10A140000320EA6EEFCFCAF6036A4F50200FE96E84
:10A15000010E0320EA6EEFCFCBF6EACFCDF6E9CFC2
:10A16000CCF64FC0F3F6010EF56F300EF46F000120
:10A17000A2EC13F0CDC6EAFFCCC6E9FF000E01B099
:10A18000010E0601CE6FEACFD0F6E9CFCFF64FC071
:10A19000F3F6010EF56F320EF46F0001A2EC13F02E
:10A1A000D0C6EAFFCFC6E9FF000E01B0010E0601DE
:10A1B000D16FC9C6EDF6C8C6ECF6C7C6EBF6C6C683
:10A1C000EAF6EF6B240EEE6FCAC6F0F6CBC6F1F6D8
:10A1D000CEC6F2F6D1C6F3F6000168DE4F2A4F5024
:10A1E0000F0801E24F6A6CEF61F0D8B204D0060E9E
:10A1F000EA6EFA0EE96E006A016A026A036A0601F3
:10A20000FA6BFB6BFC6BFD6BF951F811F711F61152
:10A210002CE0200EFE6FD890F237F337F437F53785
:10A22000FA37FB37FC37FD37F951FD5D08E1F8518E
:10A23000FC5D05E1F751FB5D02E1F651FA5D0FE3CC
:10A24000F651FA5FF751D8A0F73DFB5FF851D8A05F
:10A25000F83DFC5FF951D8A0F93DFD5FD88000368C
:10A26000013602360336FE2FD6D7FAC6EFFFFBC6FD
:10A27000ECFFFCC6ECFFFDC6ECFF00011200A5C61A
:10A28000EAFFA4C6E9FF0601F2C6EFFFE92AD8B447
:10A29000EA2AEF6AA42BD8B4A52B000191EF51F064
:10A2A000E9500601EA6F3B0EF16F9A0EF06FCA0E8D
:10A2B000EF6FEE6B0A0EEC6FD882060EEA6EE60EBA
:10A2C000E96EE9C6F5F6E8C6F4F6E7C6F3F6E6C6C3
:10A2D000F2F6F1C6F9F6F0C6F8F6EFC6F7F6EEC6F6
:10A2E000F6F6000182DF0150005213E10601EC5145
:10A2F000010AD8A402D000010CD0EA510CE00F0BE7
:10A30000EC5D01E00FE2EABF0DD0EABD04D0200E03
:10A3100003D00601EA6B300E002600C0F2F6000101
:10A32000AED70601D892F1C6F5F6F0C6F4F6EFC640
:10A33000F3F6EEC6F2F6F96BF86BF76B0A0EF66FF2
:10A34000000153DF03C0F1F602C0F0F601C0EFF6E2
:10A3500000C0EEF60601EC2FAFD700017CEF52F003
:10A36000EAC601F0E9C600F00066012A0900F5CF4F
:10A37000EEFF002EFBD7012EF9D7F86A1200060E69
:10A38000EA6EE60EE96EEF5011E0140E016EBF0E9C
:10A39000006E0400002EFDD7012EF9D7BF0E006E0F
:10A3A000002EFED700000400EF2EEFD723EF55F06C
:10A3B000010E0601E75F0EE3060EEA6EE70EE96E98
:10A3C000EF5008E0030E006E002EFED700D0040010
:10A3D000EF2EF8D700012AEF55F00601D16BD06BB4
:10A3E000E16B010EC625E66F000EC721E76FF26F25
:10A3F000E6C6F1F6F46B070EF36F0001FCEC0AF011
:10A40000010E06010124CF6F200E246EC6C625F072
:10A41000C7C626F0CFC627F02868C8C629F0C9C627
:10A420002AF02B6A180EE96FEC0EE86FCAC6E7F641
:10A430001BC0E6F6E9C6EDF6EC6FCAC6EBF61BC02C
:10A44000EAF6EF6B240EEE6F080EF06F030EF16F5D
:10A45000010EF26FF36B000129DD0601C55374E1B3
:10A46000F2CFE6F6F29E756A140E746E7F9C7F9EA4
:10A470007F807350E6BFF28EE76FF2CFE8F6F29E70
:10A48000756A130E746E7F9C7F9E7F807350E8BF49
:10A49000F28EE96FF2CFEAF6F29E756A120E746ED2
:10A4A0007F9C7F9E7F807350EABFF28EEB6FF2CF6E
:10A4B000ECF6F29E756A110E746E7F9C7F9E7F8013
:10A4C0007350ECBFF28EED6FE7C6E0F6E9C6DFF63B
:10A4D000EBC6DEF6EDC6DDF6060EA56FD20EA46F56
:10A4E000410EE96EE0C6E9F6DFC6E8F6DEC6E7F63D
:10A4F000DDC6E6F60001D4D6F86A0B0EF76EFA0E4A
:10A50000F66E060EEA6EE20EE96E0601EA6B040EC6
:10A51000E96F000125DF0601CB6BCB51030814E383
:10A52000036ACB51E20FE96E060E0320EA6EEF3CA0
:10A5300009D0036ACB51E20FE96E060E0320EA6EE2
:10A540003F0EEF6ECB2BE9D7CB6BCF51CB5DD8B0A5
:10A5500086D2010ECB25246ECC6BCC510608D8A038
:10A5600050D2C551000A000107E0010AD8B4FED15B
:10A57000030AD8B428D242D20601D05310E1D153F5
:10A580000EE1010ECC25036A240FE96E000E0320B4
:10A59000EA6E070EEF6ED02BD8B4D12BE5D1D15394
:10A5A00034E1D0510F0831E3CE69EE0ECD6F010ECC
:10A5B000D05D006E000ED159036E0050CD270350C0
:10A5C000CE23010ECC25036A240F016E000E032258
:10A5D0000150E66F03C0E7F6F86ACEC6F7FFCDC6B6
:10A5E000F6FF060EEA6EE80EE96EEA6B010EE96F01
:10A5F0000001B6DEE7C6EAFFE6C6E9FFE8C6EFFF00
:10A600000601D02BD8B4D12BAFD1D051100810E116
:10A61000D1530EE1010ECC25036A240FE96E000E22
:10A620000320EA6E2A0EEF6ED02BD8B4D12B9CD12A
:10A63000D1533AE1D0512A0837E3CE69D20ECD6F1B
:10A64000100ED05DE66F000ED159E76F010EE65D8A
:10A65000006E000EE759036E0050CD270350CE2345
:10A66000010ECC25036A240F016E000E0322015057
:10A67000E66F03C0E7F6F86ACEC6F7FFCDC6F6FF71
:10A68000060EEA6EE80EE96EEA6B010EE96F000154
:10A6900067DEE7C6EAFFE6C6E9FFE8C6EFFF0601A8
:10A6A000D02BD8B4D12B60D1D0512B0810E1D1538D
:10A6B0000EE1010ECC25036A240FE96E000E032083
:10A6C000EA6E2A0EEF6ED02BD8B4D12B4DD1D153D8
:10A6D00033E1D0514B0830E3010ECC25036A240F3F
:10A6E000E96E000E0320EA6E100ED05DE86F000EDA
:10A6F000D159E96F1B0EE85F000EE95B010EE85DC2
:10A70000006E000EE959036E00501F0FE86F000E37
:10A710000320E96FF2CFEAF6F29EE9C675FFE8C6BC
:10A7200074FF7F9C7F9E7F807350EABFF28EEF6E36
:10A73000D02BD8B4D12B18D1D0514C0810E1D15323
:10A740000EE1010ECC25036A240FE96E000E0320F2
:10A75000EA6E2A0EEF6ED02BD8B4D12B05D1D1538F
:10A7600037E1D051560834E3010ECC25036A240F9B
:10A77000E96E000E0320EA6E100ED05DE86F000E49
:10A78000D159E96F1B0EE85F000EE95B210EE85F0F
:10A79000000EE95B010EE85D006E000EE959036EE4
:10A7A0000050150FE86F000E0320E96FF2CFEAF6B4
:10A7B000F29EE9C675FFE8C674FF7F9C7F9E7F808E
:10A7C0007350EABFF28EEF6ED02BD8B4D12BCCD021
:10A7D000D051570810E1D1530EE1010ECC25036A88
:10A7E000240FE96E000E0320EA6E2A0EEF6ED02BC6
:10A7F000D8B4D12BB9D0D15320E1D05161081DE399
:10A80000010ECC25036A240F016E000E032203C043
:10A81000E7F6E151E12B036AD20FE96E060E032041
:10A82000EA6EEFCFE8F6E7C6EAFF01C0E9FFE8C647
:10A83000EFFFD02BD8B4D12B97D0D051620811E1C3
:10A84000D1530FE1010ECC25036A240FE96E000EEF
:10A850000320EA6E2A0EEF6ED02BD8B4D12BE16B19
:10A8600083D0D1533FE1D05164083CE3010ECC25A5
:10A87000036A240FE96E000E0320EA6E100ED05D0D
:10A88000E86F000ED159E96F1B0EE85F000EE95B1F
:10A89000210EE85F000EE95B0B0EE85F000EE95B3E
:10A8A0000B0EE85F000EE95B010EE85D006E000E26
:10A8B000E959036E0050470FE86F000E0320E96F5F
:10A8C000F2CFEAF6F29EE9C675FFE8C674FF7F9CF8
:10A8D0007F9E7F807350EABFF28EEF6ED02BD8B48C
:10A8E000D12B42D0D051650810E1D1530EE1010EB9
:10A8F000CC25036A240FE96E000E0320EA6E2A0EAF
:10A90000EF6ED02BD8B4D12B2FD0D15320E1D05122
:10A9100069081DE3010ECC25036A240F016E000EA9
:10A92000032203C0E7F6E151E12B036AE20FE96E6F
:10A93000060E0320EA6EEFCFE8F6E7C6EAFF01C095
:10A94000E9FFE8C6EFFFD02BD8B4D12B0DD0010E14
:10A95000CC25036A240FE96E000E0320EA6E2A0E4E
:10A96000EF6ED02BD8B4D12B000148D00601CE69B0
:10A97000BC0ECD6FD051CD27D151CE23010ECC25A9
:10A98000036A240F016E000E03220150E66F03C01C
:10A99000E7F6F86ACEC6F7FFCDC6F6FF060EEA6EFA
:10A9A000E80EE96EEA6B010EE96F0001D9DCE7C63B
:10A9B000EAFFE6C6E9FFE8C6EFFF0601D02BD8B4F0
:10A9C000D12B00011BD0010E0601CC25036A240FF8
:10A9D000E96E000E0320EA6EF2CFE8F6F29ED1C6D1
:10A9E00075FFD0C674FF7F9C7F9E7F807350E8BF49
:10A9F000F28EEF6ED02BD8B4D12B00010601CC2BF8
:10AA0000ACD5180EE96FEB0EE86FCAC6E7F61BC0AF
:10AA1000E6F6E9C6EDF6EC6FCAC6EBF61BC0EAF641
:10AA2000EF6B240EEE6F080EF06F030EF16F010E48
:10AA3000F26FF36B000156EC4FF00400010E0601BB
:10AA4000E66F00019CD4020E0601E66FF90EE76F77
:10AA50000001AED40601E62FF9D7CB2B76D5000145
:10AA600012008B0E246EE00E256EB00E266E040EC4
:10AA7000276E0601C76BC751030833E3C669D20EC0
:10AA8000C56FC751010806E3020EC725C527000E92
:10AA9000C62305D0030EC725C527000EC623040E06
:10AAA000C725036A240F016E000E03220150C86FF0
:10AAB00003C0C9F6F86AC6C6F7FFC5C6F6FF060E9C
:10AAC000EA6ECA0EE96EEA6B010EE96F000148DC1E
:10AAD000C9C6EAFFC8C6E9FFCAC6EFFF0601C72B11
:10AAE000CAD71BC0C8F6F20EC96FFF0ECA6F180E88
:10AAF000CB6FED6FCAC6ECF6C9C6EBF61BC0EAF623
:10AB0000EF6B240EEE6F080EF06F020EF16F010E68
:10AB1000F26FF36B000156EC4FF0A2EF61F0110EF3
:10AB2000246E25682CC326F027682868030128C3F3
:10AB300029F029C32AF02AC32BF0180E0601C86F8A
:10AB4000EC0EC76F24C3EBF61BC0C5F6C8C6EDF606
:10AB5000EC6F1BC0EAF6EF6B240EEE6F080EF06F81
:10AB6000030EF16F010EF26FF36B000156EC4FF024
:10AB7000DEEF61F00601C52D02D0246A02D0010E7D
:10AB8000246EC6C625F0266827682868030128C3F6
:10AB900029F029C32AF02AC32BF0180E0601CA6F28
:10ABA000E80EC96F24C3EBF61BC0C7F6CAC6EDF6A4
:10ABB000EC6F1BC0EAF6EF6B240EEE6F080EF06F21
:10ABC000030EF16F010EF26FF36B000156EC4FF0C4
:10ABD00012000601CA6BC96BC535026EC635036E1D
:10ABE00002360336023603360236033602360336A1
:10ABF000E00E02160250B40FEE6F020E0320EF6F4C
:10AC0000F2CFF0F6F29EEFC675FFEEC674FF7F9CA2
:10AC10007F9E7F807350F0BFF28EC76FC535026E86
:10AC2000C635036E02360336023603360236033665
:10AC300002360336E00E02160250B40FEE6F020E1B
:10AC40000320EF6F010EEE27000EEF23F2CFF0F698
:10AC5000F29EEFC675FFEEC674FF7F9C7F9E7F80DD
:10AC60007350F0BFF28EC86FC751000A00010BE0AD
:10AC7000010A35E0030A52E0010A5AE0070AD8B493
:10AC800004D374EF5AF00601CB6BCB51030819E3E0
:10AC9000036ACB511F0FE96E030E0320EA6EEF50DB
:10ACA00001080DE2036ACB511F0FE96E030E03206A
:10ACB000EA6EEF3C01D003D0030ECA6FC969CB2BFB
:10ACC000E4D701016E51010808E26E3D01D005D0C4
:10ACD000030E0601CA6FC969010178EF5AF0060137
:10ACE000CB6BCB5103080FE3036ACB511F0FE96E07
:10ACF000030E0320EA6EEF50010803E3030ECA6F50
:10AD0000C969CB2BEED701016E51010805E3030E93
:10AD10000601CA6FC969010178EF5AF019A405D07C
:10AD2000030E0601CA6FC9690001010178EF5AF0EC
:10AD3000C5C6F3F6060E0601F56F860EF46F000128
:10AD4000A2EC13F00150010B0108D8A499D206011E
:10AD5000C535026EC635036E02360336023603363B
:10AD60000236033602360336E00E02160250B40FE6
:10AD7000EE6F020E0320EF6F070EEE27000EEF239B
:10AD8000EFC644F7EEC643F70001B2EC15F003C07E
:10AD9000CFF602C0CEF601C0CDF600C0CCF606015B
:10ADA000C535026EC635036E0236033602360336EB
:10ADB0000236033602360336E00E02160250B40F96
:10ADC000EE6F020E0320EF6F0B0EEE27000EEF2347
:10ADD000EFC644F7EEC643F70001B2EC15F003C02E
:10ADE000D3F602C0D2F601C0D1F600C0D0F60601FB
:10ADF000C535026EC635036E02360336023603369B
:10AE00000236033602360336E00E02160250B40F45
:10AE1000EE6F020E0320EF6F060EEE27000EEF23FB
:10AE2000F2CFF0F6F29EEFC675FFEEC674FF7F9C80
:10AE30007F9E7F807350F0BFF28EE36FC535026E48
:10AE4000C635036E02360336023603360236033643
:10AE500002360336E00E02160250B40FEE6F020EF9
:10AE60000320EF6F050EEE27000EEF23F2CFF0F672
:10AE7000F29EEFC675FFEEC674FF7F9C7F9E7F80BB
:10AE80007350F0BFF28EE46FC535026EC635036EA7
:10AE900002360336023603360236033602360336EE
:10AEA000E00E02160250B40FEE6F020E0320EF6F99
:10AEB0000F0EEE27000EEF23F2CFF0F6F29EEFC654
:10AEC00075FFEEC674FF7F9C7F9E7F807350F0BF3E
:10AED000F28EE56FC535026EC635036E0236033657
:10AEE000023603360236033602360336E00E021609
:10AEF0000250B40FEE6F020E0320EF6F100EEE271C
:10AF0000000EEF23EFC644F7EEC643F70001B2ECA4
:10AF100015F003C0D7F602C0D6F601C0D5F600C0C2
:10AF2000D4F60601C535026EC635036E0236033609
:10AF3000023603360236033602360336E00E0216B8
:10AF40000250B40FEE6F020E0320EF6F140EEE27C7
:10AF5000000EEF23EFC644F7EEC643F70001B2EC54
:10AF600015F003C0DBF602C0DAF601C0D9F600C066
:10AF7000D8F60601DF6BDE6BDD6BDC6BE16BE26B41
:10AF8000DF6BDE6BDD6BDC6BE06BE051070848E3E9
:10AF9000CB6BCB51070842E3E351E15D3CE3E45165
:10AFA000E25D39E2C535EE6FC635EF6FEE37EF374C
:10AFB000EE37EF37F80EEE17036AE051EE25016E1B
:10AFC000EF5103220150760FE96E060E0320EA6E60
:10AFD000EFCF00F0CB51016E04E0D8900032012E8B
:10AFE000FCD700A017D0036A026A016A010E006E46
:10AFF000E251EE6F07E0D890003601360236033694
:10B00000EE2FF9D70050DC130150DD130250DE1390
:10B010000350DF13E22BE12BCB2BBBD7E02BB5D7B3
:10B02000DFC6F1F6DEC6F0F6DDC6EFF6DCC6EEF6FC
:10B03000000123EC33F003C0E9F602C0E8F601C0DA
:10B04000E7F600C0E6F6E9C656F7E8C655F7E7C6E4
:10B0500054F7E6C653F7D7C65AF7D6C659F7D5C63A
:10B0600058F7D4C657F7AFEC11F003C0E9F602C0A9
:10B07000E8F601C0E7F600C0E6F6D892E9C65AF74E
:10B08000E8C659F7E7C658F7E6C657F7DBC65EF7D6
:10B09000DAC65DF7D9C65CF7D8C65BF773EC10F07B
:10B0A00003C0E9F602C0E8F601C0E7F600C0E6F624
:10B0B000D8900601C535026EC635036E0250870F63
:10B0C000E96E060E0320EA6EECCFEFF6ED52EFCFFD
:10B0D000EEF6EE5368E1EF5366E1E551030BFC0F2A
:10B0E00061E2040F000196EF5AF00601CA6BC96BCA
:10B0F00059D0E9C648F7E8C647F7E7C646F7E6C6B7
:10B1000045F7CFC64CF7CEC64BF7CDC64AF7CCC6EF
:10B1100049F736EC10F006E1030E0601CA6FC96963
:10B1200004D000010601CA6BC96B3CD0CFC648F7FA
:10B13000CEC647F7CDC646F7CCC645F7E9C64CF7AD
:10B14000E8C64BF7E7C64AF7E6C649F736EC10F013
:10B1500006E3030E0601CA6FC96904D000010601A7
:10B16000CA6BC96B1FD0CFC648F7CEC647F7CDC64E
:10B1700046F7CCC645F7E9C64CF7E8C64BF7E7C635
:10B180004AF7E6C649F736EC10F001E206E1030E95
:10B190000601CA6FC96904D000010601CA6BC96BF8
:10B1A00001D006016BD0E5510C0B006E003200326D
:10B1B0003F0E00160050FC0F61E2040F0001A7EFE4
:10B1C0005AF00601CA6BC96B59D0E9C648F7E8C600
:10B1D00047F7E7C646F7E6C645F7D3C64CF7D2C6EB
:10B1E0004BF7D1C64AF7D0C649F736EC10F005E167
:10B1F0000601CA6BC96B05D00001030E0601CA6FB8
:10B20000C9693CD0E9C648F7E8C647F7E7C646F73C
:10B21000E6C645F7D3C64CF7D2C64BF7D1C64AF7B8
:10B22000D0C649F736EC10F005E30601CA6BC96BCE
:10B2300005D00001030E0601CA6FC9691FD0E9C617
:10B2400048F7E8C647F7E7C646F7E6C645F7D3C668
:10B250004CF7D2C64BF7D1C64AF7D0C649F736EC01
:10B2600010F001E205E10601CA6BC96B05D00001CF
:10B27000030E0601CA6FC96901D0060104D000019E
:10B280000601CA6BC96B010133D1C5C6F3F6060EC0
:10B290000601F56F860EF46F0001A2EC13F0015069
:10B2A000010B0108D8A419D10601C535026EC635B7
:10B2B000036E023603360236033602360336023692
:10B2C0000336E00E02160250B40FEE6F020E03209A
:10B2D000EF6F060EEE27000EEF23F2CFF0F6F29E90
:10B2E000EFC675FFEEC674FF7F9C7F9E7F80735014
:10B2F000F0BFF28EE36FC535026EC635036E0236BF
:10B300000336023603360236033602360336E00EC3
:10B3100002160250B40FEE6F020E0320EF6F050EFF
:10B32000EE27000EEF23F2CFF0F6F29EEFC675FF88
:10B33000EEC674FF7F9C7F9E7F807350F0BFF28EBD
:10B34000E46FDF6BDE6BDD6BDC6BE16BE26BDF6BA5
:10B35000DE6BDD6BDC6BE06BE051070848E3CB6B29
:10B36000CB51070842E3E351E15D3CE3E451E25D88
:10B3700039E2C535EE6FC635EF6FEE37EF37EE3792
:10B38000EF37F80EEE17036AE051EE25016EEF512C
:10B3900003220150760FE96E060E0320EA6EEFCF0E
:10B3A00000F0CB51016E04E0D8900032012EFCD7A2
:10B3B00000A017D0036A026A016A010E006EE25112
:10B3C000EE6F07E0D8900036013602360336EE2FD6
:10B3D000F9D70050DC130150DD130250DE13035087
:10B3E000DF13E22BE12BCB2BBBD7E02BB5D7ED6BDB
:10B3F000EC6BEB6B010EEA6FE451EE6F07E0D89057
:10B40000EA37EB37EC37ED37EE2FF9D7010EEA5F6D
:10B41000000EEB5BEC5BED5BDFC6F1F6DEC6F0F633
:10B42000DDC6EFF6DCC6EEF6000123EC33F003C018
:10B43000E9F602C0E8F601C0E7F600C0E6F6EDC6A0
:10B44000F1F6ECC6F0F6EBC6EFF6EAC6EEF623EC44
:10B4500033F0E9C656F7E8C655F7E7C654F7E6C62F
:10B4600053F703C05AF702C059F701C058F700C09C
:10B4700057F7E0EC13F003C0E9F602C0E8F601C0AC
:10B48000E7F600C0E6F6E9C656F7E8C655F7E7C6A0
:10B4900054F7E6C653F707015A6BC00E596F7F0E7B
:10B4A000586F880E576F0001AFEC11F003C0E9F63A
:10B4B00002C0E8F601C0E7F600C0E6F6E9C6F1F61C
:10B4C000E8C6F0F6E7C6EFF6E6C6EEF62AEC12F0AE
:10B4D00002C0CAF601C0C9F604D00601CA6BC96B26
:10B4E0000001010105D000010601CA6BC96B010111
:10B4F000D8900601C535026EC635036E0250870F1F
:10B50000E96E060E0320EA6ECAC6ECFFED52C9C60C
:10B51000EFFFC8AF05D0FF0ED880C957030ECA573A
:10B52000C9C601F0CAC602F000011200E824F76A99
:10B53000F736470FF66EB50EF7220A00F550FA6E91
:10B540000800F550F96EEAB0F2B02CB166B1E8240B
:10B55000F76AF736690FF66EB50EF7220A00F55056
:10B56000FA6E0800F550F96EC2B1CAB104B23EB22B
:10B57000F86AD09E078E19901A6A1B6A4E6A4F6A43
:10B5800001015C6B606B5F6B5E6B5D6B646B636B2F
:10B59000626B616B1992666B656B1994686B676B74
:10B5A000FE0E6A6F69696B6B6D6B6C6B6E696F6BAE
:10B5B0000301046F0369640E0D6F0E6B19961998E1
:10B5C000199A199C320E0601676F8F69630E996F85
:10B5D000199E9B6B9C6B9D919F6B9E6BA06BA16B4F
:10B5E000A56BA46B0F015C51800B5C6F000E5D6F4F
:10B5F000C196C198C19A5E6B5F6B20D00541CFFFA9
:10B600000841DE000402DEFFFFFFFF0942FA0008E6
:10B610000305FFFEFFFEFFFEFFFE10430F0004C008
:10B62000FF01800010465700040668000000000972
:10B63000468600040690000000000000000EF86E30
:10B64000B50EF76EFC0EF66E0900F550006E000A9E
:10B6500013E00900F550016EE8BE05D03F0BEA6E1D
:10B660000900F5CFE9FF01BC090001AC0900F5CFE5
:10B67000EEFF004EE9D7F9D7F86A320E0601A66F41
:10B68000050EA76FA891A893A895A897A899A89B1D
:10B69000A89D010EB96FA89FBA6BBF6BBE6BC06B44
:10B6A000C16BC291C293C369640EC46FC295D36A61
:10B6B000400E9B6E646AC00E0F015B6FF19E5C5181
:10B6C000800B03095C6FDF0E5D6FC196C198C19A54
:10B6D000C050C00B3709C06EC08EC28001016F35EB
:10B6E000006E0036FC0E0016C250830B0010C26EB6
:10B6F000000E016EC150F80B0110C16E95988C9828
:10B700000C0EBB6EBE6ABF6A010E9C6E999094943B
:10B710008B940C0E0F01506F9992BC6A516B700E96
:10B720000609CA6EFF0ECB6E370ECD6EAA6A9D80DB
:10B73000B10ECF6EE00ECE6E1990B06A370EB16EBC
:10B74000B36AB26AA082F288C00EF2120001BAECAB
:10B7500006F001C09AF606019A5312E100013AEF91
:10B760000BF00601C56B0001B2EC0DF009EF0EF015
:10B7700028EF0EF0B7EF0EF0DCEF0FF01AD0060155
:10B78000BC6B010EBB6FBC530FE1BB5104080CE353
:10B79000BBC6CFF6030ED06F0001AEEC09F0060178
:10B7A000BB2BD8B4BC2BEFD7010EC56F0001B2EC98
:10B7B0000DF0040019A03DD119900601A65302E036
:10B7C000A60703D0320EA66FA871A75302E0A70701
:10B7D00003D0050EA76FA873BC6BBB6BBC532BE1EA
:10B7E000BB510A0828E3D890BB35026EBC35036E06
:10B7F0000250340FE96E000E0320EA6EECCFC6F65D
:10B80000ED52EFCFC5F6C55302E1C65310E0D89014
:10B81000BB35026EBC35036E0250340FE96E000E6C
:10B820000320EA6EFF0EEF2602E2EE52ED06BB2B7E
:10B83000D8B4BC2BD3D7B95301E0B907BA5301E050
:10B84000BA07C45301E0C4071A5201E01A06BE53F6
:10B8500002E1BF5305E0BE51D8B4BF07BE0722D0F6
:10B86000C1531CE0C2B10ED0C151C05D05E3010E51
:10B87000C06F9CC6C1F601D0C02BBF6B190EBE6F46
:10B88000C2810BD0C151C05D04E3BF6BC80EBE6F57
:10B8900003D0BF6B190EBE6FC29104D0C06BC291B2
:10B8A0009CC6C1F603010D5301E00D070E5301E0E4
:10B8B0000E0701016B5301E06B076C5302E16D53FE
:10B8C00004E06C51D8B46D076C070601BC6BBB6B10
:10B8D000BC5367E1BB51030864E3BB35C56FBC359E
:10B8E000C66FC537C637FC0EC517570EC525E96E9E
:10B8F000060EC621EA6EECCFC8F6ED52EFCFC7F6C2
:10B90000C75302E1C85313E0BB35C56FBC35C66FE2
:10B91000C537C637FC0EC517570EC525E96E060E8E
:10B92000C621EA6EFF0EEF2602E2EE52ED06BB35AF
:10B93000C56FBC35C66FC537C637FC0EC517020EBE
:10B94000C525016E000EC621036E0150570FE96E2A
:10B95000060E0320EA6EECCFC6F6ED52EFCFC5F629
:10B96000C55302E1C65319E0BB35C56FBC35C66F80
:10B97000C537C637FC0EC517020EC525016E000E71
:10B98000C621036E0150570FE96E060E0320EA6EC2
:10B99000FF0EEF2602E2EE52ED06BB2BD8B4BC2B15
:10B9A00097D7685302E1695304E06851D8B4690736
:10B9B00068076A5302E16B5304E06A51D8B46B071D
:10B9C0006A07905302E1915304E09051D8B4910773
:10B9D0009007925302E1935304E09251D8B4930735
:10B9E0009207675301E067078B5302E18C5304E031
:10B9F0008B51D8B48C078B078D5302E18E5304E032
:10BA00008D51D8B48E078D07995302E0990703D062
:10BA1000198E630E996F9E5302E19F5304E09E516D
:10BA2000D8B49F079E07A05301E0A007A88FC28348
:10BA300000010601B9530AE19A5308E1010EB96FFA
:10BA4000000103EF2BF032EF31F00601A8AF46D032
:10BA50009A5344E1A89F19A22FD060C1F1F65FC1AB
:10BA6000F0F65EC1EFF65DC1EEF6000123EC33F0B7
:10BA7000800E0701566F960E556F180E546F970E75
:10BA8000536F03C05AF702C059F701C058F700C0FE
:10BA900057F70001E0EC13F003C0F1F602C0F0F636
:10BAA00001C0EFF600C0EEF62AEC12F002C066F11B
:10BAB00001C065F105D006010101666B656B0001EF
:10BAC00066C1C6F665C1C5F63FEF33F0F5EF33F05A
:10BAD000FAEF35F0199401B0198406010001DEEF88
:10BAE00038F060BE2BD00F0130AF02D0000126D05D
:10BAF0000E0180AF04D07DB502D000011FD090AF01
:10BB000004D07DB702D0000119D0A0AF04D07DB918
:10BB100002D0000113D0B0AF04D07DBB02D0000131
:10BB20000DD0C0AF04D07DBD02D0000107D0D0AF92
:10BB300018EF61F07DBF18EF61F000010601C66BE0
:10BB40002C0EC56F60AE1FD0A35304E1F10E6F142D
:10BB50006F6E04D0E00E72141009726EB06BA353B6
:10BB600008E0AE9171BCAE81719C60501F0BAF6F4D
:10BB700009D0AE9171BEAE81719E60A403D0AF6B4F
:10BB800060B0AF2BB0D00F0130AF24D00601A3536B
:10BB900005E1F10E6F140A096F6E04D0E00E721405
:10BBA0001109726E010EB06FA3530AE0AE9171BC21
:10BBB000AE81719C0F0130511F0B0601AF6F09D090
:10BBC000AE9171BCAE81719C0F013051070B060123
:10BBD000AF6F89D00E0180AF14D07DB512D0E00ECA
:10BBE00072141209726E020E0601B06FAE9171BC32
:10BBF000AE81719C0E0180511F0B0601AF6F73D097
:10BC00000E0190AF14D07DB712D0E00E721413095C
:10BC1000726E030E0601B06FAE9171BCAE81719C65
:10BC20000E0190511F0B0601AF6F5DD00E01A0AF4A
:10BC300014D07DB912D0E00E72141409726E040E85
:10BC40000601B06FAE9171BCAE81719C0E01A05126
:10BC50001F0B0601AF6F47D00E01B0AF14D07DBBF4
:10BC600012D0E00E72141509726E050E0601B06F47
:10BC7000AE9171BCAE81719C0E01B0511F0B0601DB
:10BC8000AF6F31D00E01C0AF14D07DBD12D0E00E29
:10BC900072141609726E060E0601B06FAE9171BC79
:10BCA000AE81719C0E01C0511F0B0601AF6F1BD0FE
:10BCB0000E01D0AF14D07DBF12D0E00E7214170960
:10BCC000726E070E0601B06FAE9171BCAE81719CB1
:10BCD0000E01D0511F0B0601AF6F05D00E01000EF3
:10BCE000016E90D0060165500F0BAD6FB19165BC30
:10BCF000B181B19362B6B183000EB1B3010ECA6FC8
:10BD00000F0ED26F640ED16FCAC6D3F60001FDEFDD
:10BD100039F003C0ACF602C0ABF601C0AAF600C011
:10BD2000A9F60F0E0601C96F660EC86FC76BAD513D
:10BD3000C75D18E2C6C6CBF6C9C603F0C8C6E9FFA0
:10BD400003C0EAFFEFCFCCF6CBC6EAFFC5C6E9FFDA
:10BD5000CCC6EFFFC52BD8B4C62BC82BD8B4C92B83
:10BD6000C72BE5D7B051000A00010FE0010A16E029
:10BD7000030A19E0010A1CE0070A1FE0010A22E099
:10BD8000030A25E0010A28E02BD0609E0601A35398
:10BD900002E0779201D07790000122D00F01309F0E
:10BDA000779200011DD00E01809F7792000118D07C
:10BDB0000E01909F7792000113D00E01A09F779201
:10BDC00000010ED00E01B09F7792000109D00E0144
:10BDD000C09F7792000104D00E01D09F779200019E
:10BDE0000601B19577BEB185779EA35304E1F10EAC
:10BDF0006F146F6E04D0E00E72141009726E010E93
:10BE0000016E0E010601AAC6B2F6ABC6B3F6AC517E
:10BE1000010BB46FB56BA9C6B6F6640EBA6FB2511A
:10BE200004081FE1B351F0081CE1B4531AE1B55303
:10BE300018E130C06AF12FC069F101016A51FE08B2
:10BE40000CE303E16951FE0808E36A3369336A339E
:10BE500069336A3369331F0E6A17140E6B6FE6D0AD
:10BE600006011BC001F0EA0E036E1B50B25D07E134
:10BE70000350B35D04E1B45302E1B55309E0B23DB0
:10BE800049D0B351EA0846E1B45344E1B55342E125
:10BE90002DC0B8F62CC0B7F6B751006EB851036E7E
:10BEA000FE0E035C05E1DA0E005C000122E00601F3
:10BEB000FD0E035C05E1C50E005C00011DE00601FE
:10BEC000FF0E035C05E1F20E005C000118E00601C4
:10BED000FF0E035C05E1F00E005C000113E00601BB
:10BEE000FF0E035C05E1F10E005C000110E00601AD
:10BEF00010D00601A8850DD00601A8870AD006013A
:10BF0000A88907D0B6C6BDF60601A88B02D00601E7
:10BF1000A88D8AD0B351EC082BE1B2511B5C28E10B
:10BF20002C50100A000107E0010A1CE0020A1BE085
:10BF3000EC0A1AE01BD0B6C624F32EC026F32DC09F
:10BF400025F32FC027F303012B6B33C02AF332C034
:10BF500029F331C028F30601566B556B000106EF3B
:10BF60003BF004D003D002D0199619985ED0060198
:10BF7000B351EB0859E1B2511B5C56E119A654D0FC
:10BF80002C5003012C5DD8B402D006014DD006011F
:10BF9000BC6B010EBB6FBC5329E1BB51070826E304
:10BFA000565103081FE303E1555126081BE356C60B
:10BFB000C6F65551552BD8B4562BC56F2D0EC52539
:10BFC000016E030EC621036E2C0EBB25E96E000E1A
:10BFD000BC21EA6EEFCFC9F603C0EAFF01C0E9FF5A
:10BFE000C9C6EFFFBB2BD8B4BC2BD5D703012C2B74
:10BFF0002C51275D1AE2000122EF3BF0015210E0C4
:10C00000BAEC06F001C09AF606019A5304E09BC60A
:10C01000C3F6198C01D0198A050E1A6E05D00001DD
:10C02000010E0601C36F198C0301010106016C3D6D
:10C0300007D06D3D05D06E3D03D06F3D01D06AD075
:10C04000C56BAAC6C6F6ABC6C7F6AC51010BC86F26
:10C050006CC6C9F66DC6CAF66E51010BCB6FCC6BC0
:10C06000036E6DC602F06CC601F0006A0050C55D3B
:10C0700051E10150C65D4EE10250C75D4BE10350F6
:10C08000C85D48E1B651745D02E0743D43D0BC6BBD
:10C09000BB6BBC531EE1BB5107081BE3760EBB25EF
:10C0A000016E060EBC21036E01C0C5F6C66F2C0ED4
:10C0B000BB25E96E000EBC21EA6EEFCFC7F603C0C8
:10C0C000EAFF01C0E9FFC7C6EFFFBB2BD8B4BC2B0A
:10C0D000E0D78681F2CFC5F6F29E020E756EB50EE0
:10C0E000746E7F9C7F9E7F807350C5BFF28E7F0BE6
:10C0F0008B6F8C6B8CC642F78BC641F70701446B84
:10C10000640E436F0001A9EC06F002C08CF601C07A
:10C110008BF60601703D07D0713D05D0723D03D00E
:10C12000733D01D06AD0C56BAAC6C6F6ABC6C7F6CA
:10C13000AC51010BC86F70C6C9F671C6CAF6725110
:10C14000010BCB6FCC6B036E71C602F070C601F0B1
:10C15000006A0050C55D51E10150C65D4EE10250DC
:10C16000C75D4BE10350C85D48E1B651755D02E023
:10C17000753D43D0BC6BBB6BBC531EE1BB51070884
:10C180001BE37E0EBB25016E060EBC21036E01C0B3
:10C19000C5F6C66F2C0EBB25E96E000EBC21EA6EFB
:10C1A000EFCFC7F603C0EAFF01C0E9FFC7C6EFFF44
:10C1B000BB2BD8B4BC2BE0D78683F2CFC5F6F29E5A
:10C1C000020E756ED50E746E7F9C7F9E7F807350BD
:10C1D000C5BFF28E7F0B8D6F8E6B8EC642F78DC6FC
:10C1E00041F70701446B640E436F0001A9EC06F0B0
:10C1F00002C08EF601C08DF60601B2519F0817E10C
:10C20000B33D15D0B45313E1B55311E1AD51070857
:10C210000EE12C50FA080BE12D50DC0808E19F6B71
:10C22000320E9E6F9D81000101EF3CF006010E0170
:10C2300001016B5303E1FE0E6A6F6969F2CFC5F627
:10C24000F29E020E756EB50E746E7F9C7F9E7F808F
:10C2500073500601C5BFF28E7F0B000A05E08B53B9
:10C2600003E18C5301E18691F2CFC5F6F29E020EF6
:10C27000756ED50E746E7F9C7F9E7F807350C5BF98
:10C28000F28E7F0B000A05E08D5303E18E5301E12E
:10C2900086939E2D04D09F5302E1010E1A6E9DB12C
:10C2A00014D0675311E19A530FE10001B8EF3FF04A
:10C2B0003E5209E13F5207E13F6A640E3E6E7EEF57
:10C2C00049F0FCEF4AF0060104D000011EEF4DF0EA
:10C2D000060100012DEF50F00601C2B502D08B9E81
:10C2E00001D08B8E949E006AC2B5002A010E001AFE
:10C2F000C29500B0C285A8A50ED0A895C56BC76B26
:10C300006A0EC66FFE0EC96FDA0EC86FCA690001E9
:10C31000EDEC51F00601A8A70FD0A897010EC56F4C
:10C32000C76B140EC66FFD0EC96FC50EC86FCA6904
:10C330000001EDEC51F00601A8A905D0A899000173
:10C3400031EF55F00601A8AB10D0A89B020EC56FC7
:10C35000030EC76F260EC66FC969F00EC86FBDC643
:10C36000CAF60001EDEC51F00601A8AD21D0A89D60
:10C370009AC624F09BC625F01BC0C5F6F10EC66F09
:10C38000FF0EC76F180EC86FF66FC7C6F5F6C6C6A4
:10C39000F4F61BC0F3F6F86B240EF76F020EF96F7C
:10C3A000FA6F010EFB6FFC6B00013AEC3FF00601E7
:10C3B00019A805D0199800018FEF55F0060119AAA8
:10C3C00008D0199A010EC56FC6690001BAEC55F084
:10C3D000060119AC08D0199CC56BC3C6C6F600018E
:10C3E000BAEC55F006010F0120A728D010A726D0DF
:10C3F00000A724D00E0180B704D07DA502D00F0184
:10C400001DD090B704D07DA702D00F0117D0A0B7E0
:10C4100004D07DA902D00F0111D0B0B704D07DABFC
:10C4200002D00F010BD0C0B704D07DAD02D00F01F8
:10C4300005D0D0B707D07DAF05D00F01640E06013F
:10C44000C46F0E010601C2A33AD09A5338E19DB1E0
:10C4500036D0C293C66BC56B0001E9EC55F002C043
:10C46000C6F601C0C5F60601C633C533C633C533AB
:10C47000C633C5C6BCFFC633C631300B006EBB50D9
:10C48000CF0B0010BB6EC66B010EC56F0001E9EC4F
:10C4900055F002C0C6F601C0C5F60601C633C53365
:10C4A000C633C533C633C5C651FFC633C631300B9C
:10C4B000006E0F015051CF0B0010506F06019DB15F
:10C4C0002CD003010E5304E0010E06019C6F07D02F
:10C4D00006019A5303E09AC69CF601D09C6B9C53CC
:10C4E00015E1C45307E1A8B302D08C9E01D08C8E15
:10C4F000959E0BD0BA5307E1A8B102D08C9E01D013
:10C500008C8E959E02D0959E8C8E06D0C2B102D0A4
:10C510008C9E01D08C8E959E02D0959E8C8E1A2C6E
:0EC5200001D003D00001D9EF5BF0FF00030053
:04FFBC0053656E64B7
:10FFC000657243414E20506C75732056632020208B
:10FFD00000FF563030312E78782032342D4175674D
:10FFE0002D32322032303A31353A333900FF37384A
:10FFF0002E37302E3036383320202020202000FFAE
:020000040030CA
:0E00000015C36617008991000FC00FE00F4076
:00000001FF
